:100000000C9470120C94A1120C94A1120C94A112D5
:100010000C94A1120C94A1120C94A1120C94A11294
:100020000C94A1120C94A1120C94A1120C94A11284
:100030000C94A1120C948CCB0C94A1120C94A112D0
:100040000C94A1120C947C6D0C94A1120C94A1122E
:100050000C94A1120C94A1120C944F7E0C947AC5AE
:100060000C94A1120C949B160C94A1120C94A11246
:100070000C94A1120C94A1120C94A1120C94A11234
:100080000C94A1120C94A1120C94A1120C94A11224
:100090000C94A1120C94A1120C94A1120C94A11214
:1000A0000C94A1120C94A1120C94A1120C94A11204
:1000B0000C94A1120C94A1120C94A1120C94A112F4
:1000C0000C94A1120C94A1120C94A1120C94A112E4
:1000D0000C94A1120C94A1120C94A1120C94A112D4
:1000E0000C94A112C67ED57EF17E007F1A7F297FF7
:1000F000437F477FFFBE1CBF1EBF2ABF30BF33BF39
:100100003DBFB0C6B5C6BAC6C4C6CEC647C7D8C6B8
:10011000E0C6E8C6F2C6FCC606C715C71FC747C774
:1001200029C733C73DC769C76CC75BC75FC765C70A
:10013000A3C770C774C77AC77EC782C788C78CC772
:1001400090C7A3C796C79AC79EC7084AD73B3BCE5E
:10015000016E84BCBFFDC12F3D6C74319ABD5683C6
:100160003DDA3D00C77F11BED9E4BB4C3E916BAA7E
:10017000AABE000000803F05A84CCDB2D44EB938CD
:1001800036A9020C50B9918688083CA6AAAA2ABEB4
:10019000000000803F0048617264636F6465642002
:1001A00044656661756C742053657474696E677319
:1001B000204C6F616465640053746F7265642073D2
:1001C000657474696E6773207265747269657665AB
:1001D000640053657474696E67732053746F72653D
:1001E00064006563686F3A004B494C4C45442E20CF
:1001F000005072696E7465722068616C7465642E5B
:10020000206B696C6C28292063616C6C656421002B
:100210006F6B00526573656E643A20002200556E64
:100220006B6E6F776E20636F6D6D616E643A202226
:10023000004D323230362020444F4E45004D323290
:100240003036004D3035004D3035004D30330047ED
:1002500031205A383020463138303000473238208B
:100260005A30004D3035006F6B20506C65617365FE
:1002700020776561722070726F746563746976654A
:1002800020676C617373657320666F722074686594
:10029000206E65787420737465702E00486F7465E5
:1002A0006E64206F6666736574733A007A5F6D6979
:1002B0006E3A2000795F6D696E3A2000785F6D6953
:1002C0006E3A20005A3A00593A0020436F756E7416
:1002D00020583A00453A005A3A00593A00583A0034
:1002E0004649524D574152455F4E414D453A4D5456
:1002F000325F33445072696E7465725F50524F477B
:1003000052414D2056455253494F4E3A312E3131CC
:10031000322045585452554445525F434F554E5430
:100320003A32204D414348494E455F545950453A71
:100330005265705261702020576562736974653A26
:10034000687474703A2F2F7777772E6D756C746F91
:100350006F2E636F6D200A0042656420646F6E65C6
:100360002E0020423A002054313A0054303A0042E4
:1003700065642048656174696E672E004865617424
:10038000696E6720646F6E652E0020573A00205416
:10039000313A0054303A0048656174696E672E2E18
:1003A0002E002042403A0020403A00202F002042F8
:1003B0003A00202F002054313A00202F006F6B208C
:1003C000543A002569206D696E2C202569207365DB
:1003D0006300456E642066696C65206C6973740007
:1003E000426567696E2066696C65206C697374008C
:1003F0004E6F206D6F76652E005072696E74696E57
:1004000067202E2E2E005761697420666F7220754A
:100410007365722E2E2E004732382020616C726573
:100420006164792070726F6365737365640047322D
:10043000382020736B697020746869732066696C5A
:100440006500536C6565702E2E2E0046696E6973CB
:100450006865642E00446F6E65207072696E746901
:100460006E672066696C6500473332310053544F24
:10047000505045442E20005072696E74657220738E
:10048000746F707065642064756520746F20657288
:10049000726F72732E2046697820746865206572C9
:1004A000726F7220616E6420757365204D39393921
:1004B00020746F20726573746172742E20285465E5
:1004C0006D706572617475726520697320726573F1
:1004D00065742E205365742069742061667465729A
:1004E0002072657374617274696E6729006F6B00A6
:1004F0004E6F204C696E65204E756D626572207777
:1005000069746820636865636B73756D2C204C613A
:100510007374204C696E653A20004E6F2043686505
:10052000636B73756D2077697468206C696E6520E4
:100530006E756D6265722C204C617374204C696E0F
:10054000653A2000636865636B73756D206D697330
:100550006D617463682C204C617374204C696E6506
:100560003A20004C696E65204E756D626572206997
:1005700073206E6F74204C617374204C696E65201B
:100580004E756D6265722B312C204C617374204C5A
:10059000696E653A20004D31313000446F6E652040
:1005A000736176696E672066696C652E006F6B00FB
:1005B0004D3239002020506C616E6E657242756656
:1005C00066657242797465733A20002046726565EB
:1005D000204D656D6F72793A2000446563202039A3
:1005E000203230313700436F6D70696C65643A209A
:1005F000004D554C544F4F00207C20417574686F5E
:10060000723A20004465632020392032303137208F
:1006100031313A31303A323000204C617374205518
:100620007064617465643A20004D54320020536F49
:100630006674776172652052657365740020576136
:10064000746368646F67205265736574002042723A
:100650006F776E206F757420526573657400204546
:10066000787465726E616C20526573657400506FAA
:100670007765725570007374617274002200656E44
:10068000717565696E672022002200656E7175655F
:10069000696E67202200FFFFFF0000A0400000A05D
:1006A000400000803F00000000000000000000004B
:1006B000006563686F3A004572726F723A007C3C65
:1006C0003E5E2B3D3F2F5B5D3B2C2A225C004D386C
:1006D0003420582059205A2045004D3234004D32E4
:1006E00033202573006175746F25692E670065726C
:1006F000726F722077726974696E6720746F2066FA
:10070000696C65004E6F74205344207072696E747A
:10071000696E67002F005344207072696E74696EB1
:1007200067206279746520002E0044656C657469E9
:100730006F6E206661696C65642C2046696C653A51
:10074000200046696C652064656C657465643A00D8
:100750002E006F70656E206661696C65642C2046A2
:10076000696C653A200057726974696E6720746F0E
:100770002066696C653A20002E006F70656E2066F9
:1007800061696C65642C2046696C653A20002E0016
:100790006F70656E206661696C65642C2046696CBB
:1007A000653A200046696C652073656C6563746505
:1007B00064002053697A653A200046696C65206FB1
:1007C00070656E65643A20002E006F70656E20665D
:1007D00061696C65642C2046696C653A20006F7015
:1007E000656E46696C65202E2E2E2E2E2E66616952
:1007F0006C0053442063617264206F6B006F7065FE
:100800006E526F6F74206661696C656400766F6C00
:10081000756D652E696E6974206661696C6564002A
:10082000534420696E6974206661696C0065636871
:100830006F3A004572726F723A0020746F6F206CCD
:100840006F6E6720657874727573696F6E20707251
:100850006576656E7465640020636F6C64206578EE
:1008600074727573696F6E2070726576656E7465EB
:1008700064006563686F3A00656E6473746F7073CB
:10088000206869743A205A00205A3A00656E6473F1
:10089000746F7073206869743A20590020593A00C7
:1008A000656E6473746F7073206869743A205800C1
:1008B00020583A00656E6473746F707320686974B1
:1008C0003A200024F4D43050C38E20C2A2401782B4
:1008D0008B7011127A910D816CD90AA861E108C759
:1008E000586607615143061E4B5D05C145A7041AB2
:1008F000411104093D9803713931034036DB02652B
:10090000339102D4305402802E1D02632CEE017507
:100910002AC501B028A001102781018F2564012B71
:10092000244B01E0223401AC211F018D200D0180F8
:100930001FFC00841EED00971DDF00B81CD200E6EE
:100940001BC600201BBC00641AB200B219A8000A22
:1009500019A0006A189900D117910040178B00B5B3
:1009600016840031167E00B31579003A157300C75E
:10097000146F0058146A00EE136600881363002594
:10098000135E00C7125B006C12570015125400C1B1
:1009900011510070114F0021114B00D61049008DEC
:1009A0001047004610440002104200C00F40008073
:1009B0000F3E00420F3C00060F3B00CB0E38009369
:1009C0000E37005C0E3500270E3400F30D3200C1E7
:1009D0000D3100900D3000600D2E00320D2D000500
:1009E0000D2C00D90C2B00AE0C2900850C29005CC5
:1009F0000C2700350C27000E0C2600E80B2400C441
:100A00000B2400A00B23007D0B23005A0B2100397F
:100A10000B2100180B2000F80A1F00D90A1E00BB8A
:100A20000A1E009D0A1D00800A1D00630A1C004763
:100A30000A1B002C0A1B00110A1A00F7091A00DD14
:100A4000091900C4091900AB091900920917007BA4
:100A5000091800630917004C091600360916002012
:100A60000916000A091500F5081500E0081400CC65
:100A7000081400B8081400A4081400900813007D9E
:100A80000812006B081300580812004608120034C0
:100A9000081100230811001208110001081100F0CC
:100AA000071000E0071000D0071000C0071000B0CA
:100AB000070F00A107100091070E0083070F0074B5
:100AC000070F0065070E0057070E0049070E003B91
:100AD000070D002E070E0020070D0013070D00065E
:100AE000070D00F9060C00ED060D00E0060C00D421
:100AF000060C00C8060C00BC060C00B0060C00A4D6
:100B0000060B0099060C008D060B0082060B007781
:100B1000060B006C060B0061060A0057060B004C22
:100B2000060A0042060A0038060A002E060A0024B9
:100B3000060A001A060A001006090007060A00FD48
:100B4000050900F4050900EB050900E2050900D9D3
:100B5000050900D0050900C7050900BE050900B553
:100B6000050800AD050800A50509009C05080094CE
:100B70000508008C050800840508007C0508007441
:100B80000508006C050700650508005D05070056AF
:100B90000508004E05070047050700400508003816
:100BA000050700310507002A050700230507001C7B
:100BB000050600160507000F0507000805060002D8
:100BC000050700FB040600F5040700EE040600E834
:100BD000040600E2040700DB040600D5040600CF8B
:100BE000040600C9040600C3040600BD040600B7DD
:100BF000040600B1040500AC040600A6040600A02B
:100C00000405009B04060095040500900406008A74
:100C100004050085040500800406007A04050075BB
:100C2000040500700405006B0405006604050061FE
:100C30000405005C04050057040500520405004D3E
:100C400004050048040500430405003E0404003A7E
:100C500004050035040500300404002C04050027B9
:100C6000040400230405001E0404001A04040016F2
:100C7000040500110404000D040400090405000427
:100C800004040000040400FC030400F8030400F45E
:100C9000030400F0030400EC030400E8030400E490
:100CA000030400E0030400DC030400D8030400D4C0
:100CB000030400D0030400CC030400C8030300C5F0
:100CC00003030024F404D9201BC40C5C0E9804C454
:100CD000095F0265077101F405F900FB04B30048E0
:100CE000048700C10369005803550003034500BE93
:100CF000023A008402310053022A0029022500042E
:100D0000022000E4011C00C8011900AF011700987F
:100D100001140084011300710110006101100051E1
:100D2000010E0043010D0036010B002B010B0020CA
:100D3000010B00150109000C01090003010800FB6B
:100D4000000800F3000800EB000700E4000600DEE6
:100D5000000600D8000600D2000600CC000500C73F
:100D6000000500C2000500BD000400B9000400B584
:100D7000000400B1000400AD000400A9000400A5B7
:100D8000000300A20003009F0004009B00030098E2
:100D90000003009500020093000300900003008D03
:100DA0000002008B0003008800020086000200841D
:100DB000000300810002007F0002007D0002007B32
:100DC0000002007900020077000100760002007442
:100DD00000020072000100710002006F0002006D4D
:100DE0000001006C0002006A000100690002006757
:100DF000000100660001006500010064000200625D
:100E000000010061000100600001005F0002005D60
:100E10000001005C0001005B0001005A0001005964
:100E20000001005800010057000100560001005564
:100E30000001005400010053000000530001005263
:100E400000010051000100500001004F0001004E60
:100E50000000004E0001004D0001004C0001004B5D
:100E60000000004B0001004A000100490001004859
:100E70000000004800010047000100460000004655
:100E8000000100450000004500010044000100434E
:100E90000000004300010042000000420001004148
:100EA00000000041000100400001003F0000003F41
:100EB0000001003E0000003E0001003D0000003D3A
:100EC0000001003C0000003C0000003C0001003B31
:100ED0000000003B0001003A0000003A0001003928
:100EE0000000003900010038000000380000003820
:100EF0000001003700000037000100360000003616
:100F0000000000360001003500000035000000350B
:100F10000001003400000034000000340001003300
:100F200000000033000000330001003200000032F6
:100F300000000032000100310000003100000031EB
:100F40000001003000000030000000300001002FE0
:100F50000000002F0000002F0000002F0001002ED5
:100F60000000002E0000002E0001002D0000002DCA
:100F70000000002D0000002D0001002C0000002CBE
:100F80000000002C0000002C0001002B0000002BB2
:100F90000000002B0000002B0001002A0000002AA6
:100FA0000000002A0000002A00010029000000299A
:100FB000000000290000002900000029000100288D
:100FC0000000002800000028000000280000002881
:100FD0000001002700000027000000270000002774
:100FE0000000002700010026000000260000002667
:100FF000000000260000002600010025000000255A
:10100000000000250000002500000025000000254C
:10101000000100240000002400000024000000243F
:101020000000002400010023000000230000002332
:101030000000002300000023000000230000002324
:101040000001002200000022000000220000002217
:101050000000002200000022000100210000002109
:1010600000000021000000210000002100000021FC
:1010700000000021000100200000002000000020EE
:1010800000000020000000200000002000000020E0
:10109000000000200001001F0000001F0000001FD2
:1010A0000000001F0000001F0000001F0000001FC4
:1010B0000001001E0000001E0000001E0000001EB7
:1010C0000000006563686F3A00202D20496E76614C
:1010D0006C6964206578747275646572206E756DD4
:1010E000626572202100504944204175746F747507
:1010F0006E652066696E6973686564202120506C96
:1011000061636520746865204B702C204B692061F9
:101110006E64204B6420636F6E7374616E74732011
:10112000696E2074686520636F6E666967757261A9
:1011300074696F6E2E6800504944204175746F7455
:10114000756E65206661696C6564212074696D65E2
:101150006F75740020403A006F6B20543A006F6B3B
:1011600020423A00504944204175746F74756E6591
:10117000206661696C6564212054656D70657261DB
:101180007475726520746F206869676800204B640D
:101190003A2000204B693A2000204B703A20002072
:1011A000436C617369632050494420002054753AB0
:1011B0002000204B753A2000206D61783A200020F5
:1011C0006D696E3A200020643A20002062696173E4
:1011D0003A20004572726F723A00A0007201B000AE
:1011E0006D01B0006801C0006301D0005E01D00055
:1011F0005901E0005401F0004F0100014A011001C3
:1012000045012001400130013B01400136016001F0
:10121000310170012C0190012701B0012201C001B0
:101220001D01F00118011002130130020E016002CD
:10123000090190020401C002FF000003FA0040030C
:10124000F5008003F000D003EB002004E6007004FA
:10125000E100E004DC004005D700C005D2004006F4
:10126000CD00D006C8008007C3003008BE00F008DB
:10127000B900C009B400B00AAF00B00BAA00D00C8E
:10128000A500000EA000500F9B00C0109600501249
:10129000910000148C00C0158700B0178200B019AF
:1012A0007D00D01B7800001E730040206E0090224D
:1012B0006900F024640040275F0090295A00E02B69
:1012C0005500102E500020304B0010324600E03305
:1012D000410090353C001037370070383200A0399B
:1012E0002D00B03A2800A03B2300603C1E00103DBA
:1012F0001900903D1400103E0F00703E0A00C03EE1
:101300000500003F0000436172642072656D6F76D6
:101310006564004361726420696E7365727465640C
:10132000004D3234004D32332025730025730020E8
:1013300025730025730020257300517569740051D1
:10134000756974004E657874205061676500436F5D
:101350006D706C6574652053656C656374696F6E40
:10136000005072652050616765004D61696E004DE7
:101370003234004D3233202573004D30350050613A
:10138000757365642E004D6174657269616C2069C6
:1013900073206F75742E002D2D3A2D2D004D38348D
:1013A0000046494E495348004241434B004E455880
:1013B0005400466C6F7700466C6F770046616E2074
:1013C00073706565640046616E20737065656400C6
:1013D0004E6F7A7A6C6532004E6F7A7A6C653200A5
:1013E0004E6F7A7A6C65004E6F7A7A6C65004D6F3D
:1013F0007665004D6F7665004D61696E0053746FC0
:101400007265206D656D6F7279004E6F7A7A6C65CA
:10141000004E6F7A7A6C650046616E207370656568
:10142000640046616E20737065656400507265707B
:101430006172650053746F7265206D656D6F7279AE
:10144000004E6F7A7A6C65004E6F7A7A6C65004652
:10145000616E2073706565640046616E207370650F
:1014600065640050726570617265004865696768FF
:1014700074285A2900486569676874285A29004405
:101480006570746828592900446570746828592962
:10149000005769647468285829005769647468287B
:1014A0005829004D616368696E65205365747469DD
:1014B0006E6773005A204F6666736574005A204F3A
:1014C00066667365740059204F66667365740059CB
:1014D000204F66667365740058204F6666736574A6
:1014E0000058204F6666736574004D616368696ECD
:1014F000652053657474696E6773004531202D2033
:1015000059202D204F6666736574004531202D20CB
:1015100059202D204F6666736574004531202D20BB
:1015200058202D204F6666736574004531202D20AC
:1015300058202D204F6666736574004D616368699D
:101540006E652053657474696E677300436F6E66D1
:1015500069726D2053657474696E677300592D6FDD
:10156000757465722D41636300592D6F75746572D2
:101570002D416363004531206F6666736574207486
:101580006F204530004E6F7A7A6C65206F66667307
:10159000657420746F20426564004D616368696EF4
:1015A000652053697A65005072657061726500410B
:1015B000626F75742075730052657365742044659D
:1015C0006661756C74004F6666004F6E20004F6652
:1015D00066004F6E20004F6E65206279206F6E6549
:1015E000004D616368696E652053657474696E6748
:1015F0007300507265686561742041425320436FE7
:101600006E66005072656865617420504C412043DD
:101610006F6E660046616E2073706565640046619A
:101620006E207370656564004C6173657220456E51
:1016300067726176696E67204D6F646500436F6FF6
:101640006C646F776E00507265686561742041420A
:1016500053005072656865617420504C41004D6FB5
:101660007665204178697300473238205900486F09
:101670006D65205900473238205800486F6D65204D
:101680005800473238205A00486F6D65205A004D87
:1016900038340044697361626C65205374657070FE
:1016A000657273004D61696E004732380052657390
:1016B000756D65205072696E740047333232004791
:1016C0003332320046696E69736865642E004D38A6
:1016D00034004D383420582059205A2045004D6F91
:1016E000766520302E316D6D004D6F766520316D41
:1016F0006D004D6F76652031306D6D0050726570F4
:10170000617265005800590045787472756465729D
:1017100000457874727564657200457874727564FA
:1017200065722031004578747275646572203000EE
:101730004D6F7665205A004D6F76652059004D6FCC
:1017400076652058004D6F76652041786973005AA0
:10175000004D3035004D30330041626F7574207597
:101760007300536176652064697374616E6365000C
:10177000466F63616C2064697374616E63650046D3
:101780006F63616C2064697374616E636500547586
:10179000726E206F6666204C6173657200547572BC
:1017A0006E206F6E204C61736572004D6F76652000
:1017B0005A00473238205A3000486F6D65205A0071
:1017C0004D61696E204D656E75004E6F20436172EC
:1017D0006400456E67726176652066726F6D205396
:1017E0004420636172640053746F7020456E6772A9
:1017F0006176696E6700526573756D6520456E6729
:10180000726176696E6700506175736520456E6719
:10181000726176696E67004D3232303500536574FF
:10182000206261736520706F696E74004F626A6533
:10183000637420686569676874004F626A656374E1
:101840002068656967687400466F63616C20536542
:101850007474696E6773004D6F7665004D6F7665C1
:10186000004E6F2043617264005072696E7420668E
:10187000726F6D20534420636172640053746F7003
:10188000205072696E7400526573756D65205072D8
:10189000696E74005061757365205072696E7400D2
:1018A000506C617465204C6576656C696E670047A5
:1018B000323800486F6D6520616C6C005072657045
:1018C000617265004F6666004F6E20004F666600CD
:1018D0004F6E2000456E61626C652046570054755E
:1018E0006E6500507265706172650054756E6500BA
:1018F0005374617475732073637265656E00000BB9
:101900001000000D000000003039000D000D00092E
:101910000D1A0B0000FF80FF80C180C180C180C113
:1019200080C180C180C180C180C180FF80FF8004F0
:101930000D0D060000F0F0303030303030303030F7
:101940003030090D1A0A0000FF80FF8001800180FD
:101950000180FF80FF80C000C000C000C000FF8089
:10196000FF80090D1A0B0000FF80FF8001800180BD
:101970000180FF80FF800180018001800180FF8065
:10198000FF800B0D1A0D00000180038007800D8081
:10199000198031806180FFE0FFE0018001800180DB
:1019A0000180090D1A0A0000FF80FF80C000C000FE
:1019B000C000FF80FF800180018001800180FF80E6
:1019C000FF80090D1A0A0000FF80FF80C000C000E0
:1019D000C000FF80FF80C180C180C180C180FF80C6
:1019E000FF80090D1A0A0000FF80FF80018001803E
:1019F00001800180018001800180018001800180DF
:101A00000180090D1A0B0000FF80FF80C180C1809A
:101A1000C180FF80FF80C180C180C180C180FF8004
:101A2000FF80090D1A0B0000FF80FF80C180C1807C
:101A3000C180FF80FF800180018001800180FF80E4
:101A4000FF8000060900000701850308207FFE07CC
:101A5000FE07FE00000005000001070702000080ED
:101A6000808080800080030202040005A0A0060799
:101A700007060000C0D82420202418050707060008
:101A8000002078A07028F02007070708000042A473
:101A90004810244A8406050507000210387C10F01F
:101AA000FF030707040000204080808040200307D8
:101AB0000704000080402020204080050505060026
:101AC00000A870F870A80505050600002020F82081
:101AD000200203030300FF404080030101040002D1
:101AE000E0010202020000808005070706000008EE
:101AF000081020408080050707060000F8888888C5
:101B00008888F8020707030000C04040404040407A
:101B1000050707060000F80808F88080F8050707A1
:101B2000060000F80808F80808F80607070700008C
:101B300008182848FC0808050707060000F88080F8
:101B4000F80808F8050707060000F88080F888887C
:101B5000F8050707060000F8080808080808050740
:101B600007060000F88888F88888F8050707060047
:101B700000F88888F80808F8010505020000808050
:101B80000080800205050300FF40004040800505FD
:101B9000050600001860806018040303050001F0CA
:101BA00000F0050505060000C0300830C005070735
:101BB00007010070880810200020080707090000AE
:101BC0003C4299A999423C0507070600002050882D
:101BD000F8888888050707060000F08888F088885C
:101BE000F005070706000070888080808870050770
:101BF00007060000F08888888888F0040707050039
:101C000000F08080F08080F0040707050000F0807D
:101C100080F0808080050707060000708880B88803
:101C20008870050707060000888888F8888888017A
:101C300007070200008080808080808005070706FB
:101C400000000808080808887005070706000088D3
:101C500090A0C0A0908804070705000080808080C5
:101C60008080F007070708000082C6AA928282825D
:101C70000507070600008888C8A898888805070710
:101C800006000070888888888870050707060000AD
:101C9000F08888F08080800508080600FF7088883A
:101CA0008888887008050707060000F08888F08893
:101CB000888805070706000070888070088870050E
:101CC0000707060000F8202020202020050707062F
:101CD00000008888888888887005070706000088C3
:101CE000888888885020070707080000829292920F
:101CF00092926C050707060000888850205088885B
:101D000005070706000088885020202020050707C7
:101D1000060000F80810204080F8020707030000C2
:101D2000C08080808080C005070707010080804058
:101D300020100808020707030000C0404040404050
:101D4000C0FF050101060000F8FF050505060000BB
:101D500070087888780507070600008080F088887A
:101D600088F0050505060000708880887005070763
:101D700006000008087888888878050505060000B0
:101D80007088F88078030707030000608080C080B7
:101D900080800507070600FE788888887808300567
:101DA00007070600008080F08888888801070702FE
:101DB0000000800080808080800209090300FE40CE
:101DC00000404040404040800507070600008890E2
:101DD000A0C0A0908801070702000080808080805A
:101DE0008080070505080000EC9292929205050597
:101DF000060000F0888888880505050600007088C0
:101E00008888700507070600FEF0888888F08080C3
:101E10000507070600FE7888888878080804050505
:101E2000050000B0C08080800505050600007880B0
:101E30007008F00307070400004040E040404040C5
:101E400005050506000088888888780505050600D0
:101E50000088888850200705050800009292929219
:101E60006C05050506000088502050880507070608
:101E700000FE88888888780830050505060000F887
:101E8000102040F803070704000020404080404035
:101E90002001070702000080808080808080030787
:101EA0000704000080404020404080FFFF00000009
:101EB0000000000000000000000000000000000022
:101EC0000000000000000000000000000000000012
:101ED0000000000000000000000000000000000002
:101EE00000000000000000000000000000000000F2
:101EF00000000000000000000000000000000000E2
:101F000000000000000000000000000000000000D1
:101F100000000000000000000000000000000000C1
:101F200000000000000000000000000000000000B1
:101F300000000000000000000000000000000000A1
:101F4000701C606301FFC1F807E0000000000000A2
:101F5000701C606301FFC3FC0FF000000000000074
:101F6000783C606301FFC70E1C38000000000000D1
:101F7000783C6063000C0E07381C00000000000075
:101F8000783C6063000C0C03300C00000000000083
:101F90007C7C6063000C0C03300C0000000000002F
:101FA0006C6C6063000C0C03300C0000000000003F
:101FB0006C6C6063000C0C03300C0000000000002F
:101FC00066CC6063000C0C03300C000000000000C5
:101FD00067CC6063000C0C03300C000000000000B4
:101FE000638C70E3000C0E07381C0000000000003A
:101FF000638C3FC3FC0C070E1C380000000000007F
:10200000610C1F83FC0C03FC0FF0000000000000BB
:10201000610C0F03FC0C01F807E000000000000059
:1020200000000000000000000000000000000000B0
:1020300000000000000000000000000000000000A0
:102040000000000000000000000000000000000090
:102050000000000000000000000000000000000080
:102060000000000000000000000000000000000070
:102070000000000000000000000000000000000060
:102080000000000000000000000000000000000050
:102090000000000000000000000000000000000040
:1020A0000000000000000000000000000000000030
:1020B0000001E0071FFF83E00000000000000000B7
:1020C0000001F00F1FFF8FF800000000000000006B
:1020D0000001F00F1FFF9F780000000000000000CB
:1020E0000001F81F00E01C1C0000000000000000C0
:1020F0000001F81F00E0181C0000000000000000B4
:102100000001F81F00E0001C0000000000000000BB
:102110000001DC3B00E0001C0000000000000000AB
:102120000001DC3300E0001C0000000000000000A3
:102130000001DC3300E00038000000000000000077
:102140000001CE7300E000700000000000000000FD
:102150000001CE6300E000E000000000000000008D
:102160000001CE6300E001C000000000000000009C
:102170000001C66300E007800000000000000000CE
:102180000001C7C300E00F000000000000000000D5
:102190000001C7C300E01E000000000000000000B6
:1021A0000001C38300E01FFC0000000000000000ED
:1021B0000001C38300E01FFC0000000000000000DD
:1021C000000000000000000000000000000000000F
:1021D00000000000000000000000000000000000FF
:1021E00000000000000000000000000000000000EF
:1021F00000000000000000000000000000000000DF
:1022000000000000000000000000000000000000CE
:1022100000000000000000000000000000000000BE
:1022200000000000000000000000000000000000AE
:10223000000000000000000000000000000000009E
:10224000000000000000000000000000000000008E
:10225000000000000000000000000000000000007E
:10226000000000000000000000000000000000006E
:10227000000000000000000000000000000000005E
:10228000000000000000000000000000000000004E
:10229000000000000000000000000000000000003E
:1022A000000000000000000000000000000000002E
:1022B000000201000004008000080040001000201F
:1022C000002000100040000800FFFFFC00804804D0
:1022D00000804804008048040080480400804804CE
:1022E0000080480400FFCFFC000000000000000058
:1022F0000000000000000000000000000000300CA2
:10230000000060060000C00300018001800300009F
:10231000C0060000600C00003018000018300000FB
:102320000C600000067FFFFFFE7FFFFFFE600FF0E6
:1023300006600C3006600C3006600C3006600C3015
:1023400006600C3006600C30067FFC3FFE3FF81F35
:10235000FC00000000000000000000000000000081
:1023600000000000000000000000000000FFE0FF8F
:10237000D11000FFFEFFD0FFE0FFC1FFD140A0C899
:10238000A6A22FF800238127AC00AFFF64A5FF644D
:10239000FF64A4FFD0FFFE00000A0B02090C0D0E23
:1023A0000807030401000000000000000000000016
:1023B000000000000000000000000000000000001D
:1023C00000000012111000000000000000000000DA
:1023D00000000000000000000000000000010210EA
:1023E000202008081020401020408002010201082F
:1023F00004020101020408102040808040201008DF
:102400000402018004020180402010080402010837
:102410000402010102040810204080010204081097
:102420002040800505050507050808080802020286
:10243000020A0A080804040404010101010101015F
:10244000010303030303030303040707070C0C0C36
:102450000C0C0C0C0C02020202060606060606060E
:10246000060B0B0B0B0B0B0B0B000022002500289F
:10247000002B002E0031003400020100000501088D
:10248000010B0100002100240027002A002D00304C
:1024900000330001010000040107010A01024E415E
:1024A0004E494E495459494E46CDCCCC3D0AD723CE
:1024B0003C17B7D13877CC2B329595E6241FB14F16
:1024C0000A000020410000C84200401C4620BCBE5B
:1024D0004CCA1B0E5AAEC59D7400D7404CBDDB40A4
:1024E00011241FBECFEFD1E2DEBFCDBF00E00CBF95
:1024F00015E0A0E0B2E0E8EAFFEA01E00BBF02C0AD
:1025000007900D92A23EB107D9F725E1A2EEB5E002
:1025100001C01D92A634B207E1F714E2CEEDD4E279
:1025200000E006C022970109FE010BBF0E94F9D00E
:10253000CA3DD10780E00807A9F70E94ECCB0C94B4
:10254000C3D70C940000EF92FF920F931F93CF9389
:10255000DF931F92CDB7DEB78C017B01460FF701E9
:1025600061917F01F8018081918149830E940CD79C
:10257000F8018081918101969183808349814E1178
:10258000EECF0F90DF91CF911F910F91FF90EF90C1
:102590000895EF92FF920F931F93CF93DF931F92B3
:1025A000CDB7DEB78C017B01460FF80180819181A8
:1025B00049830E9404D7F70181937F01F80180814C
:1025C000918101969183808349814E11EECF0F90C6
:1025D000DF91CF911F910F91FF90EF9008950F938E
:1025E0001F93CF93DF93CDB7DEB72A970FB6F8943A
:1025F000DEBF0FBECDBF80E390E3A0E3B0E08D83EC
:102600009E83AF83B88704E610E01A87098744E009
:10261000BE016B5F7F4FCE01099695DF40E16AE115
:1026200073E1CE0109968FDF40E16AE273E1CE01EA
:10263000099689DF40E16AE073E1CE01099683DF04
:1026400044E062E073E1CE0109967DDF44E06EEF85
:1026500072E1CE01099677DF44E066E073E1CE01D6
:10266000099671DF44E06AEE72E1CE0109966BDFF4
:1026700044E06AE373E1CE01099665DF44E06AEF66
:1026800072E1CE0109965FDF44E066EF72E1CE01B0
:10269000099659DF44E062EF72E1CE01099653DFFB
:1026A00044E06EEE72E1CE0109964DDF4CE06AE443
:1026B00079E0CE01099647DF42E06CEC7AE0CE018A
:1026C000099641DF41E064EB79E0CE0109963BDFFA
:1026D00042E065EB79E0CE01099635DF42E067EB39
:1026E00079E0CE0109962FDF42E069EB79E0CE0177
:1026F000099629DF4CE061EC79E0CE01099623DFF1
:1027000044E062ED79E0CE0109961DDF41E064EA24
:102710007AE0CE01099617DF48E069E779E0CE015B
:10272000099611DF42E06AE874E1CE0109960BDFF9
:1027300042E068E874E1CE01099605DF42E066E810
:1027400074E1CE010996FFDE42E064E874E1CE0157
:102750000996F9DE42E062E874E1CE010996F3DE03
:1027600042E060E874E1CE010996EDDE44E069E6FE
:1027700072E0CE010996E7DE44E065E672E0CE0144
:102780000996E1DE44E061E672E0CE010996DBDE07
:1027900086E590E3A7E3B0E089839A83AB83BC83AB
:1027A0001A87098744E0BE016F5F7F4FCE0109960B
:1027B000CADEE2EEF1E08491882341F09091C000FE
:1027C00095FFFCCF8093C6003196F5CFE2EDF1E0A6
:1027D0008491882341F09091C00095FFFCCF8093B5
:1027E000C6003196F5CF8091C00085FFFCCF8AE00E
:1027F0008093C6002A960FB6F894DEBF0FBECDBFF9
:10280000DF91CF911F910F910895AF92BF92CF9218
:10281000DF92EF92FF920F931F93CF93DF93CDB789
:10282000DEB7E0970FB6F894DEBF0FBECDBF80E1F4
:10283000E9E9F2E0DE01919601900D928A95E1F7C7
:1028400080E1E9EAF2E0DE01519601900D928A956D
:10285000E1F780E1E9EBF2E0DE01119601900D92E3
:102860008A95E1F76E0181E2C80ED11C8AE1E82E5B
:1028700083E1F82E8E010F5E1F4F6AE273E1AE0115
:102880004F5F5F4F9AE0A92E93E1B92E20E030E030
:10289000F60181919191A191B1916F01F70181931D
:1028A0009193A193B1937F01F80181919191A191AD
:1028B000B1918F01FB0181939193A193B193BF01DA
:1028C000FA0181919191A191B191AF01F5018193AB
:1028D0009193A193B1935F012F5F3F4F2430310556
:1028E000B9F60E94896C80E090E0A8E4B4E480939B
:1028F000021390930313A0930413B093051380E085
:1029000090E8ABE3B5E48093FE129093FF12A0939E
:102910000013B09301131092061310920713109234
:1029200008131092091380E29EE4A0E0B0E08093C7
:102930003A1390933B13A0933C13B0933D1380E064
:1029400090E0A0EAB1E48093EA129093EB12A09396
:10295000EC12B093ED1280E090E0A0E2B1E480933D
:10296000FA129093FB12A093FC12B093FD1280E038
:1029700090E0A0E0B1E48093F6129093F712A09358
:10298000F812B093F9128DEC9CECACECBEE38093A2
:10299000F2129093F312A093F412B093F51280E028
:1029A00090E0A0EAB0E48093EE129093EF12A0932F
:1029B000F012B093F1121092520910925309109232
:1029C00054091092550910924E0910924F09109215
:1029D00050091092510910924A0910924B09109215
:1029E0004C0910924D098EE590E09093CD0A8093AA
:1029F000CC0A8CE699E00E94382288EC90E0909313
:102A00008B1480938A148CE390E0909389148093C4
:102A100088148EE790E0909387148093861420EFBB
:102A200030E030938514209384142AE530E030930D
:102A300083142093821490938114809380148AE9E4
:102A400099E9A1EBB1E48093690290936A02A093A3
:102A50006B02B0936C0261E77DE38AE89FE30E941A
:102A6000EA7F609365027093660280936702909399
:102A7000680260E070E084EE92E40E94F67F60936A
:102A800061027093620280936302909364020E94D9
:102A9000E07680E090E0A0E8BFE380935D02909351
:102AA0005E02A0935F02B093600299DDE2EEF1E076
:102AB0008491882341F09091C00095FFFCCF8093D2
:102AC000C6003196F5CFE6E9F1E08491882341F024
:102AD0009091C00095FFFCCF8093C6003196F5CF52
:102AE0008091C00085FFFCCF8AE08093C600E0960D
:102AF0000FB6F894DEBF0FBECDBFDF91CF911F910F
:102B00000F91FF90EF90DF90CF90BF90AF9008951E
:102B1000CF93DF93CDB7DEB72A970FB6F894DEBF19
:102B20000FBECDBF84E690E09A87898786E590E363
:102B3000A7E3B0E089839A83AB83BC8344E0BE0102
:102B40006B5F7F4FCE01099624DD43E050E0BE016C
:102B50006B5F7F4FCE0101960E9439D4892B09F01B
:102B6000E0C040E16AE173E1CE01099612DD40E187
:102B70006AE273E1CE0109960CDD40E16AE073E19F
:102B8000CE01099606DD0E94896C44E062E073E1A3
:102B9000CE010996FEDC44E06EEF72E1CE010996AB
:102BA000F8DC44E066E073E1CE010996F2DC44E033
:102BB0006AEE72E1CE010996ECDC44E06AE373E16F
:102BC000CE010996E6DC44E06AEF72E1CE01099697
:102BD000E0DC44E066EF72E1CE010996DADC44E025
:102BE00062EF72E1CE010996D4DC44E06EEE72E150
:102BF000CE010996CEDC4CE06AE479E0CE0109967C
:102C0000C8DC42E06CEC7AE0CE010996C2DC41E01F
:102C100064EB79E0CE010996BCDC42E065EB79E03B
:102C2000CE010996B6DC42E067EB79E0CE01099669
:102C3000B0DC42E069EB79E0CE010996AADC4CE019
:102C400061EC79E0CE010996A4DC44E062ED79E024
:102C5000CE0109969EDC41E064EA7AE0CE01099655
:102C600098DC48E069E779E0CE01099692DC42E021
:102C70006AE874E1CE0109968CDC42E068E874E110
:102C8000CE01099686DC42E066E874E1CE01099641
:102C900080DC42E064E874E1CE0109967ADC42E02F
:102CA00062E874E1CE01099674DC42E060E874E108
:102CB000CE0109966EDC44E069E672E0CE01099629
:102CC00068DC44E065E672E0CE01099662DC44E02F
:102CD00061E672E0CE0109965CDC0E94E076E2EEED
:102CE000F1E08491882341F09091C00095FFFCCFE2
:102CF0008093C6003196F5CFE8EBF1E0849188230C
:102D000041F09091C00095FFFCCF8093C6003196B2
:102D1000F5CF8091C00085FFFCCF8AE08093C6008C
:102D200001C073DD2A960FB6F894DEBF0FBECDBF8B
:102D3000DF91CF9108951F920F920FB60F92112439
:102D40000BB60F922F933F934F935F936F938F9395
:102D50009F93EF93FF936091C6002091630630919B
:102D60006406C90101968F779927409165065091B5
:102D700066068417950741F0F901ED51FA4F60831B
:102D80009093640680936306FF91EF919F918F91DA
:102D90006F915F914F913F912F910F900BBE0F90CC
:102DA0000FBE0F901F9018959A01AB01211581EE6F
:102DB00038074105510549F182E08093C00060E089
:102DC00079E08DE390E00E94C7D02150310941099C
:102DD0005109CA01B90122E030E040E050E00E9410
:102DE000C7D03093C5002093C4008091C10080619A
:102DF0008093C1008091C10088608093C100809160
:102E0000C10080688093C10008951092C00020E145
:102E100030E0E7CF20916506309166068091630629
:102E2000909164068217930771F0F901ED51FA4F02
:102E300080812F5F3F4F2F77332730936606209393
:102E4000650690E008958FEF9FEF089580916506E5
:102E500090916606909364068093630608954F925E
:102E60005F926F927F928F929F92AF92BF92CF921A
:102E7000DF92EF92FF920F931F93CF93DF93CDB723
:102E8000DEB7A0970FB6F894DEBF0FBECDBF5C01D2
:102E90004115510561057105E9F420E030E040E39A
:102EA00050E060E070E0A0960FB6F894DEBF0FBE71
:102EB000CDBFDF91CF911F910F91FF90EF90DF90E9
:102EC000CF90BF90AF909F908F907F906F905F90CA
:102ED0004F905BC08E010F5F1F4FC12CD12C76012C
:102EE0004801422E512C612C712C8FEFC81AD80A40
:102EF000E80AF80ACB01BA01A30192010E94A5D009
:102F0000CA01F80161938F01A901BC014115510566
:102F10006105710551F7F1E0CF1AD108E108F10818
:102F2000F401EC0DFD1D80818A3010F440E301C0F6
:102F300047E3480F552747FD5095652F752F20E033
:102F400030E0C50122D081E0C81AD108E108F108BB
:102F5000EFEFCE16DE06EE06FE0611F7A0960FB6D0
:102F6000F894DEBF0FBECDBFDF91CF911F910F91BF
:102F7000FF90EF90DF90CF90BF90AF909F908F9099
:102F80007F906F905F904F9008952115310539F42F
:102F90008091C00085FFFCCF4093C60008952A3081
:102FA000310509F41CC05BCFCF93DF93EC0120E027
:102FB00030E04DE050E060E070E0E7DF20E030E03E
:102FC0004AE050E060E070E0CE01DF91CF91DDCFCC
:102FD0009A01AB01662757FD6095762FD6CFCF9229
:102FE000DF92EF92FF92CF93DF93EC016A017B01B6
:102FF00077FF0FC020E030E04DE250E060E070E08D
:10300000C4DFF094E094D094C094C11CD11CE11CA6
:10301000F11C2AE0B701A601CE01DF91CF91FF900C
:10302000EF90DF90CF901BCF2115310539F48091BF
:10303000C00085FFFCCF4093C600089510CF9A01D1
:10304000462F50E060E070E0EFCFCF93DF93EC01CC
:103050009A01AB0160E070E0E7DFCE01DF91CF9134
:10306000A3CF8F929F92AF92BF92CF92DF92EF92B7
:10307000FF921F93CF93DF93EC016A017B01122F24
:1030800020E030E0A901C701B6010E94D4CC87FF3F
:103090000CC020E030E04DE250E060E070E0CE0196
:1030A00074DFF7FAF094F7F8F094B12C60E070E078
:1030B00080E09FE3B11641F020E030E040E251E4CF
:1030C0000E94DBCCB394F6CF9B01AC01C701B601E3
:1030D0000E94FBCB6B017C010E9448CD4B015C013F
:1030E0000E9474CD9B01AC01C701B6010E94FACBCE
:1030F0006B017C012AE0B501A401CE01B0DE1123F1
:1031000061F0ECEBF4E08191882339F09091C000FC
:1031100095FFFCCF8093C600F6CF112319F120E074
:1031200030E040E251E4C701B6010E94A9CF6B0133
:103130007C010E9443CD4B01AA2497FCA094BA2C99
:10314000B501A401CE014BDFC501B4010E9476CDCB
:103150009B01AC01C701B6010E94FACB6B017C0157
:103160001150DBCFDF91CF911F91FF90EF90DF9057
:10317000CF90BF90AF909F908F90089572CF7F9225
:103180008F929F92AF92BF92CF92DF92EF92FF9277
:103190000F931F93CF93DF93EC01FC01EE0FFF1F02
:1031A000EE0FFF1FEA5AF64F10821182128213822D
:1031B00022E639E04EE559E06AE579E086E599E0F6
:1031C0000E94BE6BCE018A56994F5C01FC0174903F
:1031D0004E01880C991C880C991C8401095F164FBC
:1031E000F401EE5CF64F20E030E040EC5FE36081FC
:1031F0007181828193810E94A9CF6B017C01672D2F
:10320000772767FD7095872F972F0E9476CD9B01BA
:10321000AC01C701B6010E94A9CFF8016083718398
:1032200082839383F401E15DFD4F6081718182812E
:10323000938160930A0270930B0280930C02909327
:103240000D0220E030E040E752E40E94DBCC29E1AF
:10325000C22E29E0D22E7B018C0123E139E04FE020
:1032600059E06BE079E087E099E00E94F3610E9409
:10327000A374F401EA5AF64F10821182128213826B
:1032800022E639E04EE559E06AE579E086E599E025
:103290000E94BE6BC4018756994F4C01FC01C5903A
:1032A000D590E590F490F50164918E01000F111F07
:1032B000000F111F095F164FF7FAF094F7F8F0941A
:1032C000772767FD7095872F972F0E9476CD9B01FA
:1032D000AC01C701B6010E94A9CFF80160837183D8
:1032E0008283938320E030E040E752E460910A0259
:1032F00070910B0280910C0290910D020E94DBCC28
:1033000049E1C42E49E0D42E7B018C0123E139E050
:103310004FE059E06BE079E087E099E00E94F361CB
:103320000E94A374F4016591759185919491F501C2
:1033300094905E01AA0CBB1CAA0CBB1C8501095F02
:10334000164F9B01AC010E94FBCB6B017C01692DE8
:10335000772767FD7095872F972F0E9476CD9B0169
:10336000AC01C701B6010E94A9CFF8016083718347
:1033700082839383F501E15DFD4F20E030E040E87A
:103380005EE360817181828193810E94A9CF609305
:103390000A0270930B0280930C0290930D0220E0BE
:1033A00030E040E752E40E94DBCCE9E1CE2EE9E0D8
:1033B000DE2E7B018C0123E139E04FE059E06BE028
:1033C00079E087E099E00E94F3610E94A374F5011F
:1033D000E65BF64FC080D180E280F380F501EB55CB
:1033E000F94F6591759185919491CC0FDD1FCC0FAC
:1033F000DD1F8E01025C164FA70196010E94FBCBD8
:10340000F80160837183828393838E01015E1D4F77
:10341000FE01E65EF64FA70196016081718182810F
:1034200093810E94FBCBF801608371838283938335
:10343000FE01EA5AF64F1082118212821382C95F8E
:10344000D64F188219821A821B8222E639E04EE595
:1034500059E06AE579E086E599E00E94BE6B10923A
:103460000A0210920B0210920C0210920D02DF91D0
:10347000CF911F910F91FF90EF90DF90CF90BF9071
:10348000AF909F908F907F900C946C6DFC01249175
:10349000222341F03091C00035FFFCCF2093C600BD
:1034A0000196F4CF22E030E082EE95E067CECF9334
:1034B000DF931F921F92CDB7DEB780914015909198
:1034C00041159E012F5F3F4F009719F42654354157
:1034D00002C0281B390B3A83298389819A810F9076
:1034E0000F90DF91CF91089520915C0730915D0797
:1034F000243031050CF06AC040915E0750915F079F
:1035000060E6649F9001659F300D1124BC01C901E4
:103510008A59984F0E9432D4E1EBF6E084918823D7
:1035200041F09091C00095FFFCCF8093C60031968A
:10353000F5CFEBE8F6E08491882341F09091C0004C
:1035400095FFFCCF8093C6003196F5CF80915E0742
:1035500090915F0720E6289FF001299FF00D11242C
:10356000EA59F84F8191882339F09091C00095FF76
:10357000FCCF8093C600F6CFE9E8F6E0849188237B
:1035800041F09091C00095FFFCCF8093C60031962A
:10359000F5CF8091C00085FFFCCF8AE08093C60004
:1035A00080915E0790915F07019664E070E00E9451
:1035B00092D090935F0780935E0780915C07909113
:1035C0005D07019690935D0780935C0708952091B5
:1035D0005C0730915D07243031050CF06AC04091E2
:1035E0005E0750915F0760E6649F9001659F300D14
:1035F0001124BC01C9018A59984F0E94B5D3E1EB4F
:10360000F6E08491882341F09091C00095FFFCCFB3
:103610008093C6003196F5CFEEE7F6E084918823DB
:1036200041F09091C00095FFFCCF8093C600319689
:10363000F5CF80915E0790915F0720E6289FF0010B
:10364000299FF00D1124EA59F84F8191882339F010
:103650009091C00095FFFCCF8093C600F6CFECE7B9
:10366000F6E08491882341F09091C00095FFFCCF53
:103670008093C6003196F5CF8091C00085FFFCCFC6
:103680008AE08093C60080915E0790915F07019663
:1036900064E070E00E9492D090935F0780935E0791
:1036A00080915C0790915D07019690935D078093F0
:1036B0005C07089560E080E40E94A4C79FB7F89477
:1036C000E8E0F1E08081846080839FBF0895269ABE
:1036D0002E980895809156079091570760E070E00A
:1036E00001960C940CD180915607909157074AE0AF
:1036F00050E060E070E001960C9474D2682F772758
:1037000067FD7095209160073091610740E6429F08
:10371000C001439F900D11248A59984F0E941ED4D6
:10372000909357078093560721E0892B09F420E0F6
:10373000822F08950E94C4C5609352077093530767
:103740008093540790935507E0916007F0916107CB
:10375000EE59F84F8081811114C0E0E1F2E08491CC
:10376000882341F09091C00095FFFCCF8093C60064
:103770003196F5CF8091C00085FFFCCF8AE0809321
:10378000C600089582EE95E061DBE3E1F2E084910A
:10379000882341F09091C00095FFFCCF8093C60034
:1037A0003196F5CF4091EB085091EC086091ED080F
:1037B0007091EE084F5F5F4F6F4F7F4F2AE030E010
:1037C00082EE95E0E2DB8091C00085FFFCCF8AE0CD
:1037D0008093C600AFCF7F928F929F92AF92BF929D
:1037E000CF92DF92EF92FF920F931F93CF93DF93CD
:1037F0009CE3C92E94E0D92EC6E5D9E007E019E094
:1038000028E6E22E29E0F22E712CF60181916F015B
:1038100075DF882359F18091A40A882309F459C0DF
:10382000F1E07F1256C08091C60A9091C70A0197B5
:1038300009F44FC04FDF4B015C012091AE0A30917B
:10384000AF0A4091B00A5091B10A6091A60A7091F6
:10385000A70A8091A80A9091A90A0E94FACB9B011D
:10386000AC01C501B4010E94FACB34C088819981B2
:10387000AA81BB81F80180839183A283B38373946F
:1038800024960C5F1F4FFFEFEF1AFF0A84E07812B7
:10389000BCCF86E433DF882309F43DC01BDF6B0116
:1038A0007C016093F7087093F8088093F90890936F
:1038B000FA0820E030E0A9010E94D7CE18165CF586
:1038C000C0920A02D0920B02E0920C02F0920D021A
:1038D00022C000DF4B015C01F7018081811103C030
:1038E0006091E60801C061E070E080E090E00E9435
:1038F00076CD288139814A815B810E94A9CF9B01C5
:10390000AC01C501B4010E94FBCBF8016083718357
:1039100082839383B4CFDF91CF911F910F91FF905A
:10392000EF90DF90CF90BF90AF909F908F907F905F
:10393000089551DF89E4E2DE882351F0CBDE609305
:10394000FB087093FC088093FD089093FE0808C064
:103950001092FB081092FC081092FD081092FE08CD
:103960008AE4CCDE882351F0B5DE6093FF087093C3
:103970000009809301099093020908951092FF08AD
:103980001092000910920109109202090895CF9235
:10399000DF92EF92FF92CF93DF93EC01C0903E094C
:1039A000D0903F09E0904009F0904109A7019601AD
:1039B000688179818A819B810E94D4CC87FF04C071
:1039C000C882D982EA82FB82C0904209D090430922
:1039D000E0904409F0904509A70196016C817D8132
:1039E0008E819F810E94D4CC87FF04C0CC82DD826F
:1039F000EE82FF82C0904609D0904709E0904809C6
:103A0000F0904909A7019601688579858A859B858B
:103A10000E94D4CC87FF04C0C886D986EA86FB867C
:103A2000C0901F02D0902002E0902102F09022026C
:103A3000A7019601688179818A819B810E94D7CEF6
:103A4000181624F4C882D982EA82FB82C09023022D
:103A5000D0902402E0902502F0902602A701960162
:103A60006C817D818E819F810E94D7CE181624F4AF
:103A7000CC82DD82EE82FF82C0902702D0902802A5
:103A8000E0902902F0902A02A701960168857985C5
:103A90008A859B850E94D7CE181624F4C886D986BD
:103AA000EA86FB86DF91CF91FF90EF90DF90CF9079
:103AB0000895CF92DF92EF92FF920F931F9387E0CA
:103AC00099E065DF0E94C4C5609352077093530765
:103AD0008093540790935507209107093091080966
:103AE0004091090950910A0960915609709157094E
:103AF00080915809909159090E94D4CC811179C0C4
:103B000020910B0930910C0940910D0950910E093B
:103B100060915A0970915B0980915C0990915D09EF
:103B20000E94D4CC811165C020E030E040E752E42F
:103B300060910A0270910B0280910C0290910D022B
:103B40000E94DBCC39E1C32E39E0D32E7B018C01FE
:103B500023E139E04FE059E06BE079E087E099E05C
:103B60000E94F3618091070990910809A0910909C9
:103B7000B0910A098093560990935709A093580968
:103B8000B093590980910B0990910C09A0910D09EE
:103B9000B0910E0980935A0990935B09A0935C0938
:103BA000B0935D0980910F0990911009A0911109BE
:103BB000B091120980935E0990935F09A093600908
:103BC000B09361098091130990911409A09115098E
:103BD000B09116098093620990936309A0936409D8
:103BE000B09365091F910F91FF90EF90DF90CF90F8
:103BF000089560912D0270912E02882777FD80959F
:103C0000982F0E9476CD20910A0230910B024091AC
:103C10000C0250910D020E94A9CF20E030E040E755
:103C200052E40E94DBCC20E030E048EC52E488CF44
:103C3000AF92BF92CF92DF92EF92FF920F931F93BA
:103C4000CF93DF93D82F2091FF0830910009409146
:103C50000109509102096091FB087091FC08809164
:103C6000FD089091FE080E94E4CEC62F172F082F62
:103C7000F92E60912D0270912E02882777FD809594
:103C8000982F0E9476CD20910A0230910B0240912C
:103C90000C0250910D020E94A9CF20E030E040E7D5
:103CA00052E40E94DBCC20E030E048EC52E40E9479
:103CB000DBCC209119092F93DF93FF920F931F9371
:103CC000CF935B016C0142E0E42E01E020E04BEF7A
:103CD00058E067E079E086E599E00E94C459809158
:103CE000070990910809A0910909B0910A098093E8
:103CF000560990935709A0935809B0935909809198
:103D00000B0990910C09A0910D09B0910E098093B7
:103D10005A0990935B09A0935C09B0935D09809167
:103D20000F0990911009A0911109B0911209809387
:103D30005E0990935F09A0936009B0936109809137
:103D4000130990911409A0911509B0911609809357
:103D5000620990936309A0936409B09365090E9476
:103D6000C4C5609352077093530780935407909390
:103D700055070F900F900F900F900F900F90DF91BD
:103D8000CF911F910F91FF90EF90DF90CF90BF9058
:103D9000AF900895F8940E94FB795F9A8A9A9FB732
:103DA000F894809108018160809308019FBF129A66
:103DB000479A60E08CE00E94A4C7E7EBF6E08491AC
:103DC000882341F09091C00095FFFCCF8093C600FE
:103DD0003196F5CFE1EFF1E08491882341F09091A5
:103DE000C00095FFFCCF8093C6003196F5CF80913F
:103DF000C00085FFFCCF8AE08093C60088EE91E08A
:103E00000E946993FFCFCF92DF92EF92FF920F93C0
:103E10001F930E94C4C500914E0710914F07209137
:103E2000500730915107C0905207D0905307E0904F
:103E30005407F09055076C197D098E099F090617E4
:103E400017072807390728F4012B022B032B09F049
:103E5000A1DF8091060290910702A0910802B09123
:103E60000902892B8A2B8B2BC9F180916C09873031
:103E7000D1F40E94C4C500915207109153072091BC
:103E8000540730915507601B710B820B930B653CF7
:103E900079408105910510F19091E40D8091E30D39
:103EA00098131CC027C00E94C4C5009152071091EE
:103EB00053072091540730915507601B710B820BFB
:103EC000930B009106021091070220910802309195
:103ED0000902061717072807390780F080910601A5
:103EE00082FFB6CF1F910F91FF90EF90DF90CF90A0
:103EF0000C94D66181E080934507F0CF9091E40D5A
:103F00008091E30D9813EACF5F9A8A9A9FB7F8944D
:103F1000809108018160809308019FBF129A479A9F
:103F200010926D0910926E0910926F09109270092B
:103F3000109271091092720910927309109274090B
:103F400010927509109276091092770910927809EB
:103F5000C5CFCF93DF93EC01809119098093680658
:103F600084E5CCDB811102C080E063C0B3DB0E943A
:103F700048CD609368066230B8F3E1EBF6E08491D7
:103F8000882341F09091C00095FFFCCF8093C6003C
:103F90003196F5CFC936D10599F034F4C836D1053C
:103FA000C9F5EEE0F3E015C0CD36D10531F0CA3DDC
:103FB000D10581F5E9ECF2E02AC0E0EEF2E01DC0A7
:103FC000E7EFF2E010C09091C00095FFFCCF809326
:103FD000C60081918111F7CF1DC09091C00095FF5F
:103FE000FCCF8093C60081918111F7CF13C09091CF
:103FF000C00095FFFCCF8093C60081918111F7CF5F
:1040000009C09091C00095FFFCCF8093C6008191BC
:104010008111F7CF40E050E06091680682EE95E0B4
:104020000ED88091C00085FFFCCF8AE08093C60047
:1040300081E0DF91CF9108958F929F92AF92BF92CE
:10404000CF92DF92EF92FF92CF93DF93EC01FC01CE
:10405000E75BFF4F60817181882777FD8095982FFE
:104060000E9476CD4B015C0160931F027093200289
:104070008093210290932202FE01E55BFF4F608155
:104080007181882777FD8095982F0E9476CD6B01EE
:104090007C01609323027093240280932502909305
:1040A0002602C35BDF4F68817981882777FD809581
:1040B000982F0E9476CD60932702709328028093F8
:1040C000290290932A028092320990923309A09299
:1040D0003409B0923509C0923609D0923709E0927E
:1040E0003809F092390960933A0970933B0980933B
:1040F0003C0990933D0910922609109227091092CD
:1041000028091092290910922A0910922B0910925D
:104110002C0910922D0910922E0910922F0910923D
:1041200030091092310980921A0990921B09A092CD
:104130001C09B0921D09C0921E09D0921F09E0927D
:104140002009F0922109609322097093230980933A
:10415000240990932509DF91CF91FF90EF90DF9094
:10416000CF90BF90AF909F908F900895CF93DF93A3
:10417000FC01EC01C05CDF4F8881DF01AC5BBF4F0D
:104180008E3009F41C9280818C30E1F48091CE0A4B
:104190009091CF0A843F21E0920709F42C98813D49
:1041A000974020F01092CF0A1092CE0A8091CE0A4A
:1041B0009091CF0A009709F42C9A01969093CF0A18
:1041C0008093CE0A80818D7F813039F488818E3052
:1041D00021F48091CB0A81112C988C91882349F18C
:1041E00090818EEF890F823038F52CB122952170A5
:1041F00030910301DF01AF5BBF4F8C918370EB5BAC
:10420000FF4F813039F0833081F4211105C030FD3A
:1042100003C00BC0222349F08081816080839230EB
:1042200059F4DF91CF910C945893808180788083EA
:1042300003C0EB5BFF4F1082DF91CF9108950E9486
:10424000C4C56093520770935307809354079093AB
:1042500055070895CF92DF92EF92FF92CF93DF93AD
:10426000EC011F8A188E198E1A8E1B8E1C8E1D8EC5
:104270001E8EC12CD12C58E4E52E52E4F52ECF8EA3
:10428000D8A2E9A2FAA2CBA2DCA2EDA2FEA2FC0176
:10429000E75BFF4F6081718162537109882777FD69
:1042A0008095982F0E9476CD6FA378A789A79AA7AB
:1042B000CBA6DCA6EDA6FEA66FA778AB89AB9AAB22
:1042C000FE01E55BFF4F60817181625371098827B0
:1042D00077FD8095982F0E9476CD6BAB7CAB8DAB34
:1042E0009EABCFAAD8AEE9AEFAAE6BAF7CAF8DAFC6
:1042F0009EAFDF91CF91FF90EF90DF90CF90089528
:104300004F925F926F927F928F929F92AF92BF92E5
:10431000CF92DF92EF92FF920F931F93CF93DF9391
:104320001F92CDB7DEB74C015B0169017A01AA0C7F
:10433000BB1CAA0CBB1C8C010A0D1B1DF801EB5AFF
:10434000FF4F408051806280738020E030E0A901FF
:10435000C301B2010E94D4CC20E030E0A901811158
:104360000CC0C701B6010E94D4CC81110CC0F80169
:10437000118212821382148249C0C701B6010E94C1
:10438000D4CC882341F0F501EA5AF64FC082D1829D
:10439000E282F38207C0F501EA5AF64F4082518269
:1043A00062827382F501E15DFD4F608171818281DE
:1043B0009381198220E030E040EF52E40E94DBCC90
:1043C0009E012F5F3F4F69017B018C0122E639E09E
:1043D0004EE559E06AE579E086E599E00E94F361EF
:1043E0000E94A3748A0C9B1C95012A5A364FF9012E
:1043F00080819181A281B381F40181839283A3831F
:10440000B483F90110821182128213820F90DF911E
:10441000CF911F910F91FF90EF90DF90CF90BF90C1
:10442000AF909F908F907F906F905F904F90089586
:10443000662329F0FC0111861286138614861092D9
:104440005609109257091092580910925909109262
:104450005A0910925B0910925C0910925D09109242
:104460005E0910925F091092600910926109089527
:10447000FC01EC5BFF4F1082349621E020837E9696
:104480004CE251E060E070E04083518362837383CB
:10449000EE52FF4F1082409113025091140260912E
:1044A000150270911602FC01458756876787708B4D
:1044B00040911B0250911C0260911D0270911E02DE
:1044C000418B528B638B748B08954F925F926F92E6
:1044D0007F92AF92BF92CF92DF92EF92FF920F93B3
:1044E0001F93CF93DF935C016A017B01280139019F
:1044F000EC01C659DF4F401751076207730709F4F3
:1045000075C0CB01BA01601B710B820B930B25E0C8
:1045100030E040E050E00E94A5D0C414D504E60489
:10452000F70490F5F501EB59FF4F80818823D1F016
:1045300088819981AA81BB818C159D05AE05BF0537
:1045400020F4C882D982EA82FB8288819981AA817B
:10455000BB81820F931FA41FB51F88839983AA83F1
:10456000BB8304C0C882D982EA82FB828881998198
:10457000AA81BB81481659066A067B06D8F548828F
:1045800059826A827B8236C04C145D046E047F04BB
:1045900068F5F501EB59FF4F808181111AC08881C0
:1045A0009981AA81BB8184159505A605B70520F4DC
:1045B000488259826A827B8288819981AA81BB81E3
:1045C000820F931FA41FB51F88839983AA83BB837F
:1045D00004C0488259826A827B8288819981AA813B
:1045E000BB81C816D906EA06FB0620F4C882D98228
:1045F000EA82FB82DF91CF911F910F91FF90EF90A4
:10460000DF90CF90BF90AF907F906F905F904F9072
:104610000895FC01E958FF4F1082339710823397B9
:104620001082319611821082EA59FF4F1082E056B3
:10463000F10910820895FC01DC01AC5BBF4F1C92B4
:10464000108211961C9217AE15978DE08C931696DA
:104650001C9214971C92159621E02C9311962C9382
:10466000119680E991E011969C938E931296119683
:104670009C938E93129684EF91E011969C938E9367
:104680001C971C9252968FEF9FEF11969C938E93DE
:10469000AB51BF4F2C931182128213821482A35EFE
:1046A000B1091D921D921D921C92139715821682BC
:1046B0001782108614961D921D921D921C921397BC
:1046C000118612861386148614961D921D921D92D1
:1046D0001C9213975A971C929B961C92A553BF4FFE
:1046E0001C92CF0196CF0E945A1B0E94671B40E983
:1046F00050ED63E070E082EE95E00E94D416E6E7AC
:10470000F6E08491882341F09091C00095FFFCCFA2
:104710008093C6003196F5CF8091C00085FFFCCF15
:104720008AE08093C60084B780FF14C0EEE6F6E00E
:104730009491992341F02091C00025FFFCCF9093E4
:10474000C6003196F5CF9091C00095FFFCCF9AE05E
:104750009093C60081FF14C0EEE5F6E09491992392
:1047600041F02091C00025FFFCCF9093C600319608
:10477000F5CF9091C00095FFFCCF9AE09093C600D2
:1047800082FF14C0EDE4F6E09491992341F020916A
:10479000C00025FFFCCF9093C6003196F5CF9091D5
:1047A000C00095FFFCCF9AE09093C60083FF14C031
:1047B000EDE3F6E09491992341F02091C00025FFAC
:1047C000FCCF9093C6003196F5CF9091C00095FF35
:1047D000FCCF9AE09093C60085FF14C0EDE2F6E0AE
:1047E0008491882341F09091C00095FFFCCF809385
:1047F000C6003196F5CF8091C00085FFFCCF8AE0DE
:104800008093C60014BEE9E2F6E08491882341F06B
:104810009091C00095FFFCCF8093C6003196F5CFF4
:104820008091C00085FFFCCF8AE08093C600E9E15B
:10483000F6E08491882341F09091C00095FFFCCF71
:104840008093C6003196F5CFE4E0F6E084918823AA
:1048500041F09091C00095FFFCCF8093C600319647
:10486000F5CFE8EFF5E08491882341F09091C00006
:1048700095FFFCCF8093C6003196F5CFE1EFF5E0D0
:104880008491882341F09091C00095FFFCCF8093E4
:10489000C6003196F5CF8091C00085FFFCCF8AE03D
:1048A0008093C600E6EEF5E08491882341F0909174
:1048B000C00095FFFCCF8093C6003196F5CFEAED9E
:1048C000F5E08491882341F09091C00095FFFCCFE2
:1048D0008093C6003196F5CF8091C00085FFFCCF54
:1048E0008AE08093C600EBECF5E08491882341F0E8
:1048F0009091C00095FFFCCF8093C6003196F5CF14
:104900000E94571A4AE050E0BC0182EE95E00E94F6
:10491000E817E4EBF5E08491882341F09091C00022
:1049200095FFFCCF8093C6003196F5CF4AE050E06A
:1049300060ED74E082EE95E00E94E8178091C0007F
:1049400085FFFCCF8AE08093C60010926207109228
:10495000630710926407109265078CE699E06BDE9E
:104960000E9488158CE699E067DB0E9414790E940A
:104970008D600E9416740E94CB9360ED77E080E01A
:1049800090E00E94F3C51092CA0A1092C90A0895D5
:10499000CF93DF93EC01C858DF4F65E273E0CE019F
:1049A0000E9456D4892B19F082E090E036C067E36C
:1049B00073E0CE010E9456D4892B69F569E473E057
:1049C000CE010E9456D4892B79F767E573E0CE01BA
:1049D0000E9456D4892BF9F460E673E0CE010E9460
:1049E00056D4892B09F761E773E0CE010E9456D4B3
:1049F000892B89F462E873E0CE010E9456D4892B9A
:104A000051F46DE873E0CE010E9456D4892B61F613
:104A100080E090E002C083E090E0DF91CF910895C4
:104A2000AF92BF92CF92DF92EF92FF920F931F93BC
:104A3000CF93DF931F92CDB7DEB75C01DC01AC589A
:104A4000BF4F8C918111A7C0662309F4A4C06501F2
:104A500087E7C80ED11CF601808185010E581F4FD3
:104A6000811138C0F8011182108233976B3331F411
:104A700081E013978C93118210826BC06A3009F029
:104A800068C0808191818A0D9B1DDC01A858BF4FB1
:104A90001C92118210827501F1E7EF0EF11CF701F3
:104AA00080818823A1F0C501698372DFF501EB588D
:104AB000FF4F9183808369811816190634F481E0D1
:104AC000F6018083F701108266C0F6011082F701BB
:104AD00010823FC081E090E0F80191838083A501BE
:104AE0004F585F4F6B33C1F471E0FA017083950149
:104AF00021593F4FF90180819181009731F1AC013B
:104B00004F5F5F4F518340838A0D9B1D88529F4F9B
:104B1000FC0110827C933FC06A30B9F4C501815911
:104B20009F4FFC01208131812115310541F02A0D73
:104B30003B1D28523F4FF901108221E02C93FA01CE
:104B40001082FC011182108226C0FA01808181113D
:104B500022C0F801A081B181F501E159FF4F4081E8
:104B600051819A012F5F3F4F3183208370E67A9FF6
:104B7000C0017B9F900D11248A0D9B1D840F951FF2
:104B8000DC01A858BF4F6C932E35310524F08EE51B
:104B900090E0918380830F90DF91CF911F910F91CF
:104BA000FF90EF90DF90CF90BF90AF900895CF939C
:104BB000DF93EC01FC01EC58FF4F8081882351F119
:104BC000209160073091610740E6429FC001439FFA
:104BD000900D1124BE0168527F4F8A59984F0E9450
:104BE00029D418161906B4F4FE01EB58FF4F808142
:104BF00091818230910519F47097108207C0039754
:104C000029F481E0FE01EB59FF4F8083CE01DF9153
:104C1000CF91FFCCDF91CF9108958091A40A882392
:104C200059F0FB01EE0FFF1FE55CF84F81E020819A
:104C300031812F3F3F4F09F480E090E00895FC015F
:104C400010820895FC01158686E080A311861286E5
:104C5000138614861582168217821086118212829C
:104C60001382148208953F924F925F926F927F92C7
:104C70008F929F92AF92BF92CF92DF92EF92FF926C
:104C80000F931F93CF93DF93CDB7DEB7A2970FB6E5
:104C9000F894DEBF0FBECDBF8CE699E088DF87E4D5
:104CA0000E947E1B882309F43DC30E946A1B0E9458
:104CB00043CD6C31710509F4C8C09CF462307105B4
:104CC00009F468C024F477FF5BC00C949939633011
:104CD000710509F467C06430710509F46EC00C9465
:104CE00099396C35710509F492C274F46A3571050D
:104CF00009F489C26B35710511F00C94993981E082
:104D00008093E6080C949939613421E0720709F424
:104D1000C9C26234714011F00C9499398091CD0967
:104D20009091CE09A091CF09B091D00980935E09EE
:104D300090935F09A0936009B0936109198220E004
:104D400030E040EA50E4609137027091380280917F
:104D5000390290913A020E94DBCCFE0131966F013C
:104D60007B018C0122E639E04EE559E06AE579E005
:104D700086E599E00E94F3610E94A3740C9499392E
:104D800080916706811106C00E94EB1B0E94591D8D
:104D90000C94873B80916706811104C00E94991C86
:104DA00081E007C080916706811107C00E94991CAD
:104DB00080E00E94181E0C94873B82E494E00E94DD
:104DC000AE9280E50E947E1B882339F00E946A1B08
:104DD0000E9448CD4B015C0103C0812C912C5401F1
:104DE00083E50E947E1B882361F00E946A1B20E0FD
:104DF00030E04AE754E40E94A9CF0E9448CD4B011D
:104E00005C010E94A3740E94C4C56B017C01C80CA4
:104E1000D91CEA1CFB1C0E94C4C560935207709306
:104E2000530780935407909355070E94C4C56C158F
:104E30007D058E059F0510F00C9499390E940A7724
:104E40000E94031F0E94F193F0CF8091A40A88234F
:104E500041F08091C60A9091C70A019711F00C9415
:104E60009C39F09019091092190980910A029091C9
:104E70000B02A0910C02B0910D028093F308909365
:104E8000F408A093F508B093F60880912D02909154
:104E90002E02909367098093660984E690E09093D0
:104EA0002E0280932D020E94C4C560935207709316
:104EB0005307809354079093550711E01093D1093D
:104EC0008CE699E0A6DB81E00E94736D8091560923
:104ED00090915709A0915809B091590980930709F9
:104EE00090930809A0930909B0930A0940915A09BF
:104EF00050915B0960915C0970915D0940930B09C9
:104F000050930C0960930D0970930E0940915E094E
:104F100050915F09609160097091610940930F0998
:104F2000509310096093110970931209409162091E
:104F30005091630960916409709165094093130968
:104F400050931409609315097093160910920A0280
:104F500010920B0210920C0210920D0288E50E9432
:104F60007E1B882311F0E12C0AC089E50E947E1B7C
:104F70008111F9CF8AE50E947E1BE82EE126E0929E
:104F80000E0288E50E947E1B182F89E50E947E1B79
:104F9000082FE11004C0111102C0882311F120E094
:104FA00030E040EC50E460915E0970915F098091BF
:104FB0006009909161090E94D4CC87FF12C020E063
:104FC00030E040EC50E46091750970917609809171
:104FD0007709909178090E94D4CC87FF02C00C9485
:104FE000D33980910E0281110C94EB3989E50E942E
:104FF0007E1B81110C94EB3980910E02811102C04D
:10500000112361F080E090E00E94BF1820E030E0C2
:10501000A90160E070E08CE699E072D98AE50E940F
:105020007E1BE82E80910E02811102C0EE2051F10C
:105030002091C1093091C2094091C3095091C4091E
:1050400060916D0970916E0980916F09909170095E
:105050000E94D4CC87FF0AC08091DA09811106C072
:105060008091AC098E3011F00C94FA3982E090E016
:105070000E94BF1820E030E0A90162E070E08CE6F9
:1050800099E03ED988E50E947E1B8823D1F00E94DA
:10509000731B672B682B692BA1F00E946A1B209160
:1050A0004A0930914B0940914C0950914D090E9499
:1050B000FBCB6093560970935709809358099093DE
:1050C000590989E50E947E1B8823D1F00E94731B39
:1050D000672B682B692BA1F00E946A1B20914E0957
:1050E00030914F0940915009509151090E94FBCBDA
:1050F00060935A0970935B0980935C0990935D09F2
:105100008AE50E947E1B8823D1F00E94731B672BC7
:10511000682B692BA1F00E946A1B209152093091E3
:10512000530940915409509155090E94FBCB60935B
:105130005E0970935F0980936009909361096E2DF9
:105140008CE699E075D922E639E04EE559E06AE54A
:1051500079E086E599E00E94BE6B80E00E94736D65
:105160008091F3089091F408A091F508B091F608A9
:1051700080930A0290930B02A0930C02B0930D024D
:10518000F0921909809166099091670990932E0217
:1051900080932D020E94C4C56093520770935307F9
:1051A00080935407909355070E946C6D1092DA0912
:1051B0008091A40A8823E1F080910E02882319F0DF
:1051C00087E08093B20A112329F08091B20A8160AE
:1051D0008093B20A002329F08091B20A8260809302
:1051E000B20AEE2029F08091B20A84608093B20A5C
:1051F00080916C09853011F00C94993986E0809388
:105200006C090C9499391092E6080C94993985E44C
:105210000E947E1B811102C00E94A374BCE3CB2EAE
:10522000B4E0DB2E1AE4E12E19E0F12E06E519E0D8
:10523000B12CD6018D916D010E947E1B882339F11E
:10524000B3E0BB120CC00E946A1BF801608371833B
:105250008283938382E699E00E94636C18C00E9467
:105260006A1BD7012D913D914D915C910E94FBCB22
:10527000F801608371838283938322E639E04EE5EF
:1052800059E06AE579E086E599E00E94BE6BB39447
:10529000F4E0EF0EF11C0C5F1F4F24E0B212C9CFF7
:1052A0000C94993960915E0970915F098091600951
:1052B000909161096093CD097093CE098093CF09D5
:1052C0009093D00920E030E040E251E40E94FBCB13
:1052D00060935E0970935F09809360099093610900
:1052E000198220E030E040EA50E46091370270918A
:1052F00038028091390290913A020E94DBCCDE01A3
:1053000011966D017B018C0122E639E04EE559E0F2
:105310006AE579E086E599E00E94F3610E94A37452
:105320000C9499398DE40E947E1B882311F40C940F
:1053300017380E946A1B0E9443CD6737710509F434
:10534000BEC10CF0CAC06F31710509F43DC30CF049
:105350005FC06531710509F445C2CCF56530710552
:1053600009F40BC2ACF477FF02C00C949939623097
:1053700071050CF4A7C16330710511F00C949939D3
:105380000E94A3742C9A81E08093CB0A0C949939E3
:105390006231710509F472C66431710509F4F4C112
:1053A0006131710511F00C94993980EF93E00E94FE
:1053B000AE925F988A989FB7F894809108018E7F8B
:1053C000809308019FBF129847980C9499396931CE
:1053D000710509F438C264F46731710509F408C233
:1053E0000CF01EC280ED9AE00E9483530C94993910
:1053F0006B31710509F43BC20CF42BC26C317105A1
:1054000009F43BC26E31710509F46CC20C949939F0
:105410006C35710509F46CC6D4F56135710509F474
:1054200020C67CF46934710511F40C94B3366035F0
:10543000710509F412C66A32710511F00C9499399C
:105440004AC36335710509F414C60CF40EC66435FD
:10545000710509F413C66535710511F00C9499397D
:1054600083E50E947E1B0E946A1B20E030E04AE731
:1054700054E40E94A9CF0E9448CD60934E077093D8
:105480004F0780935007909351070C9499396B36CE
:10549000710509F4DCC564F46936710509F475C356
:1054A0000CF0A5C56836710509F440C30C94993910
:1054B0006237710509F4D0C634F46D36710509F40C
:1054C00053C40C9499396337710509F494C6653750
:1054D000710509F49FC60C9499396039F1E07F0792
:1054E00011F40C948A350CF063C06D3C710511F415
:1054F0000C94EB322CF56E3B710509F4B4C464F4E2
:105500006937710509F48BC70CF485C76C387105D0
:1055100009F42AC30C9499396B3C710511F40C946D
:10552000AF3214F00C94CB32693C710511F00C943D
:1055300099390CE314E02AE0E22E23E1F22EF5C7BC
:105540006D3D710511F40C944134BCF46A3D710554
:1055500011F40C946F336C3D710511F40C943234DA
:105560006E3C710511F00C9499390CE314E08AE457
:10557000E82E89E0F82E0C9460336D3231E0730729
:1055800011F40C947E343CF46C32714011F40C94A0
:1055900050340C9499396E32A1E07A0711F40C94CE
:1055A00044356F32714011F40C9452350C94993992
:1055B0006933E8E07E0711F40C94C2360CF04FC05A
:1055C000603A23E0720709F4CBC1ACF4653F81E097
:1055D000780711F40C948D35663F91E0790711F44A
:1055E0000C949035643F714011F00C9499390E94ED
:1055F000EF120C949939663DB7E07B0711F40C94D7
:105600009335ECF4673E734011F00C949939109285
:1056100067060E946F938091E7089091E808A09137
:10562000E908B091EA088093EB089093EC08A09306
:10563000ED08B093EE080E94C21B0C949939673DA7
:1056400027E0720711F40C94C7356433784011F0E9
:105650000C9499398DE08093AC090C9499396A398E
:1056600088E0780711F40C9411379CF46839A8E0AD
:105670007A0711F40C94DB3614F00C94FC366A3380
:10568000784011F00C94993981E08093D1090C9401
:1056900099396C39F8E07F0711F40C94373714F41A
:1056A0000C941D376D3938E0730711F40C944F37A3
:1056B0006E39784011F40C9497370C949939E7EAD5
:1056C000F3E0B7C686E094E00E94AE9280E50E94C7
:1056D0007E1B882339F00E946A1B0E9448CD6B0113
:1056E0007C0103C0C12CD12C760183E50E947E1B76
:1056F000882361F00E946A1B20E030E04AE754E40E
:105700000E94A9CF0E9448CD6B017C010E94A37426
:105710000E94C4C560935207709353078093540747
:1057200090935507C114D104E104F104A9F00E943B
:10573000C4C54B015C018C0C9D1CAE1CBF1C0E949F
:10574000C4C5681579058A059B0588F40E94F794FD
:1057500081110DC00C94053A0E94F794811107C085
:105760000E940A770E94031F0E94F193F5CF89EFF0
:1057700093E00E94AE920C9499390E94A3742C98E5
:105780001092CB0A0C949939E0EEF3E084918823CF
:1057900041F09091C00095FFFCCF8093C6003196F8
:1057A000F5CF8091C00085FFFCCF8AE08093C600D2
:1057B00080ED9AE00E946952E2EDF3E08491882343
:1057C00041F09091C00095FFFCCF8093C6003196C8
:1057D000F5CF8091C00085FFFCCF8AE08093C600A2
:1057E0000C94993980ED9AE00E94C0520C9499393A
:1057F00000915607109157070C5F1F4F6AE270E047
:10580000C8010E941ED4009719F0FC013197108244
:1058100041E0B80180ED9AE00E9493530C949939CD
:1058200080ED9AE00E9487530E94C4C560934A07A6
:1058300070934B0780934C0790934D0782E08093C1
:105840006C090C94993980ED9AE00E948E530C9467
:1058500099398091D30A882311F40C94993983E5FE
:105860000E947E1B81110C940D3A0C94993980EDA5
:105870009AE00E94C8560C949939809156079091ED
:1058800057076AE270E004960E941ED48C010097CC
:10589000E1F0209160073091610740E6429FC0012E
:1058A000439F900D11246EE470E08A59984F0E9436
:1058B0001ED460E270E00E941ED4019690935707B8
:1058C00080935607F80131971082609156077091C6
:1058D00057076C5F7F4F40E080ED9AE00E94935342
:1058E0000C9499398091D30A882311F40C94993936
:1058F00080ED9AE00E948158809156079091570759
:105900006AE270E004960E941ED48C010097E1F0D8
:10591000209160073091610740E6429FC001439F9C
:10592000900D11246EE470E08A59984F0E941ED4A5
:1059300060E270E00E941ED4019690935707809316
:105940005607F801319710826091560770915707FA
:105950006C5F7F4F80ED9AE00E948F550C949939CF
:1059600080915607909157076AE270E005960E9471
:105970001ED48C010097E1F02091600730916107FF
:1059800040E6429FC001439F900D11246EE470E0F9
:105990008A59984F0E941ED460E270E00E941ED483
:1059A00001969093570780935607F801319710821C
:1059B00060915607709157076B5F7F4F80ED9AE0BB
:1059C0000E948A550C9499390E94C4C56093460779
:1059D00070934707809348079093490700914A07BF
:1059E00010914B0720914C0730914D07601B710BB4
:1059F000820B930B28EE33E040E050E00E94A5D0EC
:105A0000CA01B9012CE330E040E050E00E94A5D08B
:105A10007F936F933F932F9383EC93E09F938F93A8
:105A2000CE0101969F938F930E94E8D4E1EBF6E0BC
:105A300084910FB6F894DEBF0FBECDBF882349F026
:105A40009091C00095FFFCCF8093C6003196849161
:105A5000F5CFFE0131968191882339F09091C000F5
:105A600095FFFCCF8093C600F6CF8091C00085FFE4
:105A7000FCCF8AE08093C600CE0101960E949F92DF
:105A80008091B512882311F40C9499391092B512B3
:105A90000091190910E0000F111F0F5F1B4EF80154
:105AA00060817181882777FD8095982F0E9476CD3F
:105AB00020914702309148024091490250914A0298
:105AC0000E94D7CE181614F00C949939D8011D9263
:105AD0001C920C94993983E50E947E1B882311F453
:105AE0000C9499390E946A1B6B017C0180E50E942D
:105AF0007E1B882351F0C701B6010E9443CD6F3F42
:105B0000710509F010F40C941E3A6DE070E020E08D
:105B1000E22FEE0FFF0BE450FC4F8081918186173E
:105B2000970711F40C9499392F5FF2CF88E690E033
:105B30000E94A91F81110C94993983E50E947E1B54
:105B4000882371F0009168060E946A1B10E0000F24
:105B5000111F0F5F1B4E0E9443CDF80171836083BC
:105B60000E94FA790C94993983E50E947E1B882360
:105B700011F40C9499390E946A1B0E9443CD7093D2
:105B800000146093FF130C94993989E690E00E9409
:105B9000A91F81110C949939EDEBF3E084918823CE
:105BA00041F09091C00095FFFCCF8093C6003196E4
:105BB000F5CF4091F3135091F4136091F513709168
:105BC000F61321E030E082EE95E00E94BE18EAEB89
:105BD000F3E08491882341F09091C00095FFFCCFC1
:105BE0008093C6003196F5CF609101147091021434
:105BF000882777FD8095982F0E9476CDAB01BC0158
:105C000021E030E082EE95E00E94BE18E5EBF3E083
:105C10008491882341F09091C00095FFFCCF809340
:105C2000C6003196F5CF4091F7135091F81360916B
:105C3000F9137091FA1321E030E082EE95E00E94B2
:105C4000BE18E2EBF3E08491882341F09091C0000C
:105C500095FFFCCF8093C6003196F5CF6091031479
:105C600070910414882777FD8095982F0E9476CD37
:105C7000AB01BC0121E030E082EE95E00E94BE184D
:105C8000EEEAF3E08491882341F09091C00095FF03
:105C9000FCCF8093C6003196F5CF4091ED13509123
:105CA000EE136091EF137091F01321E030E082EE7B
:105CB00095E00E94BE18EBEAF3E08491882341F05E
:105CC0009091C00095FFFCCF8093C6003196F5CF30
:105CD0006091FF1370910014882777FD8095982FAD
:105CE0000E9476CDAB01BC0121E030E082EE95E070
:105CF0000E94BE18E7EAF3E08491882341F0909176
:105D0000C00095FFFCCF8093C6003196F5CF8091FF
:105D1000680690E00E94FF764AE050E0BC0182EE07
:105D200095E00E94E817E2EAF3E08491882341F0CD
:105D30009091C00095FFFCCF8093C6003196F5CFBF
:105D40008FEF9FEF0E94FF764AE050E0BC0182EEA9
:105D500095E00E94E8178091C00085FFFCCF8AE0A3
:105D60008093C6000C9499398DE690E00E94A91F9B
:105D700081110C94993987E993E00E94AE921092B8
:105D8000B51283E50E947E1B882371F0009168069E
:105D90000E946A1B10E0000F111F0F5F1B4E0E9434
:105DA00043CDD8016D937C9383E50E947E1B8823AD
:105DB00051F00E946A1B60934702709348028093DF
:105DC000490290934A0282E40E947E1B882351F08C
:105DD0000E946A1B60934B0270934C0280934D02A9
:105DE00090934E0286E40E947E1B882369F00E94F5
:105DF0006A1B609343027093440280934502909320
:105E0000460281E08093B5120E94FA790E94C4C5CF
:105E10004B015C010091680610E0F801EE0FFF1FD6
:105E2000EF5FFB4E60817181882777FD8095982F09
:105E30000E9476CD2B013C01F801EE0FFF1FEE0F03
:105E4000FF1FED50FC4E80819181A281B3818F8F25
:105E500098A3A9A3BAA3CC24CA94DC2C76016AE047
:105E6000362E0C94893A8091B30981110C9499399A
:105E70008FE693E00E94AE9283E50E947E1B88230A
:105E800041F00E946A1B0E9443CD709300146093FE
:105E9000FF130E94C4C54B015C010BE613E056E6FC
:105EA000E52E53E0F52E62E6C62E63E0D62E7AE0AC
:105EB000772E6091FF1370910014882777FD8095ED
:105EC000982F0E9476CD2091ED133091EE134091E2
:105ED000EF135091F0130E94D7CE18160CF077C034
:105EE0000E94C4C5681979098A099B09693E7340F3
:105EF0008105910508F461C0F8018491EBE6F3E0B7
:105F0000882349F09091C00095FFFCCF8093C60094
:105F100031968491F5CF4091F3135091F413609131
:105F2000F5137091F61322E030E082EE95E00E94C6
:105F3000BE18F7018491E6E6F3E0882349F09091DA
:105F4000C00095FFFCCF8093C60031968491F5CFB9
:105F50004091F7135091F8136091F9137091FA136F
:105F600022E030E082EE95E00E94BE18F6018491B6
:105F7000E2E6F3E0882349F09091C00095FFFCCF62
:105F80008093C60031968491F5CF4091ED135091E6
:105F9000EE136091EF137091F01321E030E082EE88
:105FA00095E00E94BE188091C00085FFFCCF7092E2
:105FB000C6000E94C4C54B015C010E940A770E9482
:105FC000031F0E94F1938091B409811172CF88E57B
:105FD00093E00E94AE920E94C4C5609352077093F2
:105FE000530780935407909355070C94993983E590
:105FF0000E947E1B882319F10E946A1B20E030E07A
:10600000A9010E94D4CC87FD0FC00E946A1B20E02A
:1060100030E04FE753E40E94D7CE181644F00E94B8
:106020006A1B0E9443CD05C060E070E002C06FEFC4
:1060300070E070931809609317090C9499398FEFE9
:1060400090E090931809809317090C949939109255
:106050001809109217090C949939269A2E980C94C5
:106060009939269A2E9A0C94993910926B090C94AE
:10607000993981E080936B090C94993983E50E94EA
:106080007E1B882399F00E946A1B20E030E04AE7DB
:1060900054E40E94A9CF0E9448CD609306027093F9
:1060A000070280930802909309021EC088E50E94AF
:1060B0007E1B81110C94633B89E50E947E1B81113C
:1060C0000C94633B8AE50E947E1B81110C94633B18
:1060D00085E40E947E1B81110C94633B0E94A37493
:1060E000129A479A0E940B751092AB090C94993939
:1060F0002CE334E038A32F8F0AE113E13AE2832E38
:1061000033E1932E4AEDA42E42E1B42E312CAF8D13
:10611000B8A18D91B8A3AF8F0E947E1B882309F48C
:106120005CC0B3E03B1252C00E946A1B6B017C0151
:1061300020E030E040EA51E40E94D4CC87FF3FC029
:10614000A7019601F80160817181828193810E948B
:10615000DBCC2B013C019B01AC016091EE127091F4
:10616000EF128091F0129091F1120E94A9CF6093EA
:10617000EE127093EF128093F0129093F112A3013C
:106180009201D4016D917D918D919C910E94A9CF36
:10619000F4016083718382839383D5016D917D9136
:1061A0008D919C910E9474CDA30192010E94A9CF70
:1061B0000E9448CDF5016083718382839383D80167
:1061C000CD92DD92ED92FC92139707C00E946A1B5C
:1061D000F801608371838283938333940C5F1F4F34
:1061E000F4E08F0E911C24E0A20EB11C34E03312B7
:1061F0008ECF0C949939E0EEF2E08491882311F46B
:106200000C9499399091C00095FFFCCF8093C60003
:106210003196F3CF00915607109157070B5F1F4F30
:106220006AE270E0C8010E941ED4009719F0FC01D8
:1062300031971082C8010E949F920E94C4C560934A
:106240004A0770934B0780934C0790934D0781E06A
:106250008093AB090C949939EDEDF2E08491882399
:1062600041F09091C00095FFFCCF8093C60031961D
:10627000F5CF409156095091570960915809709196
:10628000590922E030E082EE95E00E94BE18EAED66
:10629000F2E08491882341F09091C00095FFFCCFFB
:1062A0008093C6003196F5CF40915A0950915B0911
:1062B00060915C0970915D0922E030E082EE95E02A
:1062C0000E94BE18E7EDF2E08491882341F090919E
:1062D000C00095FFFCCF8093C6003196F5CF40916A
:1062E0005E0950915F09609160097091610922E037
:1062F00030E082EE95E00E94BE18E4EDF2E0849179
:10630000882341F09091C00095FFFCCF8093C60098
:106310003196F5CF4091620950916309609164090B
:106320007091650922E030E082EE95E00E94BE188F
:10633000EAECF2E08491882341F09091C00095FF4F
:10634000FCCF8093C6003196F5CF0E94FD740E9469
:1063500076CD20911A1330911B1340911C1350914C
:106360001D130E94DBCCAB01BC0122E030E082EEC9
:1063700095E00E94BE18E7ECF2E08491882341F09A
:106380009091C00095FFFCCF8093C6003196F5CF69
:1063900081E00E94FD740E9476CD20911E13309101
:1063A0001F1340912013509121130E94DBCCAB01AD
:1063B000BC0122E030E082EE95E00E94BE18E4ECE1
:1063C000F2E08491882341F09091C00095FFFCCFCA
:1063D0008093C6003196F5CF82E00E94FD740E9442
:1063E00076CD2091221330912313409124135091A4
:1063F00025130E94DBCCAB01BC0122E030E082EE31
:1064000095E00E94BE188091C00085FFFCCF8AE015
:106410008093C6008EC780E00E94736D8AC781E0BA
:106420000E94736D86C79091C00095FFFCCF80934A
:10643000C60081918111F7CF8091C00085FFFCCF0C
:106440008AE08093C600ECEBF2E08491882341F06F
:106450009091C00095FFFCCF8093C6003196F5CF98
:10646000659903C0E8E9F3E009C0E2EAF3E006C099
:106470009091C00095FFFCCF8093C600819181115F
:10648000F7CF8091C00085FFFCCF8AE08093C600E3
:10649000E4EBF2E08491882341F09091C00095FFF5
:1064A000FCCF8093C6003196F5CF8091030181FD2A
:1064B00003C0E8E9F3E009C0E2EAF3E006C0909126
:1064C000C00095FFFCCF8093C60081918111F7CF6A
:1064D0008091C00085FFFCCF8AE08093C600ECEA83
:1064E000F2E08491882341F09091C00095FFFCCFA9
:1064F0008093C6003196F5CF4B9903C0E8E9F3E0ED
:1065000009C0E2EAF3E006C09091C00095FFFCCF1D
:106510008093C60081918111F7CF8091C00085FFE3
:10652000FCCF8AE08093C60004C7D8018D918D010D
:106530000E947E1B882349F00E946A1B0E9448CD5E
:10654000F7016083718382839383F4E0EF0EF11C83
:1065500024E00034120749F70E94896CEAC60CE374
:1065600014E09AE2E92E93E1F92ED8018D918D0184
:106570000E947E1B882339F00E946A1BF70160830A
:10658000718382839383F4E0EF0EF11C24E00034E6
:10659000120759F7CEC683E50E947E1B882351F06F
:1065A0000E946A1B60930213709303138093041379
:1065B0009093051384E50E947E1B882309F4B9C6D5
:1065C0000E946A1B6093FE127093FF128093001367
:1065D00090930113AEC683E50E947E1B882351F081
:1065E0000E946A1B6093061370930713809308132D
:1065F0009093091384E50E947E1B882351F00E942A
:106600006A1B6093EA127093EB128093EC129093E2
:10661000ED1282E40E947E1B882361F00E946A1BB7
:106620000E9448CD60933A1370933B1380933C13C0
:1066300090933D1388E50E947E1B882351F00E94B1
:106640006A1B6093FA127093FB128093FC12909372
:10665000FD1289E50E947E1B882351F00E946A1B6F
:106660006093F6127093F7128093F8129093F912D8
:106670008AE50E947E1B882351F00E946A1B60936A
:10668000F2127093F3128093F4129093F51285E452
:106690000E947E1B882309F44CC60E946A1B6093EB
:1066A000EE127093EF128093F0129093F11241C6A4
:1066B000F4E0EF0EF11C24E00F33120709F439C6A1
:1066C000D8018D918D010E947E1B882389F30E9441
:1066D0006A1BF7016083718382839383E9CF8AED1C
:1066E00090E00E94A91F811124C688E50E947E1BAC
:1066F000882321F10091680610E00E946A1BF801CE
:10670000EE0FFF1FEE0FFF1FE15FFD4F60837183F0
:1067100082839383E091680634E0E39FF0011124C3
:10672000E15FFD4F80819181A281B38180937909DE
:1067300090937A09A0937B09B0937C0989E50E9424
:106740007E1B882321F10091680610E00E946A1BDD
:10675000F801EE0FFF1FEE0FFF1FE95EFD4F608394
:10676000718382839383E091680684E0E89FF0015F
:106770001124E95EFD4F80819181A281B3818093D4
:106780007D0990937E09A0937F09B0938009E1EB86
:10679000F6E08491882341F09091C00095FFFCCFF2
:1067A0008093C6003196F5CFECE9F2E0849188231E
:1067B00041F09091C00095FFFCCF8093C6003196C8
:1067C000F5CF1092680680916806823008F042C0CA
:1067D000E0E3F5E08191882339F09091C00095FFC6
:1067E000FCCF8093C600F6CFE091680694E0E99F65
:1067F000F0011124E15FFD4F40815181628173817D
:1068000022E030E082EE95E00E94BE18E2ECF3E078
:106810008191882339F09091C00095FFFCCF80933F
:10682000C600F6CFE0916806A4E0EA9FF0011124CB
:10683000E95EFD4F408151816281738122E030E049
:1068400082EE95E00E94BE18809168068F5F80936B
:106850006806B9CF8091C00085FFFCCF8AE08093A5
:10686000C60067C583E50E947E1B882309F461C5C5
:106870000E946A1B0E9443CD70932E0260932D02EA
:1068800058C583E50E947E1B882309F452C50E94E7
:106890006A1B0E9443CD70932C0260932B0249C562
:1068A00083E50E947E1B882331F00E946A1B0E94B0
:1068B00043CD8B0102C000E911E080E50E947E1B00
:1068C000882331F00E946A1B0E9443CD7B0104C0E3
:1068D00058EEE52E53E0F52E20E030E0A901B80196
:1068E00085E20E9458C8B701882777FD8095982FC8
:1068F0000E94F3C585E20E9479CB1BC580E50E940A
:106900007E1B882351F00E946A1B6093690270937A
:106910006A0280936B0290936C0289E40E947E1B52
:10692000882361F00E946A1B0E94EA7F60936502DF
:1069300070936602809367029093680284E40E94D9
:106940007E1B882361F00E946A1B0E94F67F609381
:10695000610270936202809363029093640283E405
:106960000E947E1B882351F00E946A1B60935D0287
:1069700070935E0280935F02909360020E94E076C3
:10698000E4ECF3E08191882339F09091C00095FF09
:10699000FCCF8093C600F6CFE7ECF3E0819188232B
:1069A00039F09091C00095FFFCCF8093C600F6CFE0
:1069B0004091690250916A0260916B0270916C0281
:1069C00022E030E082EE95E00E94BE18EBECF3E0AE
:1069D0008191882339F09091C00095FFFCCF80937E
:1069E000C600F6CF609165027091660280916702E1
:1069F000909168020E94F07FAB01BC0122E030E080
:106A000082EE95E00E94BE18EFECF3E081918823BE
:106A100039F09091C00095FFFCCF8093C600F6CF6F
:106A200060916102709162028091630290916402B0
:106A30000E94FC7FAB01BC0122E030E082EE95E0D9
:106A40000E94BE18E3EDF3E08191882339F0909124
:106A5000C00095FFFCCF8093C600F6CF40915D0249
:106A600050915E0260915F027091600222E030E01E
:106A700082EE95E00E94BE188091C00085FFFCCF99
:106A80008AE08093C60055C483E50E947E1B88235C
:106A900019F00E946A1B03C060E070E0CB010E9405
:106AA000806C47C485E40E947E1B882341F00E94CD
:106AB0006A1B0E9443CD8B0177FD0AC002C000E033
:106AC00010E0C12CD12C46E1E42E43E4F42E06C0A4
:106AD000C12CD12C3CE8E32E32E4F32E83E50E9456
:106AE0007E1B882321F00E946A1B6B017C0183E4DA
:106AF0000E947E1B882331F00E946A1B0E9443CDB6
:106B00009B0102C025E030E0A801C701B6010E9448
:106B1000217A0FC40E94A3740CC40E94881509C472
:106B20000E94051406C48091A40A882309F401C4B4
:106B300089E50E947E1B811106C081E08093A50A31
:106B40008093C50AF6C30E946A1B6B017C0120E09A
:106B500030E0A9010E94D4CC882379F38091A60A61
:106B60009091A70AA091A80AB091A90A8093C10A9E
:106B70009093C20AA093C30AB093C40AC092A60A13
:106B8000D092A70AE092A80AF092A90AD2C38091F3
:106B9000A40A882309F4CDC389E50E947E1B8823BB
:106BA00021F00E946A1B6B017C0120E030E0A9010A
:106BB000C701B6010E94D4CC811116C08091C10AD0
:106BC0009091C20AA091C30AB091C40A8093A60A08
:106BD0009093A70AA093A80AB093A90A81E0809392
:106BE000A50A8093C50AA5C38090AE0A9090AF0A0B
:106BF000A090B00AB090B10A20E030E0A901C50130
:106C0000B4010E94D4CC81110DC080E090E0A0E2DC
:106C1000B1E48093AE0A9093AF0AA093B00AB09308
:106C2000B10A26C02091A60A3091A70A4091A80A6D
:106C30005091A90A6091AA0A7091AB0A8091AC0A9E
:106C40009091AD0A0E94FACB20E030E04CE052E493
:106C50000E94FBCB9B01AC01C501B4010E94FBCBA0
:106C60006093AE0A7093AF0A8093B00A9093B10A12
:106C7000C092AA0AD092AB0AE092AC0AF092AD0A96
:106C80002091AE0A3091AF0A4091B00A5091B10AFA
:106C9000C701B6010E94FBCB2091A60A3091A70A3A
:106CA0004091A80A5091A90A0E94FACB6B017C017D
:106CB0006091B7097091B80965507109882777FD0F
:106CC0008095982F0E9476CD9B01AC01C701B6013B
:106CD0000E94D7CE181624F485EA9AE00E94222654
:106CE00083E08093C50A1092A50A8091BF0A909113
:106CF000C00A181619060CF01CC38091B20A87301E
:106D000009F017C38091AE0A9091AF0AA091B00A22
:106D1000B091B10A80935A0990935B09A0935C09E2
:106D2000B0935D09198220E030E040EF52E46091B9
:106D300033027091340280913502909136020E94A4
:106D4000DBCCFE0131966F017B018C0122E639E03C
:106D50004EE559E06AE579E086E599E00E94F36145
:106D60000E94A374E6C280E50E947E1B882309F47A
:106D7000E0C20E946A1B0E9443CD7093C0096093D9
:106D8000BF09D7C283E50E947E1B882389F00E9439
:106D90006A1B0E9443CDCB01AA2797FDA095BA2F6D
:106DA0008093D2099093D309A093D409B093D509C5
:106DB0001092D109BEC28EE08093AC091092CB0A2A
:106DC0008BE080936C09E7E6F2E08491882341F040
:106DD0009091C00095FFFCCF8093C6003196F5CF0F
:106DE0008091C00085FFFCCF8AE08093C60083E6D7
:106DF00092E00E94E71A9DC28091AC098E3009F0A2
:106E000098C28CE592E00E94E71A8FE492E00E941B
:106E1000E71A8BE492E00E94E71A81E08093CB0AA4
:106E200088C28091AC098E3009F083C287E492E079
:106E30000E94E71A1092CB0A7CC28091AC098E3076
:106E400009F077C284E40E947E1B882349F00E94E7
:106E50006A1B0E9443CD7093CD0A6093CC0A69C22D
:106E60008DE590E09093CD0A8093CC0A62C2809128
:106E7000AC098E3009F05DC288E40E947E1B882335
:106E800049F00E946A1B0E9443CD7093CA0A609326
:106E9000C90A4FC21092CA0A1092C90A4AC2809106
:106EA000AC098E3009F045C283E492E00E94E71AF3
:106EB0006091C90A7091CA0A8091CC0A9091CD0A5A
:106EC000680F791F62537109882777FD8095982F85
:106ED0000E9476CD60935E0970935F09809360098C
:106EE00090936109198220E030E040EA50E460911B
:106EF0003702709138028091390290913A020E94D3
:106F0000DBCC9E012F5F3F4F69017B018C0122E6A4
:106F100039E04EE559E06AE579E086E599E00E94BE
:106F2000F3610E94A3748CE080936C0902C280918B
:106F3000AC098E3009F0FDC1109256091092570924
:106F4000109258091092590910925A0910925B092F
:106F500010925C0910925D0922E639E04EE559E095
:106F60006AE579E086E599E00E94BE6BEDE3F2E028
:106F70008491882341F09091C00095FFFCCF8093CD
:106F8000C6003196F5CF8091C00085FFFCCF8AE026
:106F90008093C6006091C90A7091CA0A8091CC0A98
:106FA0009091CD0A680F791F882777FD8095982FDB
:106FB0000E9476CD60935E0970935F0980936009AB
:106FC00090936109198220E030E040EA50E460913A
:106FD0003702709138028091390290913A020E94F2
:106FE000DBCCDE0111966D017B018C0122E639E0DC
:106FF0004EE559E06AE579E086E599E00E94F361A3
:107000000E94A374E1E3F2E08491882341F090911F
:10701000C00095FFFCCF8093C6003196F5CF8091DC
:10702000C00085FFFCCF8AE08093C60082C184E562
:107030000E947E1B882309F438C10E946A1B0E94AB
:1070400048CD609368066230A8F1E1EBF6E08491E8
:10705000882341F09091C00095FFFCCF8093C6003B
:107060003196F5CFE7EDF3E08191882339F09091E7
:10707000C00095FFFCCF8093C600F6CF40E050E003
:107080006091680682EE95E00E941F18E9EDF3E03A
:107090008191882339F09091C00095FFFCCF8093B7
:1070A000C600F6CF8091C00085FFFCCF8AE08093B8
:1070B000C6003FC186E40E947E1B8823E1F00E9447
:1070C0006A1B6B017C016093F7087093F80880934A
:1070D000F9089093FA0820E030E0A9010E94D7CE89
:1070E00018165CF4C0920A02D0920B02E0920C02D5
:1070F000F0920D0202C0D12C02C0DD24D39419827B
:107100001A821B821C8219861A861B861C86809115
:10711000790990917A09A0917B09B0917C098D83BE
:107120009E83AF83B88780917D0990917E09A0915D
:107130007F09B09180098D879E87AF87B88BC090FB
:10714000680680911909C81609F485C090E1E6E542
:10715000F9E0A7E0B9E001900D929A95E1F70C2DC6
:1071600010E0E82EF12CE1E0F0E0EC0FFD1FB4E0C0
:107170008B9FE00DF11D11242081318142815381CB
:107180006091560970915709809158099091590959
:107190000E94FACBF801EE0FFF1FEE0FFF1F21E058
:1071A00030E02C0F3D1FE20FF31F2081318142811F
:1071B00053810E94FBCB60935609709357098093CB
:1071C000580990935909F7013296EE0FFF1FEE0F01
:1071D000FF1F81E090E08C0F9D1FE80FF91F2081B9
:1071E00031814281538160915A0970915B0980918C
:1071F0005C0990915D090E94FACBF8013296EE0F7E
:10720000FF1FEE0FFF1FA1E0B0E0AC0FBD1FEA0FA4
:10721000FB1F20813181428153810E94FBCB60930F
:107220005A0970935B0980935C0990935D09C09241
:10723000190922E639E04EE559E06AE579E086E58C
:1072400099E00E94BE6BDD2031F0809167068111CC
:1072500002C00E94591DE1EBF6E08491882341F0C1
:107260009091C00095FFFCCF8093C6003196F5CF7A
:10727000EAEEF3E08191882339F09091C00095FF08
:10728000FCCF8093C600F6CF6091190970E04AE008
:1072900050E082EE95E00E94E8178091C00085FFE3
:1072A000FCCF8AE08093C60044C0E1EBF6E0849115
:1072B000882341F09091C00095FFFCCF8093C600D9
:1072C0003196F5CFEEE1F2E08491882341F0909180
:1072D000C00095FFFCCF8093C6003196F5CF80911A
:1072E00060079091610720E6289FF001299FF00D2B
:1072F0001124EA59F84F8191882339F09091C00008
:1073000095FFFCCF8093C600F6CFECE1F2E08491CC
:10731000882341F09091C00095FFFCCF8093C60078
:107320003196F5CF8091C00085FFFCCF8AE0809335
:10733000C6000E949A1BEBC18091C50A8330C0F43D
:1073400081E08093A50AEEE2F4E08491882341F085
:107350009091C00095FFFCCF8093C6003196F5CF89
:107360008091C00085FFFCCF8AE08093C600E1CF0A
:107370008091B20A873011F00C943127E7E1F4E0F4
:107380008491882341F09091C00095FFFCCF8093B9
:10739000C6003196F5CF8091C00085FFFCCF8AE012
:1073A0008093C600C6CF20E030E040EC50E462E0BD
:1073B00070E08CE699E00E94802180E090E0A0ECF3
:1073C000B0E48093750990937609A0937709B09300
:1073D00078090C94F12781E090E00E94BF1820E02A
:1073E00030E0A90161E070E08CE699E00E94802124
:1073F0000C94FC2720E030E0A90160E070E08CE60E
:1074000099E00E9480210C9436280E940A770E94FD
:10741000031F0E94F1930C949F2B0E94731BAB01DE
:10742000BC014093C70B5093C80B6093C90B70937A
:10743000CA0B84EA9BE00E9473467BCF0E946A1BC2
:107440000E9443CD0C94872D0E94C4C58B019C01E2
:10745000C701B6016053784F8F4F9F4F601B710B70
:10746000820B930B28EE33E040E050E00E94A5D061
:10747000BA01A9012AE030E082EE95E00E941418DA
:107480008091C00085FFFCCF3092C6000E94C4C529
:107490004B015C010E940A770E94031F0E94F19336
:1074A000FFEFCF16DF06EF06FF0609F0ACC02F8D09
:1074B00038A149A15AA1C301B2010E94D7CEE091DF
:1074C0006806F0E08F01000F111F000F111F0D5013
:1074D0001C4EEE0FFF1FEF5FFB4E6081718118168F
:1074E0000CF079C0882777FD8095982F0E9476CD83
:1074F00020E030E040EA50E40E94FACB9B01AC016E
:10750000D8016D917D918D919C910E94D7CE87FF7E
:10751000B6C00E94C4C5681979098A099B09693EE9
:1075200073408105910508F4B5CFE3E9F3E0849158
:10753000882341F09091C00095FFFCCF8093C60056
:107540003196F5CF4091F3135091F4136091F513F8
:107550007091F61322E030E082EE95E00E94BE18B2
:10756000EEE8F3E08491882341F09091C00095FF0C
:10757000FCCF8093C6003196F5CF4091F713509120
:10758000F8136091F9137091FA1322E030E082EE63
:1075900095E00E94BE18EAE8F3E08491882341F068
:1075A0009091C00095FFFCCF8093C6003196F5CF37
:1075B000F7FE4ACFE0ECF3E006C09091C00095FFE3
:1075C000FCCF8093C60081918111F7CF8091C000DC
:1075D00085FFFCCF59CF882777FD8095982F0E9493
:1075E00076CD20E030E040EA50E40E94FBCB9B01E6
:1075F000AC01F80160817181828193810E94D4CCB9
:107600001816ECF586CFF7FC2FC0E0916806F0E085
:107610008F01000F111F000F111F0D501C4EEE0F98
:10762000FF1FEF5FFB4E60817181882777FD80959A
:10763000982F0E9476CD9B01AC01D8016D917D9170
:107640008D919C910E94FACB0E9443CD97FF07C079
:1076500090958095709561957F4F8F4F9F4F6730C4
:107660007105810591055CF4F7FC14C00E94C4C546
:107670006C197D09603D774008F44BCF0BC00E9428
:10768000C4C56B017C016F3FBFEF7B078B079B0776
:1076900059F73FCF8CE793E00E94AE920E94C4C599
:1076A00060934A0770934B0780934C0790934D0764
:1076B0000E94C4C560935207709353078093540788
:1076C0009093550736CE0E94A37488E50E947E1BD6
:1076D00081115F9A89E50E947E1B81118A9A8AE551
:1076E0000E947E1B882341F09FB7F8948091080187
:1076F0008160809308019FBF85E40E947E1B8823E0
:1077000011F40C947430129A479A0C947430A29627
:107710000FB6F894DEBF0FBECDBFDF91CF911F91A2
:107720000F91FF90EF90DF90CF90BF90AF909F9020
:107730008F907F906F905F904F903F900895FC01E5
:107740004091560950915709609158097091590913
:1077500046875787608B718B40915A0950915B091E
:1077600060915C0970915D09428B538B648B758BC2
:1077700040915E0950915F096091600970916109C3
:10778000468B578B608F718F0895EF92FF920F9306
:107790001F93CF93DF93EC016F3F4FEF740759F1C5
:1077A000EBE3F7E020E030E0819191918F3FAFEF84
:1077B0009A0741F18617970769F5F901EE0FFF1F48
:1077C000E55CF84F8FEF9FEF9183808380913207C4
:1077D000909133070197861B970B6AE070E00E9437
:1077E0007ED024E1289FF001299FF00D1124E75954
:1077F000F94F80E28083EBE3F7E021E030E00FEF28
:107800001FEF0EC0F901EE0FFF1FE55CF84F71830B
:107810006083F1CF2F5F3F4F2530310529F6EBCF45
:1078200080819181019621F5A90180E090E07F019E
:1078300062EDE61AF10845305105D1F00296B70124
:10784000680F791F6E527F4FDB016D917C916F3F06
:10785000BFEF7B0751F071836083DA01AA0FBB1F72
:10786000A55CB84F0D931C9303C04F5F5F4FE3CFF0
:107870002F5F3F4F32962630310591F6EBE3F7E06C
:1078800020E030E081919191019629F02F5F3F4FE8
:1078900025303105B9F73AA329A3DF91CF911F9184
:1078A0000F91FF90EF90089560913B0770913C0716
:1078B0006CDF0C949C892F923F924F925F926F9253
:1078C0007F928F929F92AF92BF92CF92DF92EF9270
:1078D000FF920F931F93CF93DF931F92CDB7DEB725
:1078E000F0E6BF2EA4E02A2E312C07E714E0BAE020
:1078F000AB2E8DEEE82E84E0F82E9924939480919F
:107900006306909164062091650630916606821B9D
:10791000930B8F779927892B09F429C280915C07F3
:1079200090915D0704970CF022C282EE95E00E94D0
:107930000A1780935B071092B00920915907309184
:107940005A078A3061F08D3051F08A3321F49091DA
:107950005807992321F02F3531050CF429C1211541
:10796000310509F443C180915E0790915F07B89E8D
:107970006001B99ED00C1124F601E20FF31FEA5901
:10798000F84F10822091580721110DC1FC01EE59CA
:10799000F84F108296012A59384F39016EE470E091
:1079A000C9010E941ED40097F1F19093570780936C
:1079B0005607861997098C0D9D1D4AE050E060E03E
:1079C00070E08959984F0E9474D26093EF087093C9
:1079D000F0088093F1089093F2084090EB085090E3
:1079E000EC086090ED087090EE083FEF431A530AE0
:1079F000630A730AC0905E07D0905F07641575052F
:107A00008605970509F4F5C0BC9CC001BD9C900D8E
:107A1000112466E975E08A59984F0E94E3D3892BB7
:107A200009F0E7C077C16AE270E0C3010E941ED48A
:107A3000892B09F444C0E7EBF6E08491882341F0F8
:107A40009091C00095FFFCCF8093C6003196F5CF92
:107A5000E0EFF4E08491882341F09091C00095FF1D
:107A6000FCCF8093C6003196F5CF4091EB08509142
:107A7000EC086091ED087091EE082AE030E082EEAB
:107A800095E00E94C5178091C00085FFFCCF8AE079
:107A90008093C60010925A0710925907D6C280915F
:107AA000EF089091F008A091F108B091F20880934E
:107AB000EB089093EC08A093ED08B093EE0880914A
:107AC0005E0790915F07B89E6001B99ED00C1124AB
:107AD000C6018A59984F3C0167E470E00E941ED4A9
:107AE000009709F44BC09093570780935607861967
:107AF00097098C0D9D1D60E070E08959984F0E9498
:107B00000CD10E9443CD6430710508F037C08091DC
:107B1000670681111AC08091D00A81112FC0F70128
:107B20008491EDEEF4E0882349F09091C00095FF38
:107B3000FCCF8093C60031968491F5CF8091C00030
:107B400085FFFCCFA092C60019C0F8018491E7E739
:107B5000F4E0882349F09091C00095FFFCCF80931A
:107B6000C60031968491F5CF8091C00085FFFCCF8F
:107B7000A092C6008DE694E00E94AE9280915E07CE
:107B800090915F070196B1010E9492D090935F0798
:107B900080935E0780915C0790915D0701969093BA
:107BA0005D0780935C0710925A0710925907A7CE81
:107BB0008B3311F4909258079091580791119FCEF2
:107BC00040915E0750915F07B9016F5F7F4F7093DF
:107BD0005A0760935907B49EF001B59EF00D112429
:107BE000E20FF31FEA59F84F808389CE10925807AD
:107BF0002CC2BC9C3001BD9C700C1124C3018A595D
:107C0000984F2C016AE270E00E941ED4009791F513
:107C1000E7EBF6E08491882341F09091C00095FF56
:107C2000FCCF8093C6003196F5CFEAE1F5E0849170
:107C3000882341F09091C00095FFFCCF8093C6004F
:107C40003196F5CF4091EB085091EC086091ED082A
:107C50007091EE082AE030E082EE95E00E94C517B0
:107C60008091C00085FFFCCF8AE08093C6000E940F
:107C7000C21B10CF20E0D12CF301E20FF11DEA5915
:107C8000F84F30813A3219F02F5FD326F5CF909319
:107C900057078093560784199509860D971D60E054
:107CA00070E08959984F0E940CD10E9443CD2D2D30
:107CB00030E02617370709F4F2CEE7EBF6E08491BF
:107CC000882341F09091C00095FFFCCF8093C600BF
:107CD0003196F5CFE4E4F5E08491882341F090916A
:107CE000C00095FFFCCF8093C6003196F5CF409140
:107CF000EB085091EC086091ED087091EE082AE0D5
:107D000030E082EE95E00E94C5178091C00085FFAB
:107D1000FCCFAACFE7EBF6E08491882341F0909165
:107D2000C00095FFFCCF8093C6003196F5CFE3E607
:107D3000F5E08491882341F09091C00095FFFCCF3D
:107D40008093C6003196F5CF4091EB085091EC0836
:107D50006091ED087091EE082AE030E082EE95E047
:107D60000E94C5178091C00085FFFCCF7DCF809118
:107D7000D20A8823E9F08091590790915A07892BFC
:107D8000B9F405E514E03AE0532E77247394EE2419
:107D9000EA94FE2C56E6C52E57E0D52E60E8A62EB6
:107DA000BB24B39470E6672EE4E08E2E912CAFC016
:107DB0008091B009882309F448C18091B10987FDF9
:107DC00044C180688093B10988E694E00F90DF9108
:107DD000CF911F910F91FF90EF90DF90CF90BF90C8
:107DE000AF909F908F907F906F905F904F903F905B
:107DF0002F900C94E71A80915C0790915D0704978F
:107E00000CF023C18091AC0B9091AD0BA091AE0B07
:107E1000B091AF0B8093C70B9093C80BA093C90B85
:107E2000B093CA0B84EA9BE095D61C0180935B0754
:107E3000682F8CE699E029820E94102529812A303A
:107E400019F02D3009F07AC08091A50A882399F0A5
:107E50004091BF0B5091C00B6091C10B7091C20B50
:107E60004093C70B5093C80B6093C90B7093CA0B18
:107E700084EA9BE038D74091C70B5091C80B6091C2
:107E8000C90B7091CA0B8091BF0B9091C00BA09150
:107E9000C10BB091C20B481759076A077B0708F05E
:107EA0007FC08091A50A81117BC020915907309134
:107EB0005A072115310509F499CE80915E079091FA
:107EC0005F07689EF001699EF00D1124E20FF31F19
:107ED000EA59F84F1082FC01EE59F84F7082209158
:107EE0005C0730915D072F5F3F4F30935D07209314
:107EF0005C070196B4010E9492D090935F07809333
:107F00005E071092580710925A0710925907409135
:107F1000C70B5091C80B6091C90B7091CA0B80912F
:107F2000BF0B9091C00BA091C10BB091C20B481731
:107F300059076A077B0708F088C05DCF2A3329F408
:107F400080915807882309F47FCF80915907909139
:107F50005A078F3591050CF077CFFFEF2F163F06AC
:107F600009F472CF2B3311F47092580720915807FF
:107F70002111CDCF20915E0730915F07AC014F5F9B
:107F80005F4F50935A0740935907629EF001639EDA
:107F9000F00D1124E80FF91FEA59F84F2082B7CFEE
:107FA000F8018491E5E5F4E0882349F09091C00060
:107FB00095FFFCCF8093C60031968491F5CF8091D8
:107FC000C00085FFFCCF5092C6008BE494E00E9475
:107FD000AE9270926C091092AB091092AE09F092B9
:107FE000C009E092BF090E94C4C560934607709320
:107FF000470780934807909349078091A50A8823F3
:1080000079F0F6019501119221503040E1F710927C
:108010005A071092590780ED9AE00E94915904C0C6
:1080200080ED9AE00E944C5961E080ED9AE00E9458
:108030008D578091A40A882309F437CF85EA9AE006
:108040007EDB85EA9AE030DC30CF0F90DF91CF9174
:108050001F910F91FF90EF90DF90CF90BF90AF9066
:108060009F908F907F906F905F904F903F902F9058
:108070000895CF93DF9380915C0790915D070397FC
:108080000CF419DC60E080ED9AE00E948D5780913D
:108090005C0790915D07892B09F470C08091D00A2C
:1080A0008823E1F0809160079091610720E6289F86
:1080B000E001299FD00D1124CA59D84F60EB75E01B
:1080C000CE010E94E3D3892BF1F4BE0180ED9AE04A
:1080D0000E941D578091D10A882319F00E943326EF
:1080E0002AC0EDEAF5E08491882341F09091C00028
:1080F00095FFFCCF8093C6003196F5CF8091C000EC
:1081000085FFFCCF15C080ED9AE00E948158EBE915
:10811000F5E08491882341F09091C00095FFFCCF59
:108120008093C6003196F5CF8091C00085FFFCCFCB
:108130008AE08093C60080915C0790915D07823051
:10814000910544F02091AE09211104C021E0209353
:10815000AF0902C01092AF09019790935D07809319
:108160005C078091600790916107019664E070E080
:108170000E9492D090936107809360070E940A77D3
:108180000E94031F0E94D16C8CE699E00E94B620E9
:10819000DF91CF910C94F19324E434E0FC0131831E
:1081A00020832781222311F0049680C6089580ED54
:1081B0009AE00C94845080EA9BE0EEDF8EE59BE031
:1081C000EBDF8FE39BE0E8DF80E29BE0E5DF8FEF12
:1081D0009AE0E2CF8FEF8EBD0DB407FEFDCF8EB5D6
:1081E00008958EBD0DB407FEFDCF089561E0FC013A
:1081F00080810C94DDC7FC012281322F306A3695D4
:108200003CBD20FD06C031E0263009F430E0232FCC
:1082100001C020E02DBD60E0FC0180810C94DDC731
:10822000CF92DF92EF92FF920F931F93CF93DF9342
:10823000EC018B017A010E94C4C56B01CBDF8B83FB
:108240008F3F49F40E94C4C56C197D096D3271409D
:10825000A8F381E103C08E3F31F08FE08983CE0126
:10826000C5DF80E024C0E114F104E1F081E0E81A08
:10827000F1088FEF8EBDF8012FEFCF01801B910B1E
:108280008E159F0538F40DB407FEFDCF8EB5819392
:108290002EBDF3CF0DB407FEFDCF8EB5F801EE0D68
:1082A000FF1D808397DF96DFCE01A0DF81E0DF91A5
:1082B000CF911F910F91FF90EF90DF90CF90089595
:1082C0000F931F93CF93DF93EB010E94C4C58B01E3
:1082D00081DF8F3F49F00E94C4C5601B710B6C1792
:1082E0007D07B0F380E001C081E0DF91CF911F9165
:1082F0000F910895CF92DF92FF920F931F93CF9328
:10830000DF9300D01F92CDB7DEB76C01F62E298324
:108310003A834B835C836FDF6CE271E0C601D0DF90
:108320008F2D80645EDF08E110E05C814B813A8133
:108330002981DA01C901002E04C0B695A795979549
:1083400087950A94D2F729833A834B835C8349DF6C
:108350000850110929813A814B815C81083F8FEFD8
:10836000180739F7FF2029F0E8E0FE1621F08FEF1B
:1083700003C085E901C087E834DFFCE0FF1201C0DB
:1083800029DF10E027DFF601838387FF04C01F3F4A
:1083900011F01F5FF7CF0F900F900F900F90DF91AC
:1083A000CF911F910F91FF90DF90CF900895BF92D2
:1083B000CF92DF92EF92FF920F931F93CF93DF93B1
:1083C000EC01B62E1C82198248830E94C4C58B0121
:1083D00061E088810E94A4C7CE0108DF60E082E3EB
:1083E0000E94A4C761E083E30E94A4C761E084E324
:1083F0000E94A4C761E085E30E94A4C761E085E311
:108400000E94DDC785E08A8382E58CBD1DBC2AE021
:10841000F22E8FEFE6DEFA94E1F720E030E0A901DA
:1084200060E0CE0167DFF82E8B8381E0F81649F01B
:108430000E94C4C5601B710B613D774070F381E001
:1084400046C02AEA31E040E050E068E0CE0152DF69
:1084500082FF02C0FC820CC094E0F92EBBDE8B834D
:10846000FA94E1F78A3A11F082E031C082E08C831D
:108470008C81823031F4C12CD12CE12C80E4F82E97
:1084800003C0C12CD12C760120E030E0A90167E3C4
:10849000CE0130DFA701960169E2CE012BDF8B838D
:1084A000882349F00E94C4C5601B710B613D774071
:1084B00058F38AE00CC08C818230B1F420E030E0C7
:1084C000A9016AE3CE0116DF882329F088E08983B9
:1084D000CE018CDE14C07EDE807C803C11F483E013
:1084E0008C8378DE77DE76DECE0180DE86E08B154B
:1084F00018F488E1898303C0BA8281E001C080E07A
:10850000DF91CF911F910F91FF90EF90DF90CF906F
:10851000BF9008950F931F93CF93DF93EC018901D0
:108520008C81833039F039E0440F551F661F771F67
:108530003A95D1F79A01AB0161E1CE01DBDE811101
:1085400009C040E052E0B801CE01DF91CF911F9108
:108550000F9166CE84E08983CE0148DE80E0DF9112
:10856000CF911F910F910895CF93DF93EC016EBDD2
:1085700020E030E00DB407FEFDCFFA01E20FF31F5B
:1085800080818EBD0DB407FEFDCF81818EBD2E5F33
:108590003F4F211582E0380769F70DB407FEFDCF84
:1085A0008FEF1FDE8FEF1DDE15DE8B838F71853021
:1085B00031F083E18983CE0119DE80E001C081E0E2
:1085C000DF91CF9108950F931F93CF93DF93EC0129
:1085D00089018C81833039F089E0440F551F661F73
:1085E000771F8A95D1F79A01AB0168E1CE0182DE4F
:1085F000882311F086E01EC0A8016EEFCE01B4DF23
:108600008823C9F068E572E0CE015ADE182F811187
:1086100002C087E10FC020E030E0A9016DE0CE018B
:1086200069DE811106C0D6DD811103C0CE01DEDD19
:1086300005C086E18983CE01D9DD10E0812FDF916D
:10864000CF911F910F910895CF93DF93EC019C017F
:108650002C5F3F4F41E050E060E070E0898D9A8DE3
:108660000E94E04D882399F04D895E896F89788D4D
:10867000452B462B472B59F44C815D816E817F81C0
:108680004D8B5E8B6F8B788F998190689983DF918A
:10869000CF910895CF92DF92EF92FF920F931F93A5
:1086A000CF93DF93EC0189899A89AB89BC89803E9D
:1086B0009F4FAF41B10510F080E06AC0CE01C4DF2A
:1086C0008823D1F30E94F44B182F8823A9F3E98D56
:1086D000FA8DCC80DD80EE80FF8032E0C31AD108B5
:1086E000E108F108058404C0CC0CDD1CEE1CFF1C65
:1086F0000A94D2F786859785A089B189C80ED91EBC
:10870000EA1EFB1E81E08093D80BC092DB0DD09255
:10871000DC0DE092DD0DF092DE0D80E092E0EBEDFD
:10872000FBE0DF019C011D9221503040E1F701E0A8
:10873000E98DFA8D8481081788F42BED3BE0B701B1
:10874000A601400F511D611D711D8091D90B9091A3
:10875000DA0B39DF8823E1F00F5FEACFC12C82E02A
:10876000D82EE12CF12C058404C0CC0CDD1CEE1CB1
:10877000FF1C0A94D2F749895A896B897C894C0D70
:108780005D1D6E1D7F1D498B5A8B6B8B7C8B812FE2
:10879000DF91CF911F910F91FF90EF90DF90CF90DD
:1087A0000895CF93DF93EC0141E0611101C040E0F7
:1087B0006C857D858E859F850E94344C882341F091
:1087C000888920E2829FC00111248552944F02C003
:1087D00080E090E0DF91CF91089530E020E04EE21C
:1087E000DC015C91503271F0383029F4FB01E20F6A
:1087F000F11D40832F5FFB01E20FF11DDC015C9155
:1088000050832F5F3F5F01963B3051F7FB01E20F32
:10881000F11D10820895CF93DF93EB01FC012381BA
:10882000211102C080E00EC02250223020F48FE2DD
:108830008883198206C060E0B4DF009799F3BE0117
:10884000CCDF81E0DF91CF910895FB012BE030E296
:1088500031932150E9F7DC0190E027E03A2FEB2F2C
:108860008D9181110AC0DA013C931196EC9381E05D
:10887000FB019081903239F525C08F32A1F38E3201
:1088800019F0EEEBF6E008C02A30E1F098E02AE0BB
:10889000E5CF31963817B1F034913111FACF29175D
:1088A00088F03FED380F3E3568F431E0390FFB01B9
:1088B000E90FF11D9FE9980F9A3108F480528083E7
:1088C000932FCCCF80E008950F931F93CF93DF9326
:1088D000EC018B018B81882311F080E042C0FB0109
:1088E0008789803139F18032C1F783E08B83F801C9
:1088F000428D538D648D758D4D8B5E8B6F8B788F14
:108900009E012F5E3F4FC8010E94EB4C882329F344
:108910001A8F098F81E089831C821D821E821F822B
:10892000188619861A861B861C861D861E861F863B
:10893000188A17C082E08B831D8A1E8A1F8A188EB0
:10894000FB01408D518D60E070E095E0440F551FB4
:10895000661F771F9A95D1F7498B5A8B6B8B7C8B4F
:10896000D7CFDF91CF911F910F9108952F923F9212
:108970004F925F926F927F928F929F92AF92BF922F
:10898000CF92DF92EF92FF920F931F93CF93DF93DB
:10899000EC015B016A018B81811103C08FEF9FEFB6
:1089A000C6C0898180FFFACF49895A896B897C8941
:1089B00088859985AA85BB852601612C712C8A0141
:1089C0009B01081B190B2A0B3B0B40165106620634
:1089D000730618F06A01C81AD90A76013E0124E02C
:1089E000620E711CE114F10409F476C048855985C2
:1089F0006A857B854A0181E098222B811A012B012F
:108A0000E9E05694479437942794EA95D1F7898DF5
:108A10009A8DFC01223049F4628D738D848D958D81
:108A2000620D731D841D951D3CC0148111501221CF
:108A300081149104C1F4111116C0452B462B472B0C
:108A400049F48D899E89AF89B88D8C839D83AE83CF
:108A5000BF8309C04C815D816E817F8193013CD7CA
:108A6000882309F49BCFE98DFA8D6C817D818E81FD
:108A70009F816250710981099109058404C0660FC4
:108A8000771F881F991F0A94D2F72685378540895A
:108A90005189620F731F841F951F610F711D811D06
:108AA000911D20E032E02819390987012E153F0574
:108AB00008F489010115F2E01F0761F52091DB0D33
:108AC0003091DC0D4091DD0D5091DE0D6217730782
:108AD0008407950719F41EC0C60129C09501AB0192
:108AE000BC018091D90B9091DA0B14DD882309F435
:108AF00055CFA00EB11E88859985AA85BB85800FAC
:108B0000911FA11DB11D88879987AA87BB87E01A8D
:108B1000F10A68CF40E0A8D6882309F43FCFB4011A
:108B20006552744FA801C5010E940AD4E2CFDF91BB
:108B3000CF911F910F91FF90EF90DF90CF90BF905A
:108B4000AF909F908F907F906F905F904F903F90ED
:108B50002F900895CF93DF931F92CDB7DEB741E0FA
:108B600050E0BE016F5F7F4F01DF019719F48981EB
:108B700090E002C08FEF9FEF0F90DF91CF910895AB
:108B8000CF92DF92EF92FF920F931F93CF93DF93D9
:108B90006C01EB017A01FC018381823060F0008579
:108BA0001185228533850F71112722273327012B49
:108BB000022B032B11F08FEF5CC04115510511F012
:108BC000F70110821DE040E250E0BE01C601CEDE9A
:108BD0008032910539F021E0892B09F420E0822FC1
:108BE000819547C028812223C1F0253E61F32E32B2
:108BF00051F33B853F733F3061F4E114F10449F0D8
:108C00004A8D5B8D452B29F42F713FEF320F3230A7
:108C100030F02B8523FDD7CF2CC080E02AC030E078
:108C200021503109129FC001139F900D1124F701AB
:108C3000E80FF91F298120832B8121832D81228335
:108C40002F812383298524832E85258328892683C4
:108C50002A8927832C8920872E892187288D22879E
:108C60002C8D23872E8D2487288126FFD2CF158631
:108C7000D0CFDF91CF911F910F91FF90EF90DF90B8
:108C8000CF9008951F93CF93DF93EC018B818230B7
:108C900018F480E090E023C0488559856A857B857B
:108CA000A5E07695679557954795AA95D1F7142F26
:108CB0001F70CE014FDF97FDECCF488559856A853F
:108CC0007B85415E5F4F6F4F7F4F488759876A872B
:108CD0007B8720E2129FC00111248552944FDF91BF
:108CE000CF911F9108954F925F926F927F92AF92B2
:108CF000BF92CF92DF92EF92FF920F931F93CF9389
:108D0000DF93EC016A017B012B81222349F08989E1
:108D10009A89AB89BC8984179507A607B70710F411
:108D200080E06BC0223009F463C0C114D104E104B7
:108D3000F10449F41C821D821E821F821886198646
:108D40001A861B8659C088859985AA85BB85E98DB9
:108D5000FA8DE585F0E03996AC01BD01415051092D
:108D6000610971090E2E04C0769567955795479550
:108D70000A94D2F79701860101501109210931099E
:108D800004C03695279517950795EA95D2F70417ED
:108D900015072607370720F0892B8A2B8B2B49F4E0
:108DA0008D899E89AF89B88D8C839D83AE83BF8367
:108DB00004C0041B150B260B370B280139015E017B
:108DC00084E0A80EB11C411451046104710481F0C7
:108DD0004C815D816E817F819501898D9A8D7CD5D5
:108DE00091E0491A5108610871088111ECCF05C062
:108DF000C886D986EA86FB8681E0DF91CF911F91F4
:108E00000F91FF90EF90DF90CF90BF90AF907F9049
:108E10006F905F904F9008950F931F93CF93DF93C0
:108E2000EC018B818823D1F1898187FF32C061E019
:108E3000CE01B7DC8C01009789F1FC018081853E71
:108E400069F18B81823040F449895A896B897C8928
:108E5000448F558F668F778F4D895E896F89788DA6
:108E6000F801538F428F758B648BE091D20BF09198
:108E7000D30B309759F0B8016A5E7F4FC80148960E
:108E80001995F801808D918D938B828B89818F77D5
:108E90008983DF91CF911F910F91A6C481E08883D0
:108EA00080E0DF91CF911F910F910895CF93DF93D1
:108EB000EC01B2DF1B82DF91CF910895FC01238189
:108EC0002111F4CF08954F925F926F927F92AF92EB
:108ED000BF92CF92DF92EF92FF920F931F93CF93A7
:108EE000DF9300D01F92CDB7DEB75C016A017B0132
:108EF000FC0183818130E9F4818181FF1AC0F50191
:108F000081899289A389B48984179507A607B70731
:108F100080F0892B8A2B8B2B09F472C0F5014084D9
:108F2000518462847384B701A601C501DCDE81111E
:108F300002C080E066C0F501818D928DC114D1041C
:108F4000E104F10469F4458956896789708D41D738
:108F5000882379F3F501158A168A178A108E37C08F
:108F6000F50144815581668177819E012F5F3F4FD6
:108F7000B3D48823F1F249815A816B817C81F50158
:108F8000818D928DFC012789203139F4483FFFEF14
:108F90005F0761057105D8F407C0483F2FEF5207FE
:108FA00062072FE0720798F414D7882309F4C1CF21
:108FB000F50144815581668177810FEF1FEF2FEF17
:108FC0003FE0818D928D6DD5882309F4B2CFF501F4
:108FD000C18AD28AE38AF48A818180688183C5014B
:108FE0001BDF882309F4A5CFB701A6014C145D044B
:108FF0006E047F0410F4B301A201C50174DE01C048
:1090000081E00F900F900F900F90DF91CF911F9103
:109010000F91FF90EF90DF90CF90BF90AF907F9037
:109020006F905F904F900895FF920F931F93CF938F
:10903000DF93EC01F42E80E2689FF0011124E552E9
:10904000F44F8385817121F0842F827109F04EC025
:109050008091DB0D9091DC0DA091DD0DB091DE0DC6
:109060008C879D87AE87BF87688B4489558960E070
:1090700070E0BA0155274427028D138D20E030E0BF
:10908000402B512B622B732B4D8B5E8B6F8B788F0C
:109090008385887151F4048D158D268D378D098B4C
:1090A0001A8B2B8B3C8B81E00BC08031F9F49E0135
:1090B0002F5E3F4F898D9A8D8ED48823B9F084E03E
:1090C0008B838F2D8F7089831C821D821E821F824D
:1090D000188619861A861B86F4FE0BC040E050E005
:1090E000BA01CE01F0DE811104C011C01B8280E004
:1090F0000EC0F5FE0BC049895A896B897C89CE0167
:10910000DF91CF911F910F91FF90EDCD81E0DF9125
:10911000CF911F910F91FF900895AF92BF92CF9280
:10912000DF92EF92FF920F931F93CF93DF937C0117
:10913000EB016A01B22E898D9A8DF701928F818F92
:1091400040E050E0BA01CE01CEDDA12C08851985A2
:109150002A853B8589899A89AB89BC8908171907B3
:109160002A073B07A0F585E03695279517950795C3
:109170008A95D1F70F70CE0185DD009709F481C083
:10918000FC012081222311F0253EB9F4A1100EC06C
:109190004091DB0D5091DC0D6091DD0D7091DE0D85
:1091A000F7014487558766877787008BFC018081AC
:1091B000AA24A3948111CACF0AC04BE050E0BC019D
:1091C000C6010E94FDD3892B09F0C0CF58C08B2D5A
:1091D0008274823409F055C0AA2049F0F701008951
:1091E00061E0C701DEDAEC01009769F44AC08B81C7
:1091F000823009F446C0CE014DDA882309F441C01B
:10920000CBEDDBE000E080E2FE0111928A95E9F708
:109210008BE0F601DE0101900D928A95E1F7E09175
:10922000D20BF091D30B309739F0BE01625F7F4FC4
:10923000CE014096199508C081E298E2998B888BFF
:1092400080E098E09F878E87888999899B8B8A8B9D
:10925000998F888F8E859F859F8B8E8BC5D2882313
:1092600081F04B2D602FC701DF91CF911F910F919E
:10927000FF90EF90DF90CF90BF90AF90D5CEB7FE2C
:10928000F0CF80E0DF91CF911F910F91FF90EF9091
:10929000DF90CF90BF90AF9008953F924F925F9232
:1092A0006F927F928F929F92AF92BF92CF92DF92F6
:1092B000EF92FF920F931F93CF93DF93CDB7DEB75B
:1092C000C354D1090FB6F894DEBF0FBECDBF5C0109
:1092D0006B0124965FAF4EAF2497522E1C8E1F8ECB
:1092E00019821C826115710511F410E073C0FC0134
:1092F00083818111FACF2496EEADFFAD2497808152
:109300008F3211F076011DC02496EEADFFAD24978B
:1093100080818F3231F431962496FFAFEEAF2497DF
:10932000F3CFF60183818250823060F3F601618DC4
:10933000728DCE010196C8DA8823B9F2CE0101966A
:109340007C018E01045E1F4F3801FE0131964F01F2
:10935000402E312E19C08823A9F121E0AE01495CCD
:109360005F4FB701C801D9DE882309F4BECFEC14E2
:10937000FD0411F0C7019ADD0615170501F1942DC2
:10938000832D7801092F182FAE014E5B5F4FBE0170
:10939000695C7F4F24968EAD9FAD249756DA882363
:1093A00009F4A3CF2496EEADFFAD249780818F32D0
:1093B00091F631962496FFAFEEAF2497F3CF982D18
:1093C000892DDFCF252DAE01495C5F4FB701C50167
:1093D000A4DE182FCE01019671DDCE014C966EDD14
:1093E000812FCD5BDF4F0FB6F894DEBF0FBECDBF30
:1093F000DF91CF911F910F91FF90EF90DF90CF9071
:10940000BF90AF909F908F907F906F905F904F90A4
:109410003F900895CF93DF93EC0140E050E0BA0114
:1094200052DD882361F061E0CE01BBD9009739F0AD
:1094300025EEFC0120831B82DF91CF91D5C180E016
:10944000DF91CF9108951F93CF93DF93CDB7DEB710
:109450006B970FB6F894DEBF0FBECDBFAB0119827C
:109460001C8222E0BC01CE01019617DF182F882351
:1094700021F0CE010196CEDF182FCE0101961EDD20
:10948000812F6B960FB6F894DEBF0FBECDBFDF9174
:10949000CF911F9108952F923F924F925F926F92BA
:1094A0007F928F929F92AF92BF92CF92DF92EF9274
:1094B000FF920F931F93CF93DF9300D01F921F92C1
:1094C000CDB7DEB78C015B013A01DC0113968C91BC
:1094D00013978130C1F411968C9181FF14C082FFE3
:1094E00018C0F80141895289638974898085918502
:1094F000A285B38584179507A607B70751F0C80161
:10950000F2DB811106C081E0F80180838FEF9FEFCD
:1095100037C1630183C0D80159968D919C915A97A8
:10952000FC01F481F1501A012B0169E05694479433
:10953000379427946A95D1F7F221FD834A0121E0FF
:109540009222FF2309F476C080E092E088199909FD
:1095500076018C159D0508F47C01D8015996ED9192
:10956000FC915A9714962D903D904D905C901797D2
:10957000B2E02B1A310841085108058404C0220CBE
:10958000331C441C551C0A94D2F786859785A08904
:10959000B189280E391E4A1E5B1EED812E0E311C2C
:1095A000411C511CE114F2E0FF0609F089C08091D2
:1095B000DB0D9091DC0DA091DD0DB091DE0D8215DB
:1095C0009305A405B50569F41092D80B8FEF9FEFB2
:1095D000DC018093DB0D9093DC0DA093DD0DB09347
:1095E000DE0D9501B201A1018091D90B9091DA0BAA
:1095F0000E94E342882309F486CFF8018085918593
:10960000A285B3858E0D9F1DA11DB11D80879187F9
:10961000A287B387AE0CBF1CCE18DF08D8011896FE
:109620004D915D916D917C911B97C114D10409F00E
:1096300072CF7AC08114910409F086CF14964D91AF
:109640005D916D917C9117974115510561057105EB
:1096500059F455968D919D910D90BC91A02D009738
:10966000A105B10539F520C09E012F5F3F4F34D1D0
:10967000882309F448CF89819A81AB81BC81F801A4
:10968000218D328DF9012789203139F4883FFFEF90
:109690009F07A105B10540F40DC0883F2FEF920749
:1096A000A2072FE0B20730F0C8010E9424438111C5
:1096B0004BCF29CFF80184839583A683B78344CF0A
:1096C0008114910411F5D80118964D915D916D9119
:1096D0007C911B9751968D919D910D90BC91A02DE1
:1096E000481759076A077B0780F07ED0882309F462
:1096F0000ACF81E08093D80B2092DB0D3092DC0DF5
:109700004092DD0D5092DE0D07C041E0C201B10173
:10971000ABD0882309F4F7CEA701B501C401855267
:10972000944F0E940AD469CF51968D919D910D90CE
:10973000BC91A02DF801218184179507A607B707D2
:1097400038F4418B528B638B748B206821830CC05F
:109750008091D20B9091D30B892B31F0611471045D
:1097600019F02068F8012183D80111968C9183FDAE
:1097700002C0C30105C0C8014FDB8111FACFC3CEBF
:109780000F900F900F900F900F90DF91CF911F913E
:109790000F91FF90EF90DF90CF90BF90AF909F9090
:1097A0008F907F906F905F904F903F902F90089593
:1097B000CF93DF931F92CDB7DEB7698341E050E0CE
:1097C000BE016F5F7F4F049666DE0F90DF91CF91F1
:1097D0000895FB0101900020E9F7AF0141505109C4
:1097E000461B570B049657CECF938091D80B8823F6
:1097F000B9F14091DB0D5091DC0D6091DD0D709160
:10980000DE0D2BED3BE08091D90B9091DA0B0E949D
:10981000E342C82F811102C0C0E023C04091D40BA5
:109820005091D50B6091D60B7091D70B4115510516
:109830006105710591F02BED3BE08091D90B909182
:10984000DA0B0E94E342882339F31092D40B109272
:10985000D50B1092D60B1092D70B1092D80B01C0DB
:10986000C1E08C2FCF910895CF92DF92EF92FF92BB
:10987000CF936B017C01C42F8091DB0D9091DC0DA7
:10988000A091DD0DB091DE0D8C159D05AE05BF05D7
:10989000C9F0AADF811102C080E018C02BED3BE0C7
:1098A000B701A6018091D90B9091DA0B0E948A42F0
:1098B000882391F3C092DB0DD092DC0DE092DD0D98
:1098C000F092DE0D81E0C1118093D80BCF91FF9013
:1098D000EF90DF90CF9008958F929F92AF92BF92BA
:1098E000CF92DF92EF92FF920F931F93CF93DF936C
:1098F000EC016A017B01890189859A85AB85BC856C
:109900000196A11DB11D84179507A607B70710F48E
:1099100080E054C08F89803129F49927872F762FD2
:10992000652F0BC08032A1F7CB01BA0127E09695D5
:109930008795779567952A95D1F78B889C88AD8810
:10994000BE88680D791D8A1D9B1D8090DB0D90904F
:10995000DC0DA090DD0DB090DE0D681579058A054F
:109960009B0581F48F89803191F4DD24EE24FF245E
:10997000F601EE0FFF1FE552F44F80819181A0E0C8
:10998000B0E016C040E070DF8111ECCFC1CFE894A9
:10999000C7F8DD24EE24FF24F601EE0FFF1FEE0FC3
:1099A000FF1FE552F44F80819181A281B381BF7086
:1099B000F80180839183A283B38381E0DF91CF910B
:1099C0001F910F91FF90EF90DF90CF90BF90AF90DD
:1099D0009F908F9008954F925F926F927F92AF9277
:1099E000BF92CF92DF92EF92FF920F931F93CF938C
:1099F000DF9300D01F92CDB7DEB78C0149835A8325
:109A00006B837C835901C12CD12C7601412C42E01F
:109A1000542E612C712C49815A816B817C819E016D
:109A20002F5F3F4FC80158DF882341F1D301C201A6
:109A3000F801058404C0880F991FAA1FBB1F0A9450
:109A4000D2F7C80ED91EEA1EFB1E49815A816B81CE
:109A50007C818789803139F481E0483F5F4F61051F
:109A6000710538F4D8CF81E0483F5F4F6F4F7F409A
:109A700090F2F501C082D182E282F3820F900F90C2
:109A80000F900F90DF91CF911F910F91FF90EF906A
:109A9000DF90CF90BF90AF907F906F905F904F908E
:109AA00008954F925F926F927F928F929F92AF92A2
:109AB000BF92CF92DF92EF92FF920F931F93CF93BB
:109AC000DF93EC014A015B01280139014230510565
:109AD0006105710508F462C049855A856B857C85EE
:109AE0004F5F5F4F6F4F7F4F481559056A057B05E4
:109AF00008F454C08F89803129F4FF24EB2CDA2C30
:109B0000C92C0CC0803209F049C07501640177E0AE
:109B1000F694E794D794C7947A95D1F74B895C89EA
:109B20006D897E89C40ED51EE61EF71E41E0C70171
:109B3000B6019ADE882391F19F89903159F49924D6
:109B4000AA24BB24F401EE0FFF1FE552F44F51820B
:109B5000408210C0E89487F89924AA24BB24F40119
:109B6000EE0FFF1FEE0FFF1FE552F44F40825182B0
:109B7000628273829A89923090F04D815E816F810A
:109B800078854C0D5D1D6E1D7F1D4093D40B509349
:109B9000D50B6093D60B7093D70B01C080E0DF919B
:109BA000CF911F910F91FF90EF90DF90CF90BF90DA
:109BB000AF909F908F907F906F905F904F9008959F
:109BC0002F923F924F925F926F927F928F929F92CD
:109BD000AF92BF92CF92DF92EF92FF920F931F93BB
:109BE000CF93DF93CDB7DEB72F970FB6F894DEBFD4
:109BF0000FBECDBF1C014C875D876E877F873B877B
:109C00002A87DC0119960D911D912D913C911C978D
:109C10000F5F1F4F2F4F3F4F0D831E832F833887BA
:109C2000EA85FB8580809180A280B38081149104B5
:109C3000A104B10431F0FFEF8F1A9F0AAF0ABF0AE7
:109C400010C0DC018D909D90AD90BC90B1E0B987C3
:109C50000C851D852E853F850130110521053105B7
:109C600009F0198675016401412C512C3201F10172
:109C700081859285A385B485481659066A067B06B8
:109C800008F04EC00D811E812F8138850C151D05F1
:109C90002E053F0550F4F2E0CF2ED12CE12CF12C13
:109CA000A2E08A2E912CA12CB12C9E012F5F3F4F58
:109CB000B701A601C10110DE882391F149815A81C3
:109CC0006B817C81D701C6010196A11DB11D452B79
:109CD000462B472B19F04C015D010FC0AC01BD01B3
:109CE000481959096A097B090C851D852E853F8510
:109CF000401751076207730741F01FEF411A510ADD
:109D0000610A710A6C017D01B2CF0FEF1FEF2FEFD7
:109D10003FE0B701A601C101C4DE8D83811113C0EC
:109D20001D823DC02601370121E0421A5108610819
:109D3000710897018601B301A201C101B2DE882337
:109D400079F3730162018C149D04AE04BF0450F3D7
:109D5000AA85BB854D915D916D917C914115510511
:109D600061057105A9F4EA85FB8580829182A28252
:109D7000B382F985FF2399F00FEF801A900AA00AA9
:109D8000B00AD1018D929D92AD92BC92139707C0FB
:109D900095018401C10185DE8111E5CFC1CF8D819F
:109DA0002F960FB6F894DEBF0FBECDBFDF91CF91D7
:109DB0001F910F91FF90EF90DF90CF90BF90AF90E9
:109DC0009F908F907F906F905F904F903F902F90DB
:109DD0000895AF92BF92CF92DF92EF92FF920F93CE
:109DE0001F93CF93DF9300D01F92CDB7DEB75C01F6
:109DF0006A017B0182E090E0A0E0B0E0F5018083A1
:109E00009183A283B3839E012F5F3F4FB701A601C9
:109E1000C50162DD811102C080E023C000E010E0D6
:109E20009801B701A601C5013CDE8823A9F3C980CA
:109E3000DA80EB80FC80F5018789803149F481E08C
:109E4000F8EFCF16FFEFDF06E104F10450F4DBCFAB
:109E500081E098EFC9169FEFD906E9069FE0F90661
:109E600090F20F900F900F900F90DF91CF911F9174
:109E70000F91FF90EF90DF90CF90BF90AF9008953B
:109E80007F928F929F92AF92BF92CF92DF92EF928A
:109E9000FF920F931F93CF93DF93EC01142F7093D6
:109EA000DA0B6093D90B1F8A82E090E0A0E0B0E06B
:109EB00088839983AA83BB831092D80B1092D40B0A
:109EC0001092D50B1092D60B1092D70B8FEF9FEFFD
:109ED000DC018093DB0D9093DC0DA093DD0DB0933E
:109EE000DE0D442349F1453008F0DEC040E060E07B
:109EF00070E0CB01B9DC882309F4D6C020E1129FC1
:109F0000F0011124E757F24F80818F7709F0CCC020
:109F100084859585A685B78584369105A105B1050B
:109F200008F4C2C0C084D184E284F384C114D10493
:109F3000E104F10421F4B8C0C12CD12C760140E039
:109F4000C701B60191DC782E882309F4ADC0809159
:109F5000E60B9091E70B8115924009F0A5C0309176
:109F6000EB0B332309F4A0C08091E90B9091EA0B2D
:109F7000892B09F499C02091E80B222309F494C09D
:109F80003A8B2C831D8630E041E050E06D85062F32
:109F9000CA01062E02C0880F991F0A94E2F72817FB
:109FA000390731F081E0860F8D87683078F37CC007
:109FB0002091F10B3091F20B2115310519F040E0A1
:109FC00050E008C02091FF0B3091000C4091010C33
:109FD0005091020C2D833E834F8358878091E90B6B
:109FE0009091EA0B46015701880E991EA11CB11CE5
:109FF0008B8A9C8AAD8ABE8AE091EC0BF091ED0BC6
:10A00000F98FE88FA091EB0BB0E00E94E9D0680DCA
:10A01000791D8A1D9B1D6A8F7B8F8C8F9D8FB5E06C
:10A02000EE0FFF1FBA95E1F7E150FE4FEF2FFF272C
:10A03000E695DC01CB018E0F9F1FA11DB11D8E8700
:10A040009F87A88BB98B8090EE0B9090EF0B8114BB
:10A05000910419F0A12CB12C08C08090FB0B9090BA
:10A06000FC0BA090FD0BB090FE0BA7019601281BE6
:10A07000390B4A0B5B0BDA01C901880D991DAA1D2A
:10A08000BB1D04C0B695A795979587950A95D2F7FD
:10A0900089879A87AB87BC87853F3FE09307A105F7
:10A0A000B10520F48CE08F8B712C15C0853F9F4F3C
:10A0B000A105B10510F480E10DC08091070C9091CD
:10A0C000080CA091090CB0910A0C8A8F9B8FAC8F61
:10A0D000BD8F80E28F8B872DDF91CF911F910F91E4
:10A0E000FF90EF90DF90CF90BF90AF909F908F90B8
:10A0F0007F900895FC01148217821382128284E4F7
:10A1000094E09183808308950F931F93CF93DF93FF
:10A11000EC018F96EFDFCE01805B9F4FEBDFCE012E
:10A1200081599F4FE7DFCE0182579F4FE3DFFE014A
:10A13000E355FF4F89E1818314823596178ACE015A
:10A1400080539F4FD7DFFE01E151FF4F10821182F4
:10A1500012821382389610821182128213821A821E
:10A160001B82188219828E010D501F4FF801108238
:10A17000118212821382389681E080831EA61DA66A
:10A180000E94C4C568577C4E8F4F9F4FF801608373
:10A19000718382839383DF91CF911F910F910895F3
:10A1A000FC0120E03EE2DB014C91403241F02830DE
:10A1B00011F430833196DB014C91408331962F5F4F
:10A1C0006F5F7F4F2B3079F7108208953F924F9247
:10A1D0005F926F927F928F929F92AF92BF92CF9237
:10A1E000DF92EF92FF920F931F93CF93DF93CDB740
:10A1F000DEB7C758D1090FB6F894DEBF0FBECDBF8A
:10A200008C016B017A01312C84E0E80EF11C2801ED
:10A21000E1E14E0E511C5801FCEFAF0EB11C48019C
:10A220008EEF880E911C80E4682E712C6C0E7D1EC2
:10A23000E4E06E0E711CA201BE016F5F7F4FC7018B
:10A240000E94C04518160CF02BC12C85322F387196
:10A25000303109F09EC0F50180819181019702970C
:10A2600008F497C0BE016F5F7F4FCE0187589F4FA4
:10A2700097DFA0961FAEA097F6018081811107C0DD
:10A2800068E474E0CE01815A9F4F0E9413D4B60156
:10A29000CE01815A9F4F0E9413D4BE0167587F4F51
:10A2A000CE01815A9F4F0E9413D468E474E0CE011E
:10A2B000815A9F4F0E9413D4CE01805C9F4F1ADFBA
:10A2C00021E0AE0147585F4FB701C3010E944D49DD
:10A2D000811139C0F50180819181892BA1F5EDE2D1
:10A2E000F8E08491882341F09091C00095FFFCCF65
:10A2F0008093C6003196F5CFEAE4F4E0819188239B
:10A3000039F09091C00095FFFCCF8093C600F6CF46
:10A310008091C00085FFFCCF8AE08093C600FE01DB
:10A32000E758FF4F8191882339F09091C00095FF45
:10A33000FCCF8093C600F6CF8091C00085FFFCCF94
:10A340008AE08093C6008BE1FE01EC5BFF4FDE01EB
:10A35000959601900D928A95E1F724968EAD9FAD6A
:10A3600024979CA38BA384E494E09AA389A3AE01D1
:10A370004F5D5F4FBE01615A7F4FC80127DFCE019D
:10A3800081960E94CC40CE01805C9F4F0E94CC40C1
:10A3900052CF8981882309F483C0853E09F44BCFCD
:10A3A0008E3209F448CF8F3509F445CFF801818901
:10A3B000882331F08E3209F43ECF8F3509F43BCF3C
:10A3C00023FD39CF81E0303109F080E0F80184A726
:10A3D000811110C09091AC0989859E3021F48E3492
:10A3E00009F029CF03C0873409F025CF8A858E373D
:10A3F00009F421CF98012C5F3F4FBE016F5F7F4F63
:10A40000C901CA57DF4F2883C658D040C957DF4F0C
:10A410003883C758D040C4DEF50180819181CA5786
:10A42000DF4F2881C658D040C957DF4F3881C75801
:10A43000D0400097F1F4F6018191882339F0909192
:10A44000C00095FFFCCF8093C600F6CFF901819143
:10A45000882339F09091C00095FFFCCF8093C6000F
:10A46000F6CF8091C00085FFFCCF8AE08093C600C4
:10A47000E2CE8130910539F4F40180819181019619
:10A4800091838083D8CE029709F0D5CE232D30E07A
:10A49000F401808191812817390711F03394CBCED4
:10A4A000C957DF4F0FB6F894DEBF0FBECDBFDF91A7
:10A4B000CF911F910F91FF90EF90DF90CF90BF90C1
:10A4C000AF909F908F907F906F905F904F903F9054
:10A4D0000895EF92FF920F931F93CF93DF93CDB721
:10A4E000DEB76F970FB6F894DEBF0FBECDBF8C01FD
:10A4F000FC01E450FF4F118210827C0183E3E80EDF
:10A50000F11C40E050E0BA01C7010E9473468BE1A4
:10A51000F701DE01159601900D928A95E1F7F80199
:10A5200081A992A99C838B8384E494E09A83898394
:10A53000AE014F5F5F4F61E375E0C80147DECE01BA
:10A5400001960E94CC406F960FB6F894DEBF0FBE06
:10A55000CDBFDF91CF911F910F91FF90EF900895A4
:10A560002BE1FB013496DC01149601900D922A95A3
:10A57000E1F7FB0122813381FC01338322830895BB
:10A58000EF92FF920F931F93CF93DF93EC011B8207
:10A590008EA9882321F0CE01C3960E9456477E01E2
:10A5A0008DEAE80EF11C45E360E0C7010E94D74147
:10A5B00081111FC0EDE2F8E08491882341F0909171
:10A5C000C00095FFFCCF8093C6003196F5CFE0E246
:10A5D000F8E08491882341F09091C00095FFFCCF72
:10A5E0008093C6003196F5CF8091C00085FFFCCFE7
:10A5F00074C08E010E541F4F41E0B701C80140DC0A
:10A60000811125C040E0B701C8013ADC81111FC0AB
:10A61000E3E3F8E08491882341F09091C00095FF36
:10A62000FCCF8093C6003196F5CFEDE0F8E0849141
:10A63000882341F09091C00095FFFCCF8093C60025
:10A640003196F5CF8091C00085FFFCCF46C0B801A0
:10A65000CE01C3960E94644481111FC0E3E3F8E079
:10A660008491882341F09091C00095FFFCCF8093A6
:10A67000C6003196F5CFEDEFF7E08491882341F0E5
:10A680009091C00095FFFCCF8093C6003196F5CF26
:10A690008091C00085FFFCCF20C081E08B83EDE27C
:10A6A000F8E08491882341F09091C00095FFFCCFA1
:10A6B0008093C6003196F5CFE2EFF7E084918823CE
:10A6C00041F09091C00095FFFCCF8093C600319679
:10A6D000F5CF8091C00085FFFCCF8AE08093C60053
:10A6E0008E01015D1F4FB801CE01805B9F4F38DFA7
:10A6F000C25BDF4F19830883DF91CF911F910F91C8
:10A70000FF90EF900895FC01128213820895FC01DE
:10A710002381222311F021E022830895FC0122816C
:10A720002111128208952F923F924F925F926F9261
:10A730007F928F929F92AF92BF92CF92DF92EF92D1
:10A74000FF920F931F93CF93DF93CDB7DEB7AD97F3
:10A750000FB6F894DEBF0FBECDBF7C016B014DA7D5
:10A76000FC018381811115C0EEEDF7E0849188230F
:10A7700041F09091C00095FFFCCF8093C6003196C8
:10A78000F5CF8091C00085FFFCCF8AE08093C600A2
:10A79000A8C14701F4ED8F0E911CC4010E945647D9
:10A7A000F7011282CE0101965C01A4DC17019EE440
:10A7B000290E311CC7018F96F10191838083F60128
:10A7C00080818F3209F07FC06FE270E0C6010E9485
:10A7D0001ED48C010F5F1F4F09F47BC06FE270E045
:10A7E000C8010E941ED42C01009709F473C00817F9
:10A7F000190708F06FC03C01601A710AA301B80183
:10A80000CE0180960E9447D4E0E2F0E0EC0FFD1FFD
:10A81000E60DF71D1082FE01B0968191882339F074
:10A820009091C00095FFFCCF8093C600F6CF809139
:10A83000C00085FFFCCFFAE0F093C600F101608113
:10A8400071816115710519F06C5F7F4F02C060E086
:10A8500070E021E0AE01405E5F4FCE0105960E94A0
:10A860004D4981112BC0EAECF7E08491882341F037
:10A870009091C00095FFFCCF8093C6003196F5CF34
:10A88000FE01B0968191882339F09091C00095FF28
:10A89000FCCF8093C600F6CFE8ECF7E084918823E4
:10A8A00041F09091C00095FFFCCF8093C600319697
:10A8B000F5CF8091C00085FFFCCFE7C0F101B182E8
:10A8C000A082820187CFC701805B9F4FF1019183F6
:10A8D00080838601FDA5FF2309F49CC0F1016081FE
:10A8E00071816115710519F06C5F7F4F02C060E0E6
:10A8F00070E021E0A801C4010E944D49882309F4B9
:10A900005FC0F40181899289A389B489F701E1517B
:10A91000FF4F80839183A283B383EAEBF7E08491B6
:10A92000D701A151BF4F882349F09091C00095FFF6
:10A93000FCCF8093C60031968491F5CFF8018191C8
:10A94000882339F09091C00095FFFCCF8093C6001A
:10A95000F6CFE2EBF7E08491882341F09091C000BC
:10A9600095FFFCCF8093C6003196F5CF4D915D9158
:10A970006D917C912AE030E082EE95E00E941418FF
:10A980008091C00085FFFCCF8AE08093C600F7016C
:10A99000E950FF4F1082118212821382E4EAF7E03D
:10A9A0008491882341F09091C00095FFFCCF809363
:10A9B000C6003196F5CF8091C00085FFFCCF88C0DE
:10A9C000E0E9F7E08491882341F09091C00095FF81
:10A9D000FCCF8093C6003196F5CFF8018191882392
:10A9E00039F09091C00095FFFCCF8093C600F6CF60
:10A9F000EEE8F7E08491882341F09091C00095FF44
:10AA0000FCCF8093C6003196F5CF8091C00085FFC2
:10AA1000FCCF3BC0F101608171816115710519F0B6
:10AA20006C5F7F4F02C060E070E026E5A801C401C2
:10AA30000E944D4981112DC0EAE7F7E084918823F7
:10AA400041F09091C00095FFFCCF8093C6003196F5
:10AA5000F5CFF8018191882339F09091C00095FFDE
:10AA6000FCCF8093C600F6CFE8E7F7E08491882317
:10AA700041F09091C00095FFFCCF8093C6003196C5
:10AA8000F5CF8091C00085FFFCCF8AE08093C6009F
:10AA900025C081E0F7018083E6E6F7E08491882312
:10AAA00041F09091C00095FFFCCF8093C600319695
:10AAB000F5CFF6018191882339F09091C00095FF80
:10AAC000FCCF8093C600F6CF8091C00085FFFCCFFD
:10AAD0008AE08093C600C8010E949F92C5010E942F
:10AAE000CC40AD960FB6F894DEBF0FBECDBFDF9160
:10AAF000CF911F910F91FF90EF90DF90CF90BF907B
:10AB0000AF909F908F907F906F905F904F903F900D
:10AB10002F90089521E0FC01218340E004CE3F9274
:10AB20004F925F926F927F928F929F92AF92BF925D
:10AB3000CF92DF92EF92FF920F931F93CF93DF9309
:10AB4000CDB7DEB7AC970FB6F894DEBF0FBECDBF62
:10AB50007C015B01FC018381882309F401C1C701E9
:10AB60008C529F4F0E945647F7011282CE010196E8
:10AB70006C01C0DA27019EE4490E511CC7018F9673
:10AB8000F20191838083F50180818F3209F084C0C6
:10AB90006FE270E0C5010E941ED48C010F5F1F4F51
:10ABA0009AE0392E0115110509F47CC06FE270E0BE
:10ABB000C8010E941ED44C01009709F474C0081704
:10ABC000190708F070C03C01601A710AA301B801AE
:10ABD000CE0180960E9447D4E0E2F0E0EC0FFD1F2A
:10ABE000E60DF71D1082FE01B0968191882339F0A1
:10ABF0009091C00095FFFCCF8093C600F6CF809166
:10AC0000C00085FFFCCF3092C600F20160817181E7
:10AC10006115710519F06C5F7F4F02C060E070E054
:10AC200021E0AE01405E5F4FCE0105960E944D4986
:10AC300081112BC0E2E5F7E08491882341F09091E7
:10AC4000C00095FFFCCF8093C6003196F5CFFE0182
:10AC5000B0968191882339F09091C00095FFFCCF88
:10AC60008093C600F6CFE0E5F7E08491882341F0B9
:10AC70009091C00095FFFCCF8093C6003196F5CF30
:10AC80008091C00085FFFCCF65C0F201D182C082F7
:10AC900084010F5F1F4F86CFC701805B9F4FF2017A
:10ACA000918380838501F20180819181009711F069
:10ACB000049602C080E090E0B8010E94234A8823F5
:10ACC00001F1E2E4F7E08491882341F09091C00023
:10ACD00095FFFCCF8093C6003196F5CFF8018191A6
:10ACE000882339F09091C00095FFFCCF8093C60077
:10ACF000F6CFF701E950FF4F1082118212821382C2
:10AD00002CC0EAE2F7E08491882341F09091C000E2
:10AD100095FFFCCF8093C6003196F5CFF801819165
:10AD2000882339F09091C00095FFFCCF8093C60036
:10AD3000F6CFE8E2F7E08491882341F09091C000DB
:10AD400095FFFCCF8093C6003196F5CF8091C0006F
:10AD500085FFFCCF8AE08093C600C6010E94CC40EC
:10AD6000AC960FB6F894DEBF0FBECDBFDF91CF918A
:10AD70001F910F91FF90EF90DF90CF90BF90AF9019
:10AD80009F908F907F906F905F904F903F9008952D
:10AD9000CF93DF93EC018B818823C1F1E6E1F7E0EB
:10ADA0008491882341F09091C00095FFFCCF80935F
:10ADB000C6003196F5CFFE01E950FF4F4081518129
:10ADC000628173812AE030E082EE95E00E941418DF
:10ADD000E4E1F7E08491882341F09091C00095FF71
:10ADE000FCCF8093C6003196F5CFC151DF4F48812B
:10ADF00059816A817B812AE030E082EE95E00E94F1
:10AE000014188091C00085FFFCCF11C0E4E0F7E08A
:10AE10008491882341F09091C00095FFFCCF8093EE
:10AE2000C6003196F5CF8091C00085FFFCCF8AE047
:10AE30008093C600DF91CF910895AF92BF92CF92D9
:10AE4000DF92EF92FF920F931F93CF93DF935C01FA
:10AE5000EB01FB0101900020E9F78F01015011097E
:10AE6000061B170B6C01F4EDCF0ED11CF6011082FE
:10AE70006EE470E0CE010E941ED47C01009729F49C
:10AE8000F8013197EC0FFD1F0DC060E270E00E94E9
:10AE90001ED4EC0121966AE270E0C7010E941ED424
:10AEA000FC0131978DE081838AE082831382BE01A9
:10AEB000C50180539F4F0E94E94BF6018081882392
:10AEC00009F1E3E3F8E08491882341F09091C00018
:10AED00095FFFCCF8093C6003196F5CFEEEEF6E0FD
:10AEE0008491882341F09091C00095FFFCCF80931E
:10AEF000C6003196F5CF8091C00085FFFCCF8AE077
:10AF00008093C600DF91CF911F910F91FF90EF903A
:10AF1000DF90CF90BF90AF9008952F923F924F92C5
:10AF20005F926F927F928F929F92AF92BF92CF92D9
:10AF3000DF92EF92FF920F931F93CF93DF93CDB7E2
:10AF4000DEB7CC55D1090FB6F894DEBF0FBECDBF2A
:10AF50008C0185509F4F5C01662339F0F50110820A
:10AF6000F801838181111DC015C0FC0180818823F7
:10AF700009F4ADC0F801ED50FF4FC080D180E280F0
:10AF8000F3800E94C4C5C616D706E806F90608F481
:10AF90009EC0E4CFC801F4DAF8018381882309F464
:10AFA00096C0F80186A58F9385A58F9385EE96E0D0
:10AFB0009F938F937E01FFE3EF0EF11CFF92EF92C0
:10AFC0000E94E8D40F900F900F900F900F900F9069
:10AFD000B12CF70101900020E9F73197EE19FF0934
:10AFE000BE1684F46701CB0CD11CB7FCDA94F601D1
:10AFF0008081992787FD90950E94ADD3F6018083CB
:10B00000B394E7CF4801F3E38F0E911C40E050E08A
:10B01000BA01C4010E947346512CCE0101966C0105
:10B020002EED622E26E0722E5E0191E2A90EB11C79
:10B0300040E050E0B601C4010E94C0451816DCF59E
:10B04000412CF60101900020E9F73197EC19FD0938
:10B050004E1674F41601240C311C47FC3A94F1018D
:10B06000808190E00E94ADD3F10180834394E9CFC9
:10B070008A858E37E9F245E050E0B701C6010E94AB
:10B0800039D4892BA9F6FF92EF927F926F92BF92EB
:10B09000AF920E94E8D4C5010E94741A8AED96E02E
:10B0A0000E94E71A0F900F900F900F900F900F9043
:10B0B00055245394BDCF511004C08FEF9FEFF8017A
:10B0C00004C0F80185A596A5019696A785A7C45A40
:10B0D000DF4F0FB6F894DEBF0FBECDBFDF91CF912B
:10B0E0001F910F91FF90EF90DF90CF90BF90AF90A6
:10B0F0009F908F907F906F905F904F903F902F9098
:10B1000008950F931F93CF93DF93EC018C010C52A2
:10B110001F4FC8010E940C47C8010E945647188261
:10B120001982DF91CF911F910F910895EF92FF92B5
:10B130000F931F93CF93DF93CDB7DEB76F970FB603
:10B14000F894DEBF0FBECDBF8C017C018EE4E80E0B
:10B15000F11CC801805B9F4FF70191838083E2550A
:10B16000FF4F22E030E031832083329670E071831C
:10B17000608340E050E0BA0104960E947346F701F4
:10B18000808191812BE1FC013496DE0115960190BE
:10B190000D922A95E1F7FC01828193819C838B8338
:10B1A00084E494E09A838983AE014F5F5F4F61E34B
:10B1B00075E0C8010BD8CE0101960E94CC406F9675
:10B1C0000FB6F894DEBF0FBECDBFDF91CF911F91B8
:10B1D0000F91FF90EF900895CF92DF92EF92FF9240
:10B1E0000F931F93CF93DF93CDB7DEB76F970FB653
:10B1F000F894DEBF0FBECDBF8C016C012EE4C20EF1
:10B20000D11C805B9F4FF60191838083E255FF4FF5
:10B2100021E030E0318320837801FEEFEF0EF11C56
:10B22000F7011182108240E050E0BA0104960E94BA
:10B230007346F601808191812BE1FC013496DE0199
:10B24000159601900D922A95E1F7FC018281938178
:10B250009C838B8384E494E09A838983AE014F5F5F
:10B260005F4F61E375E0C8010E94E650CE01019690
:10B270000E94CC40F701808191816F960FB6F894BF
:10B28000DEBF0FBECDBFDF91CF911F910F91FF9019
:10B29000EF90DF90CF900895CF93DF93EC010E9461
:10B2A000A3740E941975CE018C529F4F0E9456477D
:10B2B0001A828091A40A882341F061E070E085EA57
:10B2C0009AE00E940D26892B21F18091B5128823E6
:10B2D00029F11092B512C0911909D0E0CC0FDD1FF1
:10B2E000CF5FDB4E68817981882777FD8095982F25
:10B2F0000E9476CD20914702309148024091490248
:10B3000050914A020E94D7CE181644F4198218822E
:10B3100005C08EEC96E00E94E71AD7CFDF91CF915F
:10B320000895CF93DF93EC010E94A3740E944A75A5
:10B33000CE018C529F4F0E9456471A828091B512BF
:10B340008823F9F01092B512C0911909D0E0CC0F02
:10B35000DD1FCF5FDB4E68817981882777FD80957F
:10B36000982F0E9476CD209147023091480240915B
:10B37000490250914A020E94D7CE181614F419823D
:10B380001882DF91CF9108952F923F924F925F9252
:10B390006F927F928F929F92AF92BF92CF92DF92E5
:10B3A000EF92FF920F931F93CF93DF93CDB7DEB74A
:10B3B000C454D1090FB6F894DEBF0FBECDBF3C0117
:10B3C0001B014A012FA309A7EBA62196ACAEBDAE87
:10B3D000CEAEDFAE219734E0239F20011124440D2F
:10B3E000551D5AAB49ABDA01CD90DD90ED90FC9044
:10B3F000FC01E40DF51D2081318142815381C7019B
:10B40000B6010E94FBCB6BAB7CAB8DAB9EABB4E0CB
:10B410000B9F80011124F401E00FF11FF8AFEFAB97
:10B4200080809180A280B380F301E00FF11F208122
:10B43000318142815381C501B4010E94FBCB69AFC8
:10B440007AAF8BAF9CAF2BA5F4E02F9FC0011124E6
:10B45000F301E80FF91F2081318142815381298F47
:10B460003A8F4B8F5C8FF101E80FF91F608171817A
:10B47000828193810E94FACB6F8F78A389A39AA3CC
:10B48000D1011C968D919D910D90BC91A02D8DA701
:10B490009EA7AFA7B8ABD3011C962D913D914D91BE
:10B4A0005C911F972BA33CA34DA35EA3A70196011C
:10B4B00050582D8B3E8B4F8B588FD501C401B058FF
:10B4C000898B9A8BAB8BBC8BF101E40DF51D2BA9FD
:10B4D0003CA94DA95EA960817181828193810E94FE
:10B4E000FACB6B017C01F101E00FF11F29AD3AAD00
:10B4F0004BAD5CAD60817181828193810E94FACBFA
:10B500004B015C01A70196016D897E898F89988D19
:10B510000E94A9CF2B013C01A501940169897A8978
:10B520008B899C890E94A9CF9B01AC01C301B20108
:10B530000E94FBCB2B013C01A50194016D897E8902
:10B540008F89988D0E94A9CF4B015C01A7019601BC
:10B5500069897A898B899C890E94A9CF9B01AC015A
:10B56000C501B4010E94FACBA30192010E946ECCE6
:10B570006B017C0120E030E0A9010E94D4CC87FF60
:10B580000AC02BED3FE049EC50E4C701B6010E9430
:10B59000FBCB6B017C016F968FAD6F97882351F0C9
:10B5A0002BED3FE049EC50E4C701B6010E94FACB15
:10B5B0006B017C016E962CAD3DAD4EAD5FAD6E97CF
:10B5C000C701B6010E94A9CF2F8D38A149A15AA168
:10B5D0005F770E94E4CE4B015C012FE632E143E845
:10B5E0005AE30E94D4CC87FDC4C1C501B4010E94B6
:10B5F000B1CD0E9448CD7E8F6D8FDB01AB2B21F446
:10B60000E1E0F0E0FE8FED8F2D8D3E8DB90180E001
:10B6100090E00E9474CD4B015C019B01AC01C7011D
:10B62000B6010E94DBCC2B013C01A50194016F8D7A
:10B6300078A189A19AA10E94DBCC25966CAF7DAF41
:10B640008EAF9FAF25972BA13CA14DA15EA16DA50B
:10B650007EA58FA598A90E94FACBA50194010E940E
:10B66000DBCC6DA77EA78FA798AB20E030E040E051
:10B670005FE3C301B2010E94A9CFA30192010E941E
:10B68000A9CF9B01AC0160E070E080E89FE30E94DD
:10B69000FACB6F8F78A389A39AA3CE010196FC0100
:10B6A0004BA534E0439FE00DF11D1124298D3A8D07
:10B6B0004B8D5C8D20833183428353832BA13CA12E
:10B6C0004DA15EA12D873E874F87588BB12C41E05D
:10B6D00050E05A8F498F81E090E08C0F9D1FBFA1F1
:10B6E000A4E0BA9F800D911D11249CA78BA721E097
:10B6F00030E02C0F3D1F59A544E0549F200D311D13
:10B7000011243AA729A7F8A7EFA3498D5A8D8D8D4B
:10B710009E8D4817590708F017C188E18B150CF466
:10B7200044C02F8D38A149A15AA169897A898B8992
:10B730009C890E94A9CF6B017C01A30192016D89B4
:10B740007E898F89988D0E94A9CFA70196010E94BA
:10B75000FBCBA62E172F982E892E2F8D38A149A10D
:10B760005AA16D897E898F89988D0E94A9CF6B011E
:10B770007C01A301920169897A898B899C890E9445
:10B78000A9CF9B01AC01C701B6010E94FACB6D8B1A
:10B790007E8B8F8B988FB3948A2D912FA92DB82DE6
:10B7A000898B9A8BAB8BBC8B6AC0A98DBA8DBD017E
:10B7B00080E090E00E9474CDA30192010E94A9CF85
:10B7C0006B017C010E94D8CC698B7A8B8B8B9C8B14
:10B7D000C701B6010E940CD04B015C01E9A9FAA98E
:10B7E000C080D180E280F380F7FAF094F7F8F0940B
:10B7F000AFA9B8AD2D913D914D915C912BA33CA388
:10B800004DA35EA329893A894B895C89C701B6019A
:10B810000E94A9CF6D8B7E8B8F8B988FA501940191
:10B820006BA17CA18DA19EA10E94A9CF9B01AC011F
:10B830006D897E898F89988D0E94FBCB6D8B7E8B65
:10B840008F8B988FA5019401C701B6010E94A9CFE3
:10B850006B017C0129893A894B895C896BA17CA1A8
:10B860008DA19EA10E94A9CF9B01AC01C701B60189
:10B870000E94FACB698B7A8B8B8B9C8BB12C2D8998
:10B880003E894F89588D6BA97CA98DA99EA90E94DC
:10B89000FBCBEBA5FCA5608371838283938329890D
:10B8A0003A894B895C8969AD7AAD8BAD9CAD0E94BC
:10B8B000FBCBA9A5BAA56D937D938D939C9313970C
:10B8C00025962CAD3DAD4EAD5FAD2597EFA1F8A50A
:10B8D00060817181828193810E94FBCBAFA1B8A569
:10B8E0006D937D938D939C9313972DA53EA54FA5A6
:10B8F00058A96D857E858F8598890E94FBCB6D87C1
:10B900007E878F87988BCE0101960E94C71CFE010F
:10B91000E15AFF4F6F012196ECACFDAC0EAD1FADAF
:10B9200021979E01235F3F4FAE01475F5F4FBE01EE
:10B930006B5F7F4FCE01019656D5298D3A8D2F5FD3
:10B940003F4F3A8F298FE1CE9101245F3F4FA101F4
:10B95000485F5F4FB1016C5F7F4FDE01A15ABF4F5F
:10B960006D012196ECACFDAC0EAD1FAD2197C10170
:10B970003AD5CC5BDF4F0FB6F894DEBF0FBECDBF1C
:10B98000DF91CF911F910F91FF90EF90DF90CF90BB
:10B99000BF90AF909F908F907F906F905F904F90EF
:10B9A0003F902F9008952F923F924F925F926F9207
:10B9B0007F928F929F92AF92BF92CF92DF92EF923F
:10B9C000FF920F931F93CF93DF93CDB7DEB76897A6
:10B9D0000FB6F894DEBF0FBECDBF1C012A013B019C
:10B9E00048015901DC01D8966D917D918D919C9112
:10B9F000DB970E9474CD6B017C01A30192010E9430
:10BA0000A9CF0E94C1CC0E9448CD6D877E878F87C9
:10BA1000988BA5019401C701B6010E94A9CF0E948D
:10BA2000C1CC0E9448CD698B7A8B8B8B9C8B2D85EA
:10BA30003E854F855889283731054105510540F429
:10BA400088E790E0A0E0B0E08D879E87AF87B88B55
:10BA500029893A894B895C89283731054105510587
:10BA600040F488E790E0A0E0B0E0898B9A8BAB8B44
:10BA7000BC8B91012C5B3F4FD9018D919D910D9015
:10BA8000BC91A02D8D839E83AF83B887BC01CD016F
:10BA90000E9476CD69837A838B839C83F10164ADA8
:10BAA00075AD86AD97AD0E9474CD69877A878B8717
:10BAB0009C8720E030E0A90169817A818B819C819B
:10BAC0000E94D4CC882339F1A7019601C701B601A1
:10BAD0000E94A9CF4B015C0129853A854B855C8585
:10BAE000CA01B9010E94A9CF9B01AC01C501B401F3
:10BAF0000E94FACB4B015C0129813A814B815C8128
:10BB0000CA01B9010E94FBCB9B01AC01C501B40184
:10BB10000E94DBCC03C060E070E0CB010E94C1CC8E
:10BB20000E9443CD2B013C016D817E818F819885E0
:10BB300090958095709561957F4F8F4F9F4F0E9494
:10BB400076CD4B015C01F101E05CFF4F60817181BA
:10BB5000828193810E9474CD6D837E838F839887C9
:10BB600020E030E0A901C501B4010E94D4CC8823B3
:10BB700049F12D813E814F815885CA01B9010E944A
:10BB8000A9CF6D8B7E8B8F8B988FA7019601C701F4
:10BB9000B6010E94A9CF9B01AC016D897E898F8976
:10BBA000988D0E94FACB6B017C01A5019401C5011F
:10BBB000B4010E94FBCB9B01AC01C701B6010E94FE
:10BBC000DBCC03C060E070E0CB010E94B1CDD101BD
:10BBD00050968D909D90AD90BC90539775016401E7
:10BBE000C418D508E608F7080E9443CDC61AD70A3C
:10BBF000E80AF90AF7FE6BC020E030E0A90169818C
:10BC00007A818B819C810E94D4CC882309F447C01F
:10BC100029813A814B815C81CA01B9010E94FBCB29
:10BC20006B017C01C501B4010E9474CD9B01AC0184
:10BC3000C701B6010E94A9CF6B017C0129853A8515
:10BC40004B855C85CA01B9010E94A9CF9B01AC015B
:10BC5000C701B6010E94FACB6B017C012D813E81A8
:10BC60004F815885CA01B9010E94A9CF9B01AC013F
:10BC7000C701B6010E94FBCB6B017C0120E030E0E4
:10BC800040E850E469817A818B819C810E94A9CF30
:10BC90009B01AC01C701B6010E94DBCC03C060E090
:10BCA00070E0CB010E94C1CC0E9443CD2B013C012E
:10BCB00097FF03C0412C512C3201481459046A04E7
:10BCC0007B0410F024013501C12CD12C76018FB7F3
:10BCD000F894F101E45BFF4F9081911121C0F101D3
:10BCE000448A558A668A778AC40CD51CE61CF71CE0
:10BCF000D101C08ED18EE28EF38E2D853E854F858B
:10BD0000588924AF35AF46AF57AFA05CBF4F2989E4
:10BD10003A894B895C892D933D934D935C9313979E
:10BD20008FBF68960FB6F894DEBF0FBECDBFDF9110
:10BD3000CF911F910F91FF90EF90DF90CF90BF9028
:10BD4000AF909F908F907F906F905F904F903F90BB
:10BD50002F9008954F925F926F927F92AF92BF9211
:10BD6000CF92DF92EF92FF920F931F93CF93DF93C7
:10BD7000EB017A01209709F458C04115510509F4E7
:10BD800054C0AAA4BBA40CA51DA59501A8016EA131
:10BD90007FA188A599A50E94D4CC882309F445C029
:10BDA0008FA981113AC0F70146A057A060A471A4E1
:10BDB000A3019201B501C8010E94D7CE18166CF5F7
:10BDC000A3019201C301B2010E94A9CF6B017C01C2
:10BDD0008AA99BA9ACA9BDA9BC01CD0190589B0122
:10BDE000AC010E94FBCB2EA53FA548A959A90E94F2
:10BDF000A9CF9B01AC01C701B6010E94FACB0E94FA
:10BE000016D06B017C019B01AC01B501C8010E94F9
:10BE1000D4CC87FD02C056018701A501B8014EA30D
:10BE20005FA368A779A781E08EABDF91CF911F91C7
:10BE30000F91FF90EF90DF90CF90BF90AF907F90E9
:10BE40006F905F904F900895DF92EF92FF920F9363
:10BE50001F93CF93DF938091E40D8FB7F894E09018
:10BE6000E30D8FBF8091E40D90E08E1991098F70E2
:10BE700099270497F4F01091E40D13501F7040E0DF
:10BE800050E000E0F12C8DE4D82E1E1591F0111138
:10BE900001C010E11150D19EE0011124CB51D24FCD
:10BEA000602F7F2DCE0156DF402F5F2D0C2FFD2EF2
:10BEB000ECCFDF91CF911F910F91FF90EF90DF902A
:10BEC00008954F925F926F927F92AF92BF92CF92FE
:10BED000DF92EF92FF920F931F93CF93DF938C012A
:10BEE000EB01009709F453C0FC0187A981114FC0F1
:10BEF00046A057A060A471A4AEA0BFA0C8A4D9A4B6
:10BF00009501A601C301B2010E94D4CC87FF3FC0B6
:10BF1000A3019201C301B2010E94A9CF2B013C01F0
:10BF2000F80182A993A9A4A9B5A9BC01CD01905893
:10BF30009B01AC010E94FBCBF80126A537A540A9C7
:10BF400051A90E94A9CF9B01AC01C301B2010E947B
:10BF5000FACB0E9416D07B018C019B01AC01B5018C
:10BF6000C6010E94D4CC87FF02C0750186019701EB
:10BF7000A801B501C6010E94D4CC882341F0A701D5
:10BF8000B8014EA35FA368A779A781E08EABDF91CC
:10BF9000CF911F910F91FF90EF90DF90CF90BF90C6
:10BFA000AF907F906F905F904F900895EF92FF92C7
:10BFB0000F931F93CF93DF93F090E30D00E010E019
:10BFC00080E090E02DE4E22E2091E40DF21689F05D
:10BFD000EF9CE0011124CB51D24FAE01B80171DFCB
:10BFE00081E08F0D803109F480E0F82EC8018E01C8
:10BFF000EBCF40E050E0B801DF91CF911F910F915E
:10C00000FF90EF905ECF4F925F926F927F928F92F0
:10C010009F92AF92BF92CF92DF92EF92FF920F93D7
:10C020001F93CF93DF939090E30DC0E0D0E03DE409
:10C03000832E892D992787FD90952091E40D30E07E
:10C0400082179307B9F1889E5001899EB00C112484
:10C05000C5018B51924F5C01209729F18EA9811166
:10C0600004C0F50186A98823F1F0CAA0DBA0ECA0EA
:10C07000FDA0A7019601F50166A177A180A591A574
:10C080000E94DBCC2B013C01A70196016EA17FA190
:10C0900088A599A50E94DBCCAB01BC01930182016C
:10C0A000CE0181DC1EAA9394F0E19F1201C0912C75
:10C0B000E501BFCF2097E9F0CAA0DBA0ECA0FDA06E
:10C0C000A70196016DEC7CEC8CE49DE30E94DBCC37
:10C0D0004B015C01A70196016EA17FA188A599A5DE
:10C0E0000E94DBCCAB01BC0195018401CE015BDC7D
:10C0F0001EAADF91CF911F910F91FF90EF90DF90DB
:10C10000CF90BF90AF909F908F907F906F905F90F7
:10C110004F90089599DE4ADF76CF1092E40D109289
:10C12000E30D80E1EAECF2E1DF011D928A95E9F787
:10C130001092BA121092BB121092BC121092BD1241
:10C140001092BE121092BF121092C0121092C11221
:10C150001092C2121092C3121092C4121092C51201
:10C160001092C6121092C7121092C8121092C912E1
:10C170001092B6121092B7121092B8121092B91211
:10C1800008954F925F926F927F928F929F92AF929B
:10C19000BF92CF92DF92EF92FF920F931F93CF93B4
:10C1A000DF938091B512882309F4EFC0C090470255
:10C1B000D0904802E0904902F0904A026091011448
:10C1C00070910214882777FD8095982F0E9476CD74
:10C1D00020E030E040E050E40E94FBCB9601A70154
:10C1E0000E94D4CC87FDD1C05090E30D612C712CFE
:10C1F00000E010E04DE4442E8091E40D581609F45F
:10C2000053C0852D90E0489EF001499EF00D112409
:10C21000EB51F24F4081518162817381452B462B56
:10C22000472B81F44481558166817781452B462BCC
:10C23000472B41F44085518562857385452B462BFC
:10C24000472B69F1489EE001499ED00D1124CB5146
:10C25000D24F6C857D858E859F850E9476CD4B0162
:10C260005C01688979898A899B890E9474CD9B01C8
:10C27000AC01C501B4010E94DBCC2AA13BA14CA1B9
:10C280005DA10E94A9CF5B01D82FC92F9301A801FE
:10C290000E94D7CE18161CF435010D2F1C2F539475
:10C2A000852D8F70582EA8CF2091430230914402E3
:10C2B0004091450250914602B301C8010E94A9CFA6
:10C2C0009B01AC01B601C7010E94FBCB8B01D82FAB
:10C2D000C92F9601A7010E94D4CC87FD03C0680135
:10C2E000ED2EFC2E00914B0210914C02D0914D028C
:10C2F000C0914E0298014D2F5C2FB601C7010E94DC
:10C30000D7CE18161CF08601DE2DCF2D8090DF0DC4
:10C310009090E00DA090E10DB090E20D98014D2FAE
:10C320005C2FC501B4010E94D7CE1816D4F420E0CA
:10C3300037ED43EA5CE3B8018D2F9C2F0E94A9CF13
:10C340006B017C0128E431EE4AE75FE3C501B401EB
:10C350000E94A9CFA70196010E94FBCB8B01D82F89
:10C36000C92FC801AD2FBC2F8093DF0D9093E00D36
:10C37000A093E10DB093E20DB8018D2F9C2F0E9488
:10C3800043CD7093021460930114DF91CF911F91FC
:10C390000F91FF90EF90DF90CF90BF90AF909F9064
:10C3A0008F907F906F905F904F90089560911709E4
:10C3B0009091E30D8091E40D981781F08091E30D49
:10C3C0009DE4899FF0011124E35DF14F608190911C
:10C3D000E40D891719F08F5F8F70F9CF70E089E055
:10C3E0000E948CC6CECE2F923F924F925F926F9258
:10C3F0007F928F929F92AF92BF92CF92DF92EF92F5
:10C40000FF920F931F93CF93DF93CDB7DEB7C35641
:10C41000D1090FB6F894DEBF0FBECDBF2C015B0172
:10C420004A013901E9AAFBA60CA71DA786012091A4
:10C43000E40D2F5F2FAF203109F41FAE3FADE32E87
:10C44000FF24E7FCF0948091E30D90E08E159F05AA
:10C4500039F40E940A770E94031F0E94F193F3CFE0
:10C4600020911A1330911B1340911C1350911D13EE
:10C47000D2016D917D918D919C910E94A9CF0E94D6
:10C4800079CF2A966CAF7DAF8EAF9FAF2A97209160
:10C490001E1330911F134091201350912113F50169
:10C4A00060817181828193810E94A9CF0E9479CF9E
:10C4B0002E966CAF7DAF8EAF9FAF2E97209122133B
:10C4C000309123134091241350912513D4016D9181
:10C4D0007D918D919C910E94A9CF0E9479CF629607
:10C4E0006CAF7DAF8EAF9FAF6297209126133091D6
:10C4F00027134091281350912913F3016081718112
:10C50000828193810E94A9CF0E9479CF6BAF7CAFCB
:10C510008DAF9EAF8091D6129091D712A091D81274
:10C52000B091D9122BAD3CAD4DAD5EAD281739079A
:10C530004A075B0709F4B3C0E091190934E0E39FAF
:10C54000F0011124ED50FC4E20913F023091400249
:10C5500040914102509142026081718182819381B8
:10C560000E94D4CC87FF2DC08BAD9CADADADBEADD0
:10C570008093D6129093D712A093D812B093D91269
:10C58000E2E7F8E08491882341F09091C00095FFA4
:10C59000FCCF8093C6003196F5CFE8E5F8E08491B2
:10C5A000882341F09091C00095FFFCCF8093C60096
:10C5B0003196F5CF8091C00085FFFCCF8AE0809353
:10C5C000C6008091D6129091D712A091D812B09146
:10C5D000D9122BAD3CAD4DAD5EAD281B390B4A0BCE
:10C5E0005B0BCA01B90157FF07C090958095709504
:10C5F00061957F4F8F4F9F4F0E9476CD6B017C01DD
:10C600006091B5097091B6098091B7099091B80908
:10C61000680F791F882777FD8095982F0E9476CD27
:10C6200020912613309127134091281350912913FC
:10C630000E94A9CF9B01AC01C701B6010E94D7CED1
:10C6400018166CF58BAD9CADADADBEAD8093D6121A
:10C650009093D712A093D812B093D912E2E7F8E0E2
:10C660008491882341F09091C00095FFFCCF809386
:10C67000C6003196F5CFEAE3F8E08491882341F0D3
:10C680009091C00095FFFCCF8093C6003196F5CF06
:10C690008091C00085FFFCCF8AE08093C600809126
:10C6A000E40D9DE4899F10011124D101AB51B24FDB
:10C6B0001D01FD01E45BFF4F10822091CA123091F1
:10C6C000CB124091CC125091CD122BA33CA34DA381
:10C6D0005EA32A964CAC5DAC6EAC7FAC2A97421A36
:10C6E000530A640A750A77FE08C0709460945094E7
:10C6F0004094411C511C611C711CD1014D925D92F2
:10C700006D927C9213972091CE123091CF1240916E
:10C71000D0125091D1122FA338A749A75AA72E960D
:10C720008CAC9DACAEACBFAC2E97821A930AA40A17
:10C73000B50AB7FE08C0B094A09490948094811C70
:10C74000911CA11CB11CD10114968D929D92AD92A9
:10C75000BC9217972091D2123091D3124091D412EB
:10C760005091D5122BAB3CAB4DAB5EAB6296CCACD3
:10C77000DDACEEACFFAC6297C21AD30AE40AF50A4C
:10C78000F7FE08C0F094E094D094C094C11CD11C72
:10C79000E11CF11CD1011896CD92DD92ED92FC9234
:10C7A0001B972091D6123091D7124091D8125091F8
:10C7B000D9122FAB38AF49AF5AAF2BAD3CAD4DAD11
:10C7C0005EAD8FA998ADA9ADBAAD281B390B4A0B48
:10C7D0005B0B57FF07C050954095309521953F4F13
:10C7E0004F4F5F4FA0912B02B0912C020E94F3D0CB
:10C7F00024E630E040E050E00E94C7D0D1011C9612
:10C800002D933D934D935C931F97C814D904EA046C
:10C81000FB0414F475016401C216D306E406F506A0
:10C8200014F469017A01D301C2014C145D046E0451
:10C830007F0414F4D701C601F101808B918BA28B88
:10C84000B38B0697A105B10508F47EC7E85BFF4FDF
:10C850008091170990911809AA2797FDA095BA2FE2
:10C8600080839183A283B3832A962CAD3DAD4EADD8
:10C870005FAD2A978BA19CA1ADA1BEA12817390756
:10C880004A075B0724F0D10190961C9203C081E017
:10C89000F10180A32E962CAD3DAD4EAD5FAD2E9730
:10C8A0008FA198A5A9A5BAA5281739074A075B073C
:10C8B0003CF4D10190968C919097826090968C93E5
:10C8C00062962CAD3DAD4EAD5FAD62978BA99CA934
:10C8D000ADA9BEA9281739074A075B073CF4D10167
:10C8E00090968C919097846090968C932BAD3CADF4
:10C8F0004DAD5EAD8FA998ADA9ADBAAD281739077A
:10C900004A075B073CF4D10190968C919097886020
:10C9100090968C93F8018081D10191968C93452853
:10C920004628472809F05F98F10184819581A68106
:10C93000B781892B8A2B8B2B09F08A98F10180858E
:10C940009185A285B385892B8A2B8B2B41F09FB7CC
:10C95000F894809108018E7F809308019FBFF101B8
:10C9600084859585A685B785892B8A2B8B2B11F01D
:10C9700012984798F10184859585A685B785892BFE
:10C980008A2B8B2BE9F41091EA120091EB12F091B3
:10C99000EC12FBA32091ED122FA3212F302F4F2F4C
:10C9A0005FA169A97BA58CA59DA50E94D4CC87FD1C
:10C9B00016C019A90BA53CA53BA34DA54FA30FC0BD
:10C9C0001091061300910713509108135BA38091F7
:10C9D00009138FA3212F302F452F582FE2CF80919D
:10C9E000CA129091CB12A091CC12B091CD122A967E
:10C9F0002CAD3DAD4EAD5FAD2A97281B390B4A0BD0
:10CA00005B0BCA01B9010E9476CD20911A133091B7
:10CA10001B1340911C1350911D130E94DBCC4B0142
:10CA20005C01698B7A8B8B8B9C8B8091CE12909161
:10CA3000CF12A091D012B091D1122E962CAD3DAD57
:10CA40004EAD5FAD2E97281B390B4A0B5B0BCA010D
:10CA5000B9010E9476CD20911E1330911F13409191
:10CA60002013509121130E94DBCC6BAB7CAB8DABC0
:10CA70009EAB6D8B7E8B8F8B988F8091D212909115
:10CA8000D312A091D412B091D51262962CAD3DADC7
:10CA90004EAD5FAD6297281B390B4A0B5B0BCA0189
:10CAA000B9010E9476CD2091221330912313409139
:10CAB0002413509125130E94DBCC6B017C01698FFC
:10CAC0007A8F8B8F9C8F8091D6129091D712A091E4
:10CAD000D812B091D9122BAD3CAD4DAD5EAD281B37
:10CAE000390B4A0B5B0BCA01B9010E9476CD20912C
:10CAF00026133091271340912813509129130E9437
:10CB0000DBCC2B013C0160912B0270912C02882719
:10CB100077FD8095982F0E9476CD9B01AC01C301D3
:10CB2000B2010E94A9CF20E030E048EC52E40E941C
:10CB3000DBCC6D8F7E8F8F8F98A3D1014D905D9050
:10CB40006D907C90B6E04B165104610471040CF5B5
:10CB5000F1014480558066807780F6E04F165104DD
:10CB600061047104B4F4D10118964D905D906D90FC
:10CB70007C901B97B6E04B165104610471044CF491
:10CB8000DC01CB01BF77F10186A797A7A0ABB1ABC2
:10CB900027C0C501B4010E9454D04B015C016BA9B0
:10CBA0007CA98DA99EA90E9454D09B01AC01C5010E
:10CBB000B4010E94FBCB4B015C01C701B6010E948E
:10CBC00054D09B01AC01C501B4010E94FBCB0E9473
:10CBD00016D0D1019E966D937D938D939C93D197A2
:10CBE000F10146A457A460A871A8A301920160E0D6
:10CBF00070E080E89FE30E94DBCC9B01AC01612FD9
:10CC0000702F8BA19FA10E94A9CF6DA77EA78FA790
:10CC100098AB9091E40D8091E30D292F30E0281B13
:10CC200031092F7033273AAB29AB2DA53EA54FA56F
:10CC300058A960E074E284E799E40E94DBCC0E948A
:10CC400079CF6B017C0149A95AA9423051050CF4F6
:10CC500044C04A01AA2497FCA094BA2CC501B4018F
:10CC60000E9476CD20E030E040E051E40E94D4CC38
:10CC700087FF33C080913A1390913B13A0913C13EE
:10CC8000B0913D13C816D906EA06FB0630F5BC0183
:10CC9000CD016C197D098E099F09660F771F881FCA
:10CCA000991FA50194010E94A5D0CA01B9010E9453
:10CCB00074CD0E9479CF6C0D7D1D8E1D9F1D0E942D
:10CCC00074CD9B01AC0160E074E284E799E40E94BA
:10CCD000DBCC6DA77EA78FA798AB2DA53EA54FA552
:10CCE00058A9C301B2010E94A9CF6FAB78AF89AF39
:10CCF0009AAFD10192966D937D938D939C93959766
:10CD000050966D917D918D919C9153970E9474CD19
:10CD10002DA53EA54FA558A90E94A9CF0E94C1CC20
:10CD20000E9448CD6B017C01F10160AF71AF82AF11
:10CD300093AF8E010F5E1F4F2AE233E126963FAF7D
:10CD40002EAF2697AE014F5D5F4F5AA349A3CE0188
:10CD5000019622969FAF8EAF22971BA21FA290E84A
:10CD60009BA7AFE3ACA7F80161917191819191917B
:10CD70008F012DA53EA54FA558A90E94A9CF2296A7
:10CD8000AEADBFAD22976D937D938D939D9322960B
:10CD9000BFAFAEAF22972B013C01E89477F82696FF
:10CDA000EEADFFAD269781909190A190B19026961F
:10CDB000FFAFEEAF2697A5019401C301B2010E9417
:10CDC000D7CE1816D4F4A3019201C501B4010E9474
:10CDD000DBCCB62EA72E982E892E262F372F482F44
:10CDE000592F6BA17FA18BA59CA50E94D4CC87FD58
:10CDF00004C0BBA2AFA29BA68CA629A13AA1021790
:10CE0000130709F0B0CF20E030E040E85FE36BA10A
:10CE10007FA18BA59CA50E94D4CC87FF3DC05E015D
:10CE200031E1A30EB11C8E010F5F1F4F2BA13FA15B
:10CE30004BA55CA5D8016D917D918D919C910E942F
:10CE4000A9CFF80161937193819391938F01EA15B2
:10CE5000FB0561F72BA13FA14BA55CA56FA978ADA0
:10CE600089AD9AAD0E94A9CFD10192966D937D9321
:10CE70008D939C939597C701B6010E9474CD2BA109
:10CE80003FA14BA55CA50E94A9CF0E9448CDF1010E
:10CE900060AF71AF82AF93AF00910E1310910F137B
:10CEA00020911013309111134091D2095091D30960
:10CEB0006091D4097091D5098CE699E00E946522B1
:10CEC000D10150966D917D918D919C9153970E94C7
:10CED00074CD6B017C01D1019E962D913D914D91B8
:10CEE0005C91D19768962CAF3DAF4EAF5FAF68971E
:10CEF0000E94DBCC6BA37CA38DA39EA3F101808059
:10CF00009180A280B38081149104A104B10461F5E1
:10CF100084819581A681B781892B8A2B8B2B21F562
:10CF200080859185A285B385892B8A2B8B2BE1F493
:10CF30002091FE123091FF12409100135091011385
:10CF40006BA17CA18DA19EA10E94A9CF0E94C1CC02
:10CF500081010C5B1F4F0E9448CDD8016D937D93DA
:10CF60008D939C93139714C1209102133091031356
:10CF700040910413509105136BA17CA18DA19EA13A
:10CF80000E94A9CF0E94C1CC0E9448CD81010C5BB8
:10CF90001F4FF80160837183828393834090DA127C
:10CFA0005090DB126090DC127090DD120E9474CD04
:10CFB0006FA378A789A79AA7C501B4010E9476CD6F
:10CFC0009B01AC016FA178A589A59AA50E94A9CF64
:10CFD000A70196010E94DBCC4B015C01C301B201A9
:10CFE0000E9474CD9B01AC01C501B4010E94D7CE53
:10CFF000181634F4D8014D925D926D927C9213977D
:10D000004090DE125090DF126090E0127090E112BA
:10D01000F80160817181828193810E9474CD4B01FE
:10D020005C01D10114966D917D918D919C91179722
:10D030000E9476CD9B01AC01C501B4010E94A9CF2D
:10D04000A70196010E94DBCC4B015C01C301B20138
:10D050000E9474CD9B01AC01C501B4010E94D7CEE2
:10D06000181634F58091D109882331F0F8014082F7
:10D070005182628273821CC06091D6097091D70977
:10D080008091D8099091D9090E9474CD20911E13E6
:10D0900030911F1340912013509121130E94A9CF6A
:10D0A0000E9448CDD8016D937D938D939C931397E7
:10D0B0004090E6125090E7126090E8127090E912EA
:10D0C00081010C5B1F4FF801608171818281938126
:10D0D0000E9474CD4B015C01D1011C966D917D9134
:10D0E0008D919C911F970E9476CD9B01AC01C5014B
:10D0F000B4010E94A9CFA70196010E94DBCC4B018D
:10D100005C01C301B2010E9474CD9B01AC01C50159
:10D11000B4010E94D7CE18162CF4F8014082518237
:10D12000628273824090E2125090E3126090E412A7
:10D130007090E512D8016D917D918D919C910E9426
:10D1400074CD4B015C01F101608571858285938509
:10D150000E9476CD9B01AC01C501B4010E94A9CF0C
:10D16000A70196010E94DBCC6B017C01C301B201D7
:10D170000E9474CD9B01AC01C701B6010E94D7CEBD
:10D18000181634F4D8014D925D926D927C921397EB
:10D19000F101EC5BFF4F60817181828193810E947C
:10D1A00074CD6B017C012BA13CA14DA15EA10E941D
:10D1B000DBCC6C966CAF7DAF8EAF9FAF6C97F101FF
:10D1C00062AB73AB84AB95AB2DEB37E346E051E438
:10D1D000C701B6010E94A9CF0E9443CDD1015C9640
:10D1E0006D937D938D939C935F972091FA1230916C
:10D1F000FB124091FC125091FD122FAB38AF49AF9A
:10D200005AAF20E030E040E251E46BA97CA98DA93F
:10D210009EA90E94D7CE181694F08091D109882338
:10D2200071F020E030E040E05FE36FA978AD89ADB8
:10D230009AAD0E94A9CF6BA37FA38C0104C01BA24F
:10D240001FA200E010E489859A85AB85BC85A09675
:10D250008CAF9DAFAEAFBFAFA0972091F2123091CF
:10D26000F3124091F4125091F51224962CAF3DAF79
:10D270004EAF5FAF249720E030E040E05FE32496BC
:10D280006CAD7DAD8EAD9FAD24970E94A9CFF62EDB
:10D29000E72ED82EC92EA0966CAD7DAD8EAD9FAD7C
:10D2A000A0979F772F2D3E2D4D2D5C2D0E94D7CE20
:10D2B00018167CF42F2D3E2D4D2D5C2D6BA17FA1DA
:10D2C000C8010E94D4CC87FD04C0FBA2EFA20D2DA3
:10D2D0001C2D8D859E85AF85B889A4968CAF9DAF9A
:10D2E000AEAFBFAFA497C090EE12D090EF12E09017
:10D2F000F012F090F11220E030E040E05FE3C7016F
:10D30000B6010E94A9CFB62EA72E982E892EA496DC
:10D310006CAD7DAD8EAD9FADA4979F772B2D3A2D33
:10D32000492D582D0E94D7CE18167CF42B2D3A2D5E
:10D33000492D582D6BA17FA1C8010E94D4CC87FD37
:10D3400004C0BBA2AFA2092D182DD1019296BC91A9
:10D35000BBA7F101F3A1FCA7D1019496BC91BDA795
:10D36000F101F5A1FBAB2BA53CA54B2F5F2F6BA1CA
:10D370007FA1C8010E94D4CC87FD06C02BA52BA39A
:10D380003CA53FA30DA51BA949A95AA942305105A7
:10D390000CF405C15091B61259AB8091B712259685
:10D3A0008FAF25979091B81263969FAF6397A09126
:10D3B000B9126496AFAF649727E137EB41ED58E3BC
:10D3C00069A9782F892F9A2F0E94D7CE18160CF0B2
:10D3D000E6C02091BA123091BB124091BC1250911C
:10D3E000BD1269817A818B819C810E94FACB2B01CD
:10D3F0003C012091BE123091BF124091C012509159
:10D40000C1126D817E818F8198850E94FACB4B017C
:10D410005C01A3019201C301B2010E94A9CF2B01BB
:10D420003C01A5019401C501B4010E94A9CF9B0153
:10D43000AC01C301B2010E94FBCB0E9416D04B018C
:10D440005C012FA938AD49AD5AAD0E94D7CE181650
:10D450005CF4A50194016FA978AD89AD9AAD0E94E5
:10D46000DBCC3B012C0106C0612C712C50E8452E11
:10D470006FE3562E2091C2123091C3124091C41214
:10D480005091C512A0966CAD7DAD8EAD9FADA097AD
:10D490000E94FACB4B015C01E894B7F824962CADBE
:10D4A0003DAD4EAD5FAD2497C501B4010E94D7CE0E
:10D4B0001816E4F4A501940124966CAD7DAD8EADF3
:10D4C0009FAD24970E94DBCCB62EA72E982E892ED6
:10D4D000262F372F482F592FB301C2010E94D4CCD9
:10D4E00087FD04C06B2C7A2C492C582C2091C61235
:10D4F0003091C7124091C8125091C912A4966CADD8
:10D500007DAD8EAD9FADA4970E94FACB4B015C011F
:10D51000E894B7F8A7019601C501B4010E94D7CEDF
:10D520001816C4F4A5019401C701B6010E94DBCC12
:10D53000F62EE72ED82EC92E262F372F482F592FFB
:10D54000B301C2010E94D4CC87FD04C06F2C7E2C95
:10D550004D2C5C2C9301A2016BA57CA58DA59BA9EC
:10D560000E94A9CF4B015C019B01AC0169A92596E2
:10D570007FAD259763968FAD639764969FAD649753
:10D580000E94D4CC87FF0EC089A825969FAC259712
:10D590006396AFAC63976496BFAC649703C08BA0EF
:10D5A0009FA05801C401D501F10182A793A7A4A7A8
:10D5B000B5A76C966CAD7DAD8EAD9FAD6C97905858
:10D5C0009B01AC010E94FBCB68962CAD3DAD4EADEE
:10D5D0005FAD68970E94A9CF9B01AC016BE077ED2E
:10D5E00083E29BE30E94FACB0E9416D07B01D82EE7
:10D5F000C92E9B01482F592FB401C5010E94D4CCDC
:10D6000087FD03C04701AD2CBC2CC401D501F1013D
:10D6100086A397A3A0A7B1A797014D2D5C2D6BA55D
:10D620007CA58DA59BA90E94D4CC18162CF081E076
:10D63000D101D7968C9302C0F10117AA81E0D101E4
:10D64000D6968C9380E1FE013196AAEBB2E101906F
:10D650000D928A95E1F78BA59CA5ADA5BBA98093FA
:10D66000B6129093B712A093B812B093B9129C015E
:10D67000AD016BA17FA1C8010E94DBCC6B017C01D5
:10D680002BA53CA54DA55BA9B401C5010E94DBCC2F
:10D69000AB01BC0197018601C1010E94D35CBFAD03
:10D6A000B093E40D2A962CAD3DAD4EAD5FAD2A97FB
:10D6B0002093CA123093CB124093CC125093CD12C8
:10D6C0002E968CAD9DADAEADBFAD2E978093CE1294
:10D6D0009093CF12A093D012B093D11262962CAD3A
:10D6E0003DAD4EAD5FAD62972093D2123093D31211
:10D6F0004093D4125093D5128BAD9CADADADBEAD61
:10D700008093D6129093D712A093D812B093D912C7
:10D710000E948A60CD59DF4F0FB6F894DEBF0FBE6E
:10D72000CDBFDF91CF911F910F91FF90EF90DF90D0
:10D73000CF90BF90AF909F908F907F906F905F90B1
:10D740004F903F902F90D2C1CD59DF4F0FB6F89434
:10D75000DEBF0FBECDBFDF91CF911F910F91FF9024
:10D76000EF90DF90CF90BF90AF909F908F907F9081
:10D770006F905F904F903F902F900895EF92FF929F
:10D780000F931F93CF93DF937B018A01E9012091CF
:10D790001A1330911B1340911C1350911D13FC015F
:10D7A00060817181828193810E94A9CF0E9479CF8B
:10D7B0006093CA127093CB128093CC129093CD12C7
:10D7C00020911E1330911F1340912013509121136B
:10D7D000F70160817181828193810E94A9CF0E94AB
:10D7E00079CF6093CE127093CF128093D012909322
:10D7F000D112209122133091231340912413509180
:10D800002513F80160817181828193810E94A9CFE3
:10D810000E9479CF6093D2127093D3128093D41266
:10D820009093D512209126133091271340912813FD
:10D8300050912913688179818A819B810E94A9CFA7
:10D840000E9479CF6093D6127093D7128093D8122A
:10D850009093D91226ED32E142ED52E16EEC72E185
:10D860008AEC92E10E94B0741092B6121092B71234
:10D870001092B8121092B9121092BA121092BB12F2
:10D880001092BC121092BD121092BE121092BF12D2
:10D890001092C0121092C1121092C2121092C312B2
:10D8A0001092C4121092C5121092C6121092C71292
:10D8B0001092C8121092C912DF91CF911F910F914F
:10D8C000FF90EF90089520912613309127134091F7
:10D8D000281350912913FC01608171818281938109
:10D8E0000E94A9CF0E9479CF6093D6127093D7126D
:10D8F0008093D8129093D91286ED92E10C94EC7437
:10D9000060933F02709340028093410290934202E1
:10D910000895CF92DF92EF92FF920F931F93CF93D0
:10D92000DF9300D01F92CDB7DEB7FAE0CF2EF3E140
:10D93000DF2EAAE1EA2EA3E1FA2E0AED12E1F601AA
:10D9400061917191819191916F01F70121913191D3
:10D95000419151917F0129833A834B835C830E94DB
:10D9600074CD29813A814B815C810E94A9CF0E94AC
:10D9700048CDF80161937193819391938F01FAE1FE
:10D98000CF16F3E1DF06D9F60F900F900F900F90AE
:10D99000DF91CF911F910F91FF90EF90DF90CF908B
:10D9A000089580915313811109C080915213811100
:10D9B00005C080915113811101C00895E3ECF0E19D
:10D9C0008491882341F09091C00095FFFCCF809313
:10D9D000C6003196F5CFE4EBF8E08491882341F05E
:10D9E0009091C00095FFFCCF8093C6003196F5CF93
:10D9F000809153138823F1F0609154137091551363
:10DA000080915613909157130E9476CD20911A134E
:10DA100030911B1340911C1350911D130E94DBCCBD
:10DA2000AB01BC0180EB98E00E94461A80EA98E0C6
:10DA30000E94AE92809152138823F1F060915813A6
:10DA40007091591380915A1390915B130E9476CD77
:10DA500020911E1330911F134091201350912113D8
:10DA60000E94DBCCAB01BC018CE998E00E94461A15
:10DA70008CE898E00E94AE92809151138823F1F0D7
:10DA800060915C1370915D1380915E1390915F13B0
:10DA90000E9476CD209122133091231340912413BC
:10DAA000509125130E94DBCCAB01BC0188E898E0C3
:10DAB0000E94461A88E798E00E94AE928091C000CA
:10DAC00085FFFCCF8AE08093C6001092531310921A
:10DAD000521310925113089510925313109252132F
:10DAE000109251130895809353020895EFE6F0E0E9
:10DAF00080818260808308951F920F920FB60F92EB
:10DB000011240BB60F920F931F932F933F934F93B4
:10DB10005F936F937F938F939F93AF93BF93EF9395
:10DB2000FF938091841390918513892B09F086C10E
:10DB30009091E40D8091E30D981771F0E091E30D61
:10DB40008DE4E89FF0011124EB51F24FDF01A45B5B
:10DB5000BF4F81E08C9302C0E0E0F0E0F0938513CA
:10DB6000E0938413309709F463C1DF01A45BBF4FD6
:10DB700081E08C93109267131092681310926913CE
:10DB800010926A1360AD71AD61349CE9790728F495
:10DB900061329EE4790748F002C060E47CE9769542
:10DBA00067957695679584E007C0613197E27907BC
:10DBB00030F07695679582E08093641307C0809378
:10DBC00064136032710510F460E270E06052710914
:10DBD000611588E07807D0F0872F9927880F991F63
:10DBE000880F991F8D53934FFC01329645915491A4
:10DBF000AA27659F9001649F210D3A1F06942A1F52
:10DC00003A1F1124FC01859194911DC0CB0196957A
:10DC100087958C7F8D53974FFC01459154910296C7
:10DC2000FC0185919491FB01E770FF278E9F900185
:10DC30008F9F300D9E9F300D1124E3E03695279580
:10DC4000EA95E1F7CA01821B930B84369105A0F493
:10DC5000EDE5F4E08191882339F09091C00095FFC3
:10DC6000FCCF8093C600F6CF4AE050E082EE95E00C
:10DC70000E94251884E690E09093631380936213CA
:10DC800080916413992787FD9095909361138093F9
:10DC90006013E0918413F091851364AD75AD7093BA
:10DCA00066136093651361349CE9790728F4613247
:10DCB0008EE4780748F002C060E47CE976956795C9
:10DCC0007695679584E007C0613197E2790730F077
:10DCD0007695679582E08093641308C081E0809315
:10DCE00064136032710510F460E270E060527109F3
:10DCF000611588E07807E0F0872F9927880F991F32
:10DD0000880F991F8D53934FFC01329625913491C2
:10DD1000AA27639FA001629F410D5A1F06944A1FC4
:10DD20005A1F1124FC0125913491241B350B1EC070
:10DD3000CB01969587958C7F8D53974FFC0125914C
:10DD400034910296FC0145915491FB01E770FF2745
:10DD50004E9FC0014F9F900D5E9F900D1124F3E0E8
:10DD600096958795FA95E1F7281B390B24363105EE
:10DD7000A0F4EDE5F4E08191882339F09091C000A2
:10DD800095FFFCCF8093C600F6CF4AE050E082EECC
:10DD900095E00E94251824E630E0C901A0E0B0E03B
:10DDA00080936B1390936C13A0936D13B0936E13C9
:10DDB0003093890020938800E0918413F0918513BB
:10DDC00080899189A289B389B695A79597958795FA
:10DDD000B095A095909581959F4FAF4FBF4F809381
:10DDE0007F1390938013A0938113B0938213809339
:10DDF0007B1390937C13A0937D13B0937E13809339
:10DE0000771390937813A0937913B0937A13809338
:10DE1000731390937413A0937513B09376131092A9
:10DE20006F1310927013109271131092721306C038
:10DE300080ED97E09093890080938800E0918413AF
:10DE4000F0918513309709F4DCC480A1809383138B
:10DE500080FF41C0899A8FEF80934F0280915302D7
:10DE60008823E9F12CB131E025FB222720F9232773
:10DE700079F180915013882359F1E0918413F09146
:10DE8000851380819181A281B381181619061A0623
:10DE90001B06F4F480913E1390913F13A091401320
:10DEA000B09141138093541390935513A09356133C
:10DEB000B09357133093531380899189A289B38902
:10DEC00080936F1390937013A0937113B093721398
:10DED0002093501304C0899881E080934F02809171
:10DEE000831381FF41C08F9A8FEF809350028091FE
:10DEF00053028823E9F12091030131E02695217036
:10DF0000232779F180914F13882359F1E0918413ED
:10DF1000F091851384819581A681B7811816190621
:10DF20001A061B06F4F48091421390914313A091BA
:10DF30004413B09145138093581390935913A093B1
:10DF40005A13B0935B133093521380899189A2893D
:10DF5000B38980936F1390937013A0937113B09350
:10DF6000721320934F1304C08F9881E08093500266
:10DF7000809183139FB782FF48C0F89480910B0172
:10DF80008D7F80930B019FBF8FEF80935102809113
:10DF90005302882309F443C029B131E023FB22272F
:10DFA00020F9232779F180914E13882359F1E091CC
:10DFB0008413F091851380859185A285B385181609
:10DFC00019061A061B06F4F4809146139091471324
:10DFD000A0914813B091491380935C1390935D1303
:10DFE000A0935E13B0935F1330935113808991898E
:10DFF000A289B38980936F1390937013A0937113C8
:10E00000B093721320934E130AC0F89480910B01C1
:10E01000826080930B019FBF81E0809351028091C9
:10E020008313E0918413F091851383FF08C081A1CD
:10E03000813011F4439801C0169A8FEF07C081A177
:10E04000813011F4439A01C0169881E08093520206
:10E0500020E08091641328170CF0C7C18091C000A4
:10E0600087FF19C03091C600409163065091640645
:10E07000CA0101968F7799276091650670916606AF
:10E080008617970741F0FA01ED51FA4F30839093CC
:10E09000640680936306E0918413F0918513809168
:10E0A0007F1390918013A0918113B09182134081CE
:10E0B000518162817381840F951FA61FB71F8093C2
:10E0C0007F1390938013A0938113B093821318163B
:10E0D00019061A061B06CCF5889AE0918413F09174
:10E0E000851380917F1390918013A0918113B0913B
:10E0F00082134089518962897389841B950BA60B11
:10E10000B70B80937F1390938013A0938113B093E8
:10E11000821340914F0280913E1390913F13A09142
:10E120004013B0914113552747FD5095652F752F2A
:10E13000840F951FA61FB71F80933E1390933F1324
:10E14000A0934013B09341138898E0918413F09109
:10E15000851380917B1390917C13A0917D13B091D6
:10E160007E134481558166817781840F951FA61F98
:10E17000B71F80937B1390937C13A0937D13B09370
:10E180007E13181619061A061B06CCF58E9AE09116
:10E190008413F091851380917B1390917C13A0914F
:10E1A0007D13B0917E134089518962897389841BE4
:10E1B000950BA60BB70B80937B1390937C13A093C6
:10E1C0007D13B0937E134091500280914213909141
:10E1D0004313A0914413B0914513552747FD509523
:10E1E000652F752F840F951FA61FB71F80934213AD
:10E1F00090934313A0934413B09345138E98E091EA
:10E200008413F09185138091771390917813A091E6
:10E210007913B0917A134085518562857385840F97
:10E22000951FA61FB71F8093771390937813A09321
:10E230007913B0937A13181619061A061B060CF0F8
:10E2400047C09FB7F89480910B01886080930B01C1
:10E250009FBFE0918413F091851380917713909183
:10E260007813A0917913B0917A134089518962890A
:10E270007389841B950BA60BB70B80937713909330
:10E280007813A0937913B0937A134091510280913F
:10E29000461390914713A0914813B0914913552705
:10E2A00047FD5095652F752F840F951FA61FB71F2B
:10E2B0008093461390934713A0934813B093491348
:10E2C0009FB7F89480910B01877F80930B019FBFCC
:10E2D000E0918413F09185138091731390917413DE
:10E2E000A0917513B0917613448555856685778521
:10E2F000840F951FA61FB71F8093731390937413F9
:10E30000A0937513B0937613181619061A061B06F8
:10E310000CF043C081A1813011F4419A01C0149ADC
:10E32000E0918413F091851380917313909174138D
:10E33000A0917513B09176134089518962897389D0
:10E34000841B950BA60BB70B8093731390937413D8
:10E35000A0937513B09376134091520280914A13A3
:10E3600090914B13A0914C13B0914D13552747FD3D
:10E370005095652F752F840F951FA61FB71F80938B
:10E380004A1390934B13A0934C13B0934D1381A158
:10E39000813011F4419801C0149880916F139091CD
:10E3A0007013A0917113B09172130196A11DB11D4C
:10E3B00080936F1390937013A0937113B0937213A3
:10E3C00040916F135091701360917113709172139B
:10E3D000E0918413F091851380899189A289B38992
:10E3E000481759076A077B07B0F040916F135091A7
:10E3F00070136091711370917213E0918413F09116
:10E40000851384899589A689B78984179507A607F6
:10E41000B70718F4DAC02F5F1CCE40916B135091F0
:10E420006C1360916D1370916E13048D158D268D94
:10E43000378DAA27419FB12D529FC001629F900D39
:10E44000619F800D911D429FB00D811D9A1F519FAC
:10E45000B00D811D9A1F609FB00D811D9A1F509FA6
:10E46000B10D8A1F9A1FB6958A1F9A1F112444ADB9
:10E4700055AD480F591F509366134093651380ADF7
:10E4800091ADA2ADB3AD60E070E084179507A6072B
:10E49000B70720F49093661380936513609165131A
:10E4A0007091661361349CE9790728F461328EE437
:10E4B000780748F002C060E47CE976956795769528
:10E4C000679584E007C0613197E2790730F076956F
:10E4D000679582E08093641308C081E080936413A1
:10E4E0006032710510F460E270E0605271096115EC
:10E4F00088E07807E0F0872F9927880F991F880F09
:10E50000991F8D53934FFC01329625913491AA2780
:10E51000639FA001629F410D5A1F06944A1F5A1F14
:10E520001124FC0125913491241B350B1EC0CB0115
:10E53000969587958C7F8D53974FFC01259134914B
:10E540000296FC0145915491FB01E770FF274E9F15
:10E55000C0014F9F900D5E9F900D112413E0969582
:10E5600087951A95E1F7281B390B24363105A0F45D
:10E57000EDE5F4E08191882339F09091C00095FF9A
:10E58000FCCF8093C600F6CF4AE050E082EE95E0E3
:10E590000E94251824E630E03093890020938800FB
:10E5A00080916B1390916C13A0916D13B0916E13C9
:10E5B000820F931FA11DB11D80936B1390936C1359
:10E5C000A0936D13B0936E13F7C040916F135091E9
:10E5D00070136091711370917213808D918DA28D63
:10E5E000B38D84179507A607B70708F0D9C04091E7
:10E5F0006713509168136091691370916A13048DC9
:10E60000158D268D378DAA27419FB12D529FC001B0
:10E61000629F900D619F800D911D429FB00D811DE5
:10E620009A1F519FB00D811D9A1F609FB00D811DD3
:10E630009A1F509FB10D8A1F9A1FB6958A1F9A1F65
:10E6400011242091651330916613E05CFF4F281769
:10E65000390718F42081318102C0281B390B8081D1
:10E660009181A281B381A90160E070E04817590748
:10E670006A077B0708F49C0121349CE9390728F4D8
:10E6800021328EE4380748F002C020E43CE9369598
:10E6900027953695279584E007C0213197E2390701
:10E6A00030F03695279582E08093641308C081E0AE
:10E6B000809364132032310510F420E230E0B90178
:10E6C00060527109611588E07807E0F0872F99277B
:10E6D000880F991F880F991F8D53934FFC01329615
:10E6E00025913491AA27639FA001629F410D5A1F73
:10E6F00006944A1F5A1F1124FC0125913491241BB2
:10E70000350B1EC0CB01969587958C7F8D53974F07
:10E71000FC01259134910296FC0145915491FB0135
:10E72000E770FF274E9FC0014F9F900D5E9F900D99
:10E73000112443E0969587954A95E1F7281B390BFC
:10E7400024363105A0F4EDE5F4E08191882339F019
:10E750009091C00095FFFCCF8093C600F6CF4AE0B1
:10E7600050E082EE95E00E94251824E630E03093D8
:10E770008900209388008091671390916813A0917D
:10E780006913B0916A13820F931FA11DB11D80936D
:10E79000671390936813A0936913B0936A130CC026
:10E7A0008091621390916313909389008093880005
:10E7B000809160138093641340916F135091701394
:10E7C0006091711370917213E0918413F09185132D
:10E7D00080899189A289B389481759076A077B07FD
:10E7E00080F010928513109284139091E40D809123
:10E7F000E30D981731F08091E30D8F5F8F70809358
:10E80000E30DFF91EF91BF91AF919F918F917F9118
:10E810006F915F914F913F912F911F910F910F90A9
:10E820000BBE0F900FBE0F901F901895819A879A7C
:10E83000EAE0F1E08081826080830E9A3B9A579AE9
:10E840005F9A829A8A9AE7E0F1E080818160808312
:10E850009FB7F894E8E0F1E08081816080839FBFFA
:10E860000A9A129A3F9A479A6C98749AE4E0F1E0F7
:10E8700080818E7F80839FB7F894E5E0F1E080810E
:10E88000816080839FBF6D98759AE4E0F1E080819C
:10E890008D7F80839FB7F894E5E0F1E0808182600E
:10E8A00080839FBF53985B9A809A88985F9A869AD4
:10E8B0008E988A9AEAE0F1E08081886080839FB731
:10E8C000F894EBE0F1E08081877F80839FBF9FB762
:10E8D000F894E8E0F1E08081816080839FBF0C9A2A
:10E8E0001498129A399A4198479AA1E8B0E08C910D
:10E8F0008F7E8C938C9188608C93E0E8F0E080812F
:10E900008D7F808380818E7F808380818F738083E1
:10E9100080818F7C80838C91887F82608C9380E063
:10E9200090E4909389008093880010928500109263
:10E930008400EFE6F0E080818260808381E0809354
:10E940005302789408959091E40D8091E30D981707
:10E9500031F060D20E94031F0E94F193F4CF08951A
:10E96000CF93DF93EFB7F894EC0188819981AA8166
:10E97000BB8180933E1390933F13A0934013B093B9
:10E980004113EB0188819981AA81BB818093421355
:10E9900090934313A0934413B0934513EA018881E5
:10E9A0009981AA81BB818093461390934713A093CA
:10E9B0004813B0934913E90188819981AA81BB81E9
:10E9C00080934A1390934B13A0934C13B0934D1321
:10E9D000EFBFDF91CF9108952FB7F894FC018081AC
:10E9E0009181A281B38180934A1390934B13A0939A
:10E9F0004C13B0934D132FBF08952FB7F89494E0A4
:10EA0000899FF0011124E25CFC4E6081718182815A
:10EA100093812FBF089597DF5F9A8A9A9FB7F894E2
:10EA2000E8E0F1E08081816080839FBF129A479A7D
:10EA3000089580916F008D7F80936F009091E40D19
:10EA40008091E30D981314C08091A40A882341F0AB
:10EA500061E070E085EA9AE00E940D26892BA9F01A
:10EA600080916F00826080936F0010926C0908950E
:10EA70009091E40D8091E30D981701F38091E30DDF
:10EA80008F5F8F708093E30DD9CF10928513109212
:10EA90008413E6CF80916F008D7F80936F009091FB
:10EAA000E40D8091E30D981306C080916F008260A1
:10EAB00080936F0008959091E40D8091E30D981775
:10EAC00071F38091E30D8F5F8F708093E30DE7CF3B
:10EAD0002F923F924F925F926F927F928F929F926E
:10EAE000AF92BF92CF92DF92EF92FF920F931F935C
:10EAF000CF93DF9300D000D0CDB7DEB78C01F62ED8
:10EB000021E0261760F5E3EDF1E18491882341F0DF
:10EB10009091C00095FFFCCF8093C6003196F5CF51
:10EB20008F2D90E04AE050E0BC0182EE95E00E941B
:10EB3000E817E9ECF0E18491882341F09091C0005E
:10EB400095FFFCCF8093C6003196F5CF8091C00031
:10EB500085FFFCCF8AE08093C6000E94CA1E6F2DFD
:10EB600070E0FB01EE0FFF1FE155FB4F408151812B
:10EB70005E834D83452B09F4A6C0FB01E355FB4F93
:10EB800050815A832D813E812C5F3F4F81E090E080
:10EB900089836A81861708F07BC0DC01F901459101
:10EBA00054910196B9016C5F7F4F041715070CF063
:10EBB0006DC00297AC01440F551F440F551F4E5FA7
:10EBC0005F4F6D817E81460F571FFA0165917491E9
:10EBD000880F991F880F991FED81FE818E0F9F1F4F
:10EBE000FC01A590B490FD01EE0FFF1FEE0FFF1F7B
:10EBF0003296AD81BE81EA0FFB1FC590D490FA0119
:10EC0000E590F490F90125903490FC012591349120
:10EC10003C832B83882777FD8095982F0E9476CDA3
:10EC20002B013C01B8016A197B09882777FD809583
:10EC3000982F0E9476CD4B015C01B6016E197F09B9
:10EC4000882777FD8095982F0E9476CD9B01AC0197
:10EC5000C501B4010E94A9CF6B017C01B1014B81B8
:10EC60005C81641B750B882777FD8095982F0E9427
:10EC700076CD9B01AC01C701B6010E94DBCC9B01A4
:10EC8000AC01C301B2010E94FBCB06C09B0180CF47
:10EC900060E070E080E090E0A981BA81AB132BC006
:10ECA0002D813E81E4E0AE9F200D311D11242250C4
:10ECB0003109F90165917491882777FD8095982F26
:10ECC0000E9476CD18C0B801882777FD8095982FCF
:10ECD0000E9476CD20E030E04AEF5EE30E94A9CFAB
:10ECE00020E030E040E85DE30E94A9CF20E030E082
:10ECF000A9010E94FBCB26960FB6F894DEBF0FBE8B
:10ED0000CDBFDF91CF911F910F91FF90EF90DF90DA
:10ED1000CF90BF90AF909F908F907F906F905F90BB
:10ED20004F903F902F9008958091FB139091FC138A
:10ED30009093BC098093BB092091AD0920FD09C0C7
:10ED40001092F3131092F4131092F5131092F6131D
:10ED50000AC060E0BDDE6093F3137093F4138093F8
:10ED6000F5139093F6138091FD139091FE139093F9
:10ED7000BE098093BD092091AD0921FF0BC061E060
:10ED8000A7DE6093F7137093F8138093F9139093B1
:10ED9000FA1308C01092F7131092F8131092F91397
:10EDA0001092FA131092ED131092EE131092EF13CB
:10EDB0001092F0138FB7F8941092EC138FBF089550
:10EDC000209165023091660240916702509168027D
:10EDD00060E070E08FE793E40E94DBCC6093AC13BB
:10EDE0007093AD138093AE139093AF136093B013F1
:10EDF0007093B1138093B2139093B313089597FF58
:10EE000003C08091A31304C0FC01EC55FC4E80812B
:10EE100090E008952F923F924F925F926F927F926F
:10EE20008F929F92AF92BF92CF92DF92EF92FF921A
:10EE30000F931F93CF93DF93CDB7DEB7A2970FB693
:10EE4000F894DEBF0FBECDBF8091EC13882309F488
:10EE5000D2C16ADF8091690290916A02A0916B022F
:10EE6000B0916C028D8B9E8BAF8BB88F80916502B9
:10EE700090916602A0916702B0916802898F9A8F83
:10EE8000AB8FBC8F8091610290916202A09163026E
:10EE9000B09164028D8F9E8FAF8FB8A3A3EFB3E1C3
:10EEA000BA8BA98BE1E0F4E1F88BEF878CEB93E16F
:10EEB0009A878987A4EAB3E1BA83A983E5E5F2E0FA
:10EEC000F887EF838BE993E19C8B8B8B0AEA13E144
:10EED00044EE242E43E1342EACEDB3E1BC83AB838E
:10EEE000E4ECF3E1FE83ED831AA219A2A989BA89A1
:10EEF0008D909D90AD90BD90BA8BA98BEF85F889D0
:10EF000061907190F88BEF87B301882777FD80952A
:10EF1000982F0E9476CDA50194010E94FACB6B0137
:10EF20007C01A985BA856D937D938D939D93BA8756
:10EF3000A98720E030E040E251E40E94D7CE1816C5
:10EF400024F421E0F8012083D6C020E030E040E244
:10EF500051ECC701B6010E94D4CC87FD02C06728DE
:10EF600021F4E1E0D801EC93CDC0D8018C91882345
:10EF700031F0F10110821182128213821C92A701DA
:10EF800096016D897E898F89988D0E94A9CF6B87A4
:10EF90007C878D879E87E9A1FAA1EC52FC4E6083A5
:10EFA000718382839383D1012D913D914D915C9129
:10EFB000C701B6010E94FBCB6B017C01E9A1FAA15C
:10EFC000EC54FC4E5080618072804380252D362D9C
:10EFD000472D542D0E94D4CC87FD16C0E9A1FAA17B
:10EFE000E455FC4E5080618072804380252D362D83
:10EFF000472D542DB601C7010E94D7CE181624F014
:10F000005C2C6D2C7E2C4F2C852D962DA72DB42D90
:10F01000F10180839183A283B383252D362D472D63
:10F02000542D698D7A8D8B8D9C8D0E94A9CF2B01DB
:10F030003C01E9A1FAA1E453FC4E60837183828311
:10F040009383AB81BC812D913D914D915C91C50124
:10F05000B4010E94FACB9B01AC016D8D7E8D8F8D2A
:10F0600098A10E94A9CF20ED3CEC4CE45DE30E9406
:10F07000A9CF6B017C0123E333E343E75FE3ED8139
:10F08000FE8160817181828193810E94A9CF9B0161
:10F09000AC01C701B6010E94FBCB6B017C01AD81C5
:10F0A000BE816D937D938D939C931397EB81FC812F
:10F0B00080829182A282B382A30192016B857C85BA
:10F0C0008D859E850E94FBCBA70196010E94FACBFD
:10F0D0006B017C0120E030E0A9010E94D4CC87FDC7
:10F0E00011C020E030E040E853E4C701B6010E94BF
:10F0F000D7CE181654F4C12CD12C30E8E32E33E4CB
:10F10000F32E03C0C12CD12C7601AB89BC898D9123
:10F110009D91BC8BAB8BBC01882777FD8095982F88
:10F120000E9476CD9B01AC01C501B4010E94D7CEEF
:10F130001816F4F4EF81F88580819181BC0188274D
:10F1400077FD8095982F0E9476CD9B01AC01C5017B
:10F15000B4010E94D4CC87FF0BC0C701B6010E9446
:10F1600043CDCB0195958795A981BA818C9303C036
:10F17000E981FA81108289A19AA104969AA389A3B0
:10F18000A981BA811196BA83A983EF81F885329655
:10F19000F887EF830F5F1F4FF4E02F0E311C8B8138
:10F1A0009C8104969C838B83AD81BE811496BE8323
:10F1B000AD83E9A1FAA1389709F098CE0E94C4C5A1
:10F1C0000091A6131091A7132091A8133091A913B1
:10F1D000601B710B820B930B68387341810591059D
:10F1E00050F00E94C4C56093A6137093A713809338
:10F1F000A8139093A913A2960FB6F894DEBF0FBE82
:10F20000CDBFDF91CF911F910F91FF90EF90DF90D5
:10F21000CF90BF90AF909F908F907F906F905F90B6
:10F220004F903F902F900895CF93DF93C091550258
:10F23000D09156021092B4131092B5131092B613D7
:10F240001092B713209165023091660240916702D7
:10F250005091680260E070E08FE793E40E94DBCC9D
:10F260006093AC137093AD138093AE139093AF1370
:10F27000D0935802C09357021092B8131092B9134A
:10F280001092BA131092BB136093B0137093B11322
:10F290008093B2139093B313249A809101018061FB
:10F2A000809301018091010180628093010180912E
:10F2B000010180648093010187ED80937A001092B0
:10F2C0007E0010927D0080917D00806280937D00A1
:10F2D00080917D00806880937D0080917D008064B6
:10F2E00080937D0080E888BD80916E00846080936B
:10F2F0006E006AEF70E080E090E00E94F3C585E068
:10F3000090E090939C1380939B1360E0809159024E
:10F3100090915A02DDDB20E030E040EA50E40E94A8
:10F32000D4CC87FF0AC08091590290915A0240972D
:10F3300090935A0280935902E8CF84E591E090932C
:10F3400056028093550260E080919F139091A01324
:10F35000BFDB20E030E04AEA53E40E94D7CE181623
:10F3600054F480919F139091A01340969093A01312
:10F3700080939F13E8CF85E090E090939E13809355
:10F380009D1361E080915B0290915C02A1DB20E023
:10F3900030E040EA50E40E94D4CC87FF0AC080915C
:10F3A0005B0290915C02409790935C0280935B02B9
:10F3B000E8CF84E591E0909358028093570261E092
:10F3C0008091A1139091A21383DB20E030E04AEA00
:10F3D00053E40E94D7CE181654F48091A113909153
:10F3E000A21340969093A2138093A113E8CFDF91CC
:10F3F000CF91089508951092021410920114E3E041
:10F40000F4E111821082109200141092FF131092F6
:10F41000A4132C981092A5139FB7F894E2E0F1E0A2
:10F4200080818F7E80839FBF109200141092FF1303
:10F430001092A3139FB7F89480818F7D80839FBF24
:10F4400008952F923F924F925F926F927F928F9288
:10F450009F92AF92BF92CF92DF92EF92FF920F9363
:10F460001F93CF93DF93CDB7DEB7AE970FB6F89467
:10F47000DEBF0FBECDBF6C8F7D8F8E8F9F8F5EA73F
:10F480004DA73CA72BA70E94C4C569A37AA38BA351
:10F490009CA32DA53EA5233031051CF4E0E7F4E044
:10F4A00017C0E3E8F4E08191882339F09091C0001F
:10F4B00095FFFCCF8093C600F6CF8091C00085FFFA
:10F4C000FCCF15C29091C00095FFFCCF8093C60081
:10F4D00081918111F7CF8091C00085FFFCCF8AE038
:10F4E0008093C60088DF4DA55EA580E857FF43C026
:10F4F0008093A31389A19AA1ABA1BCA1898B9A8BFC
:10F50000AB8BBC8B8D879E87AF87B88B1D8290E4B9
:10F51000998FACE1AA8FB6E4BB8F1D8A1E8A1F8A21
:10F52000188E20E830E040E050E029833A834B8396
:10F530005C83F0E84F2E512C612C712C1DA21EA271
:10F540001FA218A631E038A31C861B86312C00E0D0
:10F5500010E0212C4DA55EA54C555C4E5AA749A73D
:10F560008DA59EA5880F991F880F991F8D509C4EC1
:10F570009A87898708C0EDA5FEA5EC55FC4E8083CF
:10F58000B9CF0E94F1938091EC13882309F4DCC079
:10F59000CBDBADA5BEA5B7FF09C03090ED13009140
:10F5A000EE131091EF132090F01306C0E985FA8551
:10F5B0003080018112812380232D302F412F522D45
:10F5C0006D897E898F89988D0E94D7CE181624F078
:10F5D0003D8A0E8B1F8B288E232D302F412F522DCD
:10F5E0006D81798D8A8D9B8D0E94D4CC87FD04C05E
:10F5F0003D82098F1A8F2B8EF8A1FF2309F451C089
:10F600002C8D3D8D4E8D5F8D632D702F812F922D12
:10F610000E94D7CE18160CF097C00E94C4C5298945
:10F620003A894B895C89621B730B840B950B693893
:10F6300073418105910508F487C0D301C201298176
:10F640003A814B815C81821B930BA40BB50B4DA5BA
:10F650005EA5B595A7959795879557FF03C08093AD
:10F66000A31303C0E9A5FAA580830E94C4C56D87D2
:10F670007E878F87988B9B01AC0189899A89AB899A
:10F68000BC89281B390B4A0B5B0B2DA33EA34FA350
:10F6900058A79C8D9D8BAD8DAE8BBE8DBF8BEF8D96
:10F6A000E88F2C8D3D8D4E8D5F8D632D702F812FBA
:10F6B000922D0E94D4CC87FFF0C20E94C4C52D8534
:10F6C0003E854F855889621B730B840B950B6938F7
:10F6D00073418105910508F4E0C20E94C4C5698B9D
:10F6E0007A8B8B8B9C8BDC01CB012D853E854F85E6
:10F6F0005889821B930BA40BB50B4B855C85452B5E
:10F7000009F011C189819A81AB81BC81840D951D5D
:10F71000A61DB71D2DA53EA5B595A79597958795CF
:10F7200037FFB7C28093A3132B853C852F5F3F4FD4
:10F730003C872B873C8D3D834D8D498F5E8D5A8F45
:10F740008F8D8B8F91E098A320E030E040EA51E468
:10F750006C8D7D8D8E8D9F8D0E94FBCB9B01AC01AE
:10F76000632D702F812F922D0E94D7CE181694F4FE
:10F77000E4E6F1E18491882341F09091C00095FF87
:10F78000FCCF8093C6003196F5CF8091C00085FFF5
:10F79000FCCFADC00E94C4C529A13AA14BA15CA178
:10F7A000621B730B840B950B613D774081059105BE
:10F7B00008F450C04DA55EA557FF10C0E090A313FC
:10F7C000F12CEEE5F1E184918823C9F09091C0001D
:10F7D00095FFFCCF8093C6003196F5CFA9A5BAA5B9
:10F7E000EC90F12CE8E5F1E18491882341F09091CF
:10F7F000C00095FFFCCF8093C6003196F5CF22E084
:10F8000030E0432D502F612F722D82EE95E00E9443
:10F81000BE18E4E5F1E18491882341F09091C000A5
:10F8200095FFFCCF8093C6003196F5CF4AE050E0BB
:10F83000B70182EE95E00E94E8178091C00085FF35
:10F84000FCCF8AE08093C6000E94C4C569A37AA356
:10F850008BA39CA30E94C4C56B017C010E94C4C5FC
:10F8600089889A88AB88BC882D853E854F855889C4
:10F87000820E931EA41EB51EC818D908EA08FB08FC
:10F88000C60ED71EE81EF91E31E8C3163FE4D306A4
:10F8900032E1E306F10490F0E7E3F1E1849188239B
:10F8A00041F09091C00095FFFCCF8093C600319647
:10F8B000F5CF8091C00085FFFCCF19C04B855C85DA
:10F8C0008BA59CA5841795070CF05BCEE6EEF0E1C6
:10F8D0008491882341F09091C00095FFFCCF8093E4
:10F8E000C6003196F5CF8091C00085FFFCCF8AE03D
:10F8F0008093C600AE960FB6F894DEBF0FBECDBFA4
:10F90000DF91CF911F910F91FF90EF90DF90CF90FB
:10F91000BF90AF909F908F907F906F905F904F902F
:10F920003F902F9008958DA09EA0AFA0B8A4880E00
:10F93000991EAA1EBB1E2DA13EA14FA158A5281B92
:10F94000390B4A0B5B0BCA01B90129813A814B8102
:10F950005C810E946FD0A50194010E94C7D0240D44
:10F96000351D461D571D243131054105510504F152
:10F9700029013A013DEE43165104610471042CF053
:10F980007CEE472E512C612C712C41E84416510419
:10F9900061047104DCF08FEF90E0A0E0B0E0841926
:10F9A0009509A609B70989839A83AB83BC8312C0E2
:10F9B00064E1462E512C612C712C24E130E040E0B2
:10F9C00050E029833A834B835C8304C049825A8286
:10F9D0006B827C82EBECF1E18491882341F0909181
:10F9E000C00095FFFCCF8093C6003196F5CF2AE08A
:10F9F00030E0B301A20182EE95E00E94C517E6EC6B
:10FA0000F1E18491882341F09091C00095FFFCCFF3
:10FA10008093C6003196F5CF2AE030E049815A81C3
:10FA20006B817C8182EE95E00E94C517EFEBF1E1DE
:10FA30008491882341F09091C00095FFFCCF809382
:10FA4000C6003196F5CF22E030E04D81598D6A8DA8
:10FA50007B8D82EE95E00E94BE18E8EBF1E1849187
:10FA6000882341F09091C00095FFFCCF8093C600A1
:10FA70003196F5CF22E030E04D895E896F89788D2F
:10FA800082EE95E00E94BE188091C00085FFFCCFF9
:10FA90008AE08093C6002B853C85233031050CF429
:10FAA00031CE69817A818B819C810E9476CD20E064
:10FAB00030E040E850E40E94A9CF6B017C012D8129
:10FAC000398D4A8D5B8D6D897E898F89988D0E94D5
:10FAD000FACB20ED3FE049E450E40E94A9CF20E0BA
:10FAE00030E040E05FE30E94A9CF9B01AC01C70179
:10FAF000B6010E94DBCC6B017C01C501B4010E9400
:10FB000076CD20E030E04AE754E40E94DBCC4B01A4
:10FB10005C01E2EBF1E18491882341F09091C00017
:10FB200095FFFCCF8093C6003196F5CF22E030E000
:10FB3000B701A60182EE95E00E94BE18ECEAF1E161
:10FB40008491882341F09091C00095FFFCCF809371
:10FB5000C6003196F5CF22E030E0B501A40182EE77
:10FB600095E00E94BE188091C00085FFFCCF8AE01E
:10FB70008093C6002AE939E949E15FE3C701B6018C
:10FB80000E94A9CF6B017C019B01AC010E94FBCBC1
:10FB9000A50194010E94DBCC6D837E838F839887BF
:10FBA000A5019401C701B6010E94A9CF20E030E071
:10FBB00040E05EE30E94A9CF4B015C01EFE9F1E177
:10FBC0008491882341F09091C00095FFFCCF8093F1
:10FBD000C6003196F5CF8091C00085FFFCCF8AE04A
:10FBE0008093C600E9E9F1E18491882341F0909186
:10FBF000C00095FFFCCF8093C6003196F5CF22E080
:10FC000030E0B701A60182EE95E00E94BE18809117
:10FC1000C00085FFFCCF8AE08093C600E3E9F1E1F4
:10FC20008491882341F09091C00095FFFCCF809390
:10FC3000C6003196F5CF22E030E04D815E816F81C4
:10FC4000788582EE95E00E94BE188091C00085FF05
:10FC5000FCCF8AE08093C600EDE8F1E1849188232F
:10FC600041F09091C00095FFFCCF8093C600319683
:10FC7000F5CF22E030E0B501A40182EE95E00E94CC
:10FC8000BE188091C00085FFFCCF8AE08093C6003B
:10FC900039CDE9A5FAA5808347CD18A255CD1F928D
:10FCA0000F920FB60F9211240BB60F922F933F9322
:10FCB0004F935F936F937F938F939F93AF93BF9374
:10FCC000EF93FF9380915402811127C08091A41378
:10FCD00080939A13882329F08091AC098D3009F420
:10FCE0002C9A8091A51380939913882341F09FB794
:10FCF000F894809102018061809302019FBF8091FE
:10FD0000A31380939813882341F09FB7F8948091B0
:10FD100002018062809302019FBF90919A138091AB
:10FD20005402891728F08091AC098D3009F42C9881
:10FD30009091991380915402891740F09FB7F894DD
:10FD4000809102018F7E809302019FBF9091981352
:10FD500080915402891740F09FB7F8948091020176
:10FD60008F7D809302019FBF809154028F5F8F77B8
:10FD7000809354028091971390E08830910508F0A9
:10FD80008DC0FC01EE58FF4F0C94E3D088E08093C7
:10FD90007B0085E480937C0080917A00806480936E
:10FDA0007A000E94729381E019C02091780030910E
:10FDB00079008091931390919413A0919513B09131
:10FDC0009613820F931FA11DB11D809393139093DF
:10FDD0009413A0939513B093961382E08093971396
:10FDE0005DC088E080937B0086E480937C008091F6
:10FDF0007A00806480937A000E94729383E0EECF51
:10FE0000209178003091790080918F139091901318
:10FE1000A0919113B0919213820F931FA11DB11D58
:10FE200080938F1390939013A0939113B093921398
:10FE300084E0D4CF88E080937B0087E480937C00CB
:10FE400080917A00806480937A000E94729385E0AA
:10FE5000C5CF209178003091790080918B139091DB
:10FE60008C13A0918D13B0918E13820F931FA11D3F
:10FE7000B11D80938B1390938C13A0938D13B0932B
:10FE80008E1386E0ABCF0E94729387E0A7CF1092CB
:10FE9000971380918A138F5F80938A1380918A13BE
:10FEA000803108F484C08091EC13811118C08091D6
:10FEB0009313909194139093FC138093FB13809170
:10FEC0008B1390918C139093FE138093FD1380916C
:10FED0008F13909190139093F2138093F11381E01C
:10FEE0008093EC1310928A13109293131092941330
:10FEF000109295131092961310928B1310928C13EC
:10FF000010928D1310928E131092861310928713F5
:10FF1000109288131092891310928F1310929013DD
:10FF200010929113109292138091FB139091FC13F5
:10FF300020919F133091A0134091AD0928173907E4
:10FF400014F0427001C041604093AD092091590204
:10FF500030915A024091AD098217930714F0427014
:10FF600001C041604093AD098091FD139091FE1353
:10FF70002091A1133091A2134091AD0928173907A0
:10FF800014F0417001C042604093AD0920915B02C2
:10FF900030915C024091AD098217930714F04170D3
:10FFA00001C042604093AD0981E08093B309FF91A5
:10FFB000EF91BF91AF919F918F917F916F915F91E1
:10FFC0004F913F912F910F900BBE0F900FBE0F904E
:10FFD0001F9018952DEB37E346E05EE30C94A9CF14
:10FFE0002DEB37E346E05EE30C94DBCC2DEB37E3FF
:10FFF00046E05EE30C94DBCC2DEB37E346E05EE3BA
:020000021000EC
:100000000C94A9CF10922B1410922C1410922D1432
:1000100010922E1483EC93EB90936F0280936E02F8
:100020000895109202141092011410920414109268
:100030000314109200141092FF13E4CF10922B14AB
:1000400010922C1410922D1410922E1480EE9BE816
:1000500090936F0280936E0282E080936D02089508
:10006000FB0160916E0270916F0270932414609393
:10007000231460912B1470912C14709322146093AC
:10008000211462E060936D026EE170EB70936F0279
:1000900060936E029093201480931F14F0931E14AB
:1000A000E0931D14662757FD6095762F4093191431
:1000B00050931A1460931B1470931C14C901AA273F
:1000C00097FDA095BA2F8093151490931614A093C2
:1000D0001714B093181480819181AA2797FDA095D9
:1000E000BA2F80932B1490932C14A0932D14B093BB
:1000F0002E1408958F929F92AF92BF92CF92DF926B
:10010000EF92FF920F931F93CF93DF93EB0149017F
:100110005A016701780120916E0230916F0230938D
:1001200024142093231420912B1430912C143093F9
:1001300022142093211422E020936D0226E43AE950
:1001400030936F0220936E029093201480931F14BB
:1001500070931E1460931D1420E030E040E251E4DF
:10016000C501B4010E94A9CF0E9443CD6093191428
:1001700070931A1480931B1490931C1420E030E0A9
:1001800040E251E4C701B6010E94A9CF0E9443CDCD
:100190006093151470931614809317149093181489
:1001A00020E030E040E251E4688179818A819B81DE
:1001B0000E94A9CF0E9443CD60932B1470932C14FE
:1001C00080932D1490932E14DF91CF911F910F9156
:1001D000FF90EF90DF90CF90BF90AF909F908F9067
:1001E0000895CF93DF93262FFC01EB5BFF4F4081F7
:1001F0005181EC01CD5BDF4F6881798104960E94CB
:1002000017C128813981280F311D87FD3A9539831F
:10021000288381E090E0DF91CF91089581E090E024
:1002200090937B1480937A1484E190E090937D14F2
:1002300080937C1480916C09853019F463EB74E031
:1002400004C0873031F46EEB74E087E394E10E94E0
:1002500050C881E090E090937B1480937A148BE2F5
:1002600090E090937D1480937C1469EC74E087E3B4
:1002700094E10C9450C8CF93DF93FC016491EC019E
:100280002196662331F087E394E10E9451C8CE01A4
:10029000F4CFDF91CF910895EF92FF920F931F93C8
:1002A000CF93DF93EB017901E82FF0E031968CE0FA
:1002B0008E9F80018F9F100D112410927B1410923D
:1002C0007A1410937D1400937C14642F87E394E1D7
:1002D0000E9451C8FE016491662331F087E394E1E6
:1002E0000E9451C82196F6CF6AE387E394E10E9409
:1002F00051C88DE590E090937B1480937A1410930D
:100300007D1400937C14C701DF91CF911F910F9151
:10031000FF90EF90B0CFEF92FF920F931F93CF9388
:10032000DF93EB01790190E001962CE0289F80019A
:10033000299F100D112410927B1410927A1410939F
:100340007D1400937C14642F87E394E10E9451C8CC
:10035000FE016491662331F087E394E10E9451C865
:100360002196F6CF6AE387E394E10E9451C88DE5B8
:1003700090E090937B1480937A1410937D140093F3
:100380007C14B70187E394E1DF91CF911F910F9126
:10039000FF90EF900C9450C88091CB0A91E0892790
:1003A0008093CB0A882319F085E597E102C081E5A7
:1003B00097E10C94E71AAF92BF92CF92DF92EF923F
:1003C000FF920F931F93CF93DF931F92CDB7DEB7AA
:1003D0008CE6A82E89E0B82E87E0F501808380E0C6
:1003E00090E0A0E0B0E480935E0990935F09A09351
:1003F0006009B0936109198220E030E040EA50E4DE
:1004000060913702709138028091390290913A02DE
:100410000E94DBCC9E012F5F3F4F69017B018C0165
:1004200022E639E04EE559E06AE579E086E599E0B3
:100430000E94F361F501108284E99BE990936F02B9
:1004400080936E0282E080936D0210922B141092C2
:100450002C1410922D1410922E148DE993E10E9409
:10046000E71A0F90DF91CF911F910F91FF90EF90BE
:10047000DF90CF90BF90AF90089585E080936C0996
:1004800010928109109282098CE699E00E942A213B
:10049000B9DD89EA96E10C94E71A8CE699E00E94AE
:1004A0001C200C94EF12DF92EF92FF920F931F9398
:1004B000CF93DF93D82FF62ED72EC42FE22E61E0F4
:1004C0008BE394E14E3311F04632A9F40E94FDC251
:1004D0008CE0D89FA00111244D5F5F4F0CE010E02D
:1004E00020E830E060E070E08BE394E10E9454C5C6
:1004F00060E08BE394E10E94FDC210927B141092A5
:100500007A148D2F90E001962CE0289FF001299F0E
:10051000F00D1124F0937D14E0937C14CE3311F090
:100520006C2F01C060E287E394E10E9451C8CF2D97
:10053000DD2D11E11F0D912F9C1BFE01649166239F
:1005400031F087E394E10E9451C82196F4CFC92F7E
:10055000CC2339F060E287E394E10E9451C8C15096
:10056000F7CF6E2D87E394E10E9451C860E287E3E4
:1005700094E10E9451C861E08BE394E1DF91CF9157
:100580001F910F91FF90EF90DF900C94FDC2CF92DE
:10059000DF92EF92FF920F931F93CF93DF931F92FF
:1005A000CDB7DEB78CE699E00E941F21E09181096A
:1005B00028E0E29FF0011124E459F64F8789908DDD
:1005C000A18DB28D8093560990935709A093580935
:1005D000B0935909838D948DA58DB68D80935A095A
:1005E00090935B09A0935C09B0935D09198220E0A8
:1005F00030E040E752E460912F0270913002809128
:100600003102909132020E94DBCC20E030E040EADF
:1006100051E40E94FBCB9E012F5F3F4F69017B019C
:100620008C0122E639E04EE559E06AE579E086E59D
:1006300099E00E94F3610E94A37410925E091092E7
:100640005F091092600910926109198220E030E080
:1006500040E251E460913702709138028091390292
:1006600090913A020E94DBCC7B018C0122E639E0BA
:100670004EE559E06AE579E086E599E00E94F3618C
:100680000E94A3740F90DF91CF911F910F91FF9063
:10069000EF90DF90CF900895CF92DF92EF92FF928C
:1006A0000F931F93CF93DF931F92CDB7DEB787E0F1
:1006B00080936C0980E090E0A0E0B0E480935E0954
:1006C00090935F09A0936009B0936109198220E0BB
:1006D00030E040EA50E46091370270913802809136
:1006E000390290913A020E94DBCC9E012F5F3F4F6E
:1006F00069017B018C0122E639E04EE559E06AE5AB
:1007000079E086E599E00E94F3617CDC80918109C3
:10071000815080938109813039F48091820982303F
:1007200040F41092820905C0811103C084E08093D7
:1007300081092DDF0F90DF91CF911F910F91FF90D5
:10074000EF90DF90CF900895CF92DF92EF92FF92DB
:100750000F931F93CF93DF931F92CDB7DEB787E040
:1007600080936C0980E090E0A0E0B0E480935E09A3
:1007700090935F09A0936009B0936109198220E00A
:1007800030E040EA50E46091370270913802809185
:10079000390290913A020E94DBCC9E012F5F3F4FBD
:1007A00069017B018C0122E639E04EE559E06AE5FA
:1007B00079E086E599E00E94F36124DC809181096B
:1007C0008F5F80938109853031F484E080938209C2
:1007D00081E080938109DBDE0F90DF91CF911F9143
:1007E0000F91FF90EF90DF90CF900895CF9382E02C
:1007F00080936D020E94C4C56C507E4F8F4F9F4FF7
:1008000060933114709332148093331490933414A2
:10081000389ACAE0409A63E070E080E090E00E947D
:10082000F3C5409863E070E080E090E00E94F3C57B
:10083000C15081F7CF91089510922B1410922C146F
:1008400010922D1410922E148FE69BE890936F0255
:1008500080936E02CBCFCF92DF92EF92FF920F93F5
:100860001F93CF93DF9380912B1490912C14A09120
:100870002D14B0912E1481309048A105B10544F09B
:1008800010922B1410922C1410922D1410922E14DE
:1008900080912B1490912C14A0912D14B0912E14B2
:1008A000B7FF08C010922B1410922C1410922D1424
:1008B00010922E1460912B1470912C1480912D1491
:1008C00090912E1425E030E040E050E00E94C7D027
:1008D0008091351490E0A0E0B0E0281739074A076E
:1008E0005B0714F420933514D0913514C0E095E0E3
:1008F000C92ED12CE12CF12C11E060912B147091B8
:100900002C1480912D1490912E14D1113FC0209160
:100910006D02222389F0A70196010E94C7D0232BE4
:10092000242B252B19F426E246E202C026E240E2FF
:1009300065E477E18C2FB7DD8091361482FD12C01B
:1009400020E030E040E251E4609111147091121403
:1009500080911314909114140E94D4CC87FD7BC015
:1009600003E03AC160912B1470912C1480912D14E6
:1009700090912E14A70196010E94C7D0232B242BFF
:10098000252BF1F633DF82E796E870C1D13081F58F
:1009900020916D02222391F0A70196010E94C7D0F9
:1009A000213031054105510519F42AEF4EE302C00B
:1009B0002AEF40E26EE377E18C2F75DD80913614EB
:1009C00082FFBECF60912B1470912C1480912D1456
:1009D00090912E14A70196010E94C7D021303105B5
:1009E0004105510509F0ACCF01DF8BE298E93EC12A
:1009F000D23009F0A5CF20916D02222391F0A701FA
:100A000096010E94C7D0223031054105510519F4E5
:100A10002AEF4EE302C02AEF40E267E377E18C2F32
:100A200042DD8091361482FF8BCF60912B14709140
:100A30002C1480912D1490912E14A70196010E94E0
:100A4000C7D0223031054105510509F079CFCEDEFE
:100A50008EE797E90BC1D33031F08091AD0980FD6D
:100A600039C004E072C080916D028823D1F060919A
:100A70002B1470912C1480912D1490912E14A70199
:100A800096010E94C7D0233031054105510519F464
:100A90002AEF4EE302C02AEF40E260E377E18C2FB9
:100AA00002DD8091361482FFD8CF60912B147091B3
:100AB0002C1480912D1490912E14A70196010E9460
:100AC000C7D0233031054105510539F68FDE8FEA55
:100AD00095E9CCC0D43011F005E037C080916D02AB
:100AE0008823D1F060912B1470912C1480912D14D7
:100AF00090912E14A70196010E94C7D02430310591
:100B00004105510519F42AEF4EE302C02AEF40E2F5
:100B100065E277E18C2FC7DC8091361482FFDCCF51
:100B200060912B1470912C1480912D1490912E149F
:100B3000A70196010E94C7D0243031054105510517
:100B400059F654DE8BEF96E991C08091AD0981FF93
:100B500043C00D1711F00F5F3FC080916D028823D5
:100B6000F1F060912B1470912C1480912D149091C0
:100B70002E14A70196010E94C7D0802F90E0A0E01C
:100B8000B0E0281739074A075B0719F42AEF4EE34C
:100B900002C02AEF40E26AE177E18C2F84DC809189
:100BA000361482FFD8CF60912B1470912C14809151
:100BB0002D1490912E14A70196010E94C7D0802F6A
:100BC00090E0A0E0B0E0281739074A075B0719F664
:100BD0000DDE85E796E94AC060912B1470912C14C4
:100BE00080912D1490912E14A70196010E94C7D0D8
:100BF000802F90E0A0E0B0E0281739074A075B0794
:100C00008CF025E0029FC00111240197AA2797FDCF
:100C1000A095BA2F80932B1490932C14A0932D148D
:100C2000B0932E1460912B1470912C1480912D147C
:100C300090912E14A70196010E94C7D0809135147F
:100C400090E00496422F50E0841795074CF48CEF07
:100C5000820F8093351410936D02DBEFD20FCFEF2C
:100C6000CF5FDF5FC53008F448CE0CC090936F02B1
:100C700080936E0210922B1410922C1410922D144B
:100C800010922E14DF91CF911F910F91FF90EF9052
:100C9000DF90CF9008958DEC9CECACECBDE380939D
:100CA000111490931214A0931314B0931414D3CD71
:100CB00080E090E0A0E8BFE38093111490931214B9
:100CC000A0931314B0931414C6CD80E090E0A0E27A
:100CD000B1E48093111490931214A0931314B09361
:100CE0001414B9CD8F929F92AF92BF92CF92DF92A0
:100CF000EF92FF921F93CF93DF9380912B149091EB
:100D00002C14A0912D14B0912E1481309048A1057F
:100D1000B10544F010922B1410922C1410922D1443
:100D200010922E1480912B1490912C14A0912D14BC
:100D3000B0912E14B7FF08C010922B1410922C14EF
:100D400010922D1410922E1460912B1470912C146B
:100D500080912D1490912E1425E030E040E050E079
:100D60000E94C7D08091351490E0A0E0B0E0281731
:100D700039074A075B0714F420933514D0913514D2
:100D8000C0E025E0C22ED12CE12CF12C33E1832EE2
:100D9000912CA12CB12C11E060912B1470912C148A
:100DA00080912D1490912E14D1112AC020916D02A2
:100DB000222389F0A70196010E94C7D0232B242B60
:100DC000252B19F426E246E202C026E240E26CEF4F
:100DD00076E18C2F68DB8091361482FF2EC0609103
:100DE0002B1470912C1480912D1490912E14A70126
:100DF00096010E94C7D0232B242B252BF1F4D1C0C0
:100E0000D13009F045C020916D02222391F0A70155
:100E100096010E94C7D0213031054105510519F4D2
:100E20002AEF4EE302C02AEF40E262EF76E18C2F18
:100E30003ADB8091361482FD16C080912B1490917C
:100E40002C14A0912D14B0912E144497A105B10536
:100E50000CF483C080922B1490922C14A0922D1429
:100E6000B0922E147AC060912B1470912C14809142
:100E70002D1490912E14A70196010E94C7D0213005
:100E8000310541055105C9F6B1DC85E696E88CC00F
:100E9000D23081F520916D02222391F0A7019601B5
:100EA0000E94C7D0223031054105510519F42AEFBF
:100EB0004EE302C02AEF40E269EE76E18C2FF3DACE
:100EC0008091361482FFB9CF60912B1470912C144D
:100ED00080912D1490912E14A70196010E94C7D0E5
:100EE000223031054105510509F0A7CF7FDC88E5A7
:100EF00096E85AC0D33009F0A0CF20916D0222238A
:100F000091F0A70196010E94C7D023303105410519
:100F1000510519F42AEF4EE302C02AEF40E26EEDCC
:100F200076E18C2FC0DA8091361482FF86CF6091F3
:100F30002B1470912C1480912D1490912E14A701D4
:100F400096010E94C7D0233031054105510509F0B3
:100F500074CF4CDC8BE496E827C060912B14709121
:100F60002C1480912D1490912E14A70196010E94AB
:100F7000C7D08091351490E00496422F50E084173A
:100F800095074CF48CEF820F8093351410936D020B
:100F9000DBEFD20FCFEFCF5FDF5FC53008F4FCCEC1
:100FA0000FC024DC84ED93EA90936F0280936E026D
:100FB00010922B1410922C1410922D1410922E14A7
:100FC000DF91CF911F91FF90EF90DF90CF90BF9076
:100FD000AF909F908F9008952091AD0920FF08C099
:100FE00080918A1490918B14909302148093011431
:100FF00021FF08C080918A1490918B14909304145F
:10100000809303148091B309811108C080918814E2
:1010100090918914909300148093FF13809186140B
:101020009091871490931809809317090E94028069
:101030000C94FA792091AD0920FF08C080918414A6
:1010400090918514909302148093011421FF08C09D
:1010500080918414909185149093041480930314C8
:101060008091B309811108C08091821490918314FA
:10107000909300148093FF138091801490918114B9
:1010800090931809809317090E9402800C94FA79B2
:101090007F928F929F92AF92BF92CF92DF92EF9208
:1010A000FF920F931F93CF93DF93209131072F5F10
:1010B000209331078AE0289FE001112430E08091DD
:1010C0003607909137072817390720F48E01065FFD
:1010D0001F4F06C000913807109139070C0F1D1FD4
:1010E00041EEE42E4AE0F42E53E3C52E53E1D52E13
:1010F00064E1762E7AE0A72EB12CE6E38E2EE3E1B2
:101100009E2EC017D10708F051C060913207709130
:101110003307615071096C1B7D0B70933507609329
:10112000340780ED9AE00E9496588091A40A8823A3
:10113000F1F0FF92EF929F928F921F927F92CE01D9
:10114000B5010E947ED0789E9001799E300D1124C9
:101150002759394F3F932F930E94ACD48DB79EB738
:1011600008960FB6F8949EBF0FBE8DBF1DC0FF92AC
:10117000EF92DF92CF921F927F92CE01B5010E9433
:101180007ED0789E9001799E300D11242759394FD9
:101190003F932F930E94ACD48DB79EB708960FB69D
:1011A000F8949EBF0FBE8DBF2196ABCF8BE49CE819
:1011B00090936F0280936E0210922B1410922C1455
:1011C00010922D1410922E14DF91CF911F910F9138
:1011D000FF90EF90DF90CF90BF90AF909F908F9057
:1011E0007F9008957F928F929F92AF92BF92CF92FD
:1011F000DF92EF92FF920F931F93CF93DF93209193
:1012000031072150209331078AE0289FE001112403
:1012100030E080913607909137072817390720F47E
:101220008E01065F1F4F06C00091380710913907E5
:101230000C0F1D1FF1EEEF2EFAE0FF2EACE2CA2ECE
:10124000A3E1DA2EB4E17B2E8AE0A82EB12C9FE236
:10125000892E93E1992EC017D10708F051C06091F3
:10126000320770913307615071096C1B7D0B7093CD
:1012700035076093340780ED9AE00E94965880917C
:10128000A40A8823F1F0FF92EF929F928F921F920F
:101290007F92CE01B5010E947ED0789E9001799E0A
:1012A000300D11242759394F3F932F930E94ACD40E
:1012B0008DB79EB708960FB6F8949EBF0FBE8DBF30
:1012C0001DC0FF92EF92DF92CF921F927F92CE01CC
:1012D000B5010E947ED0789E9001799E300D112438
:1012E0002759394F3F932F930E94ACD48DB79EB7A7
:1012F00008960FB6F8949EBF0FBE8DBF2196ABCF58
:101300008BE49CE890936F0280936E0210922B14F2
:1013100010922C1410922D1410922E14DF91CF9154
:101320001F910F91FF90EF90DF90CF90BF90AF9003
:101330009F908F907F900895EF92FF920F931F934D
:10134000CF93DF93CDB7DEB76E970FB6F894DEBFBD
:101350000FBECDBF8091AC098E3021F48AE793E1B6
:101360000E94E71A85EA9AE00E941F2660913B07D7
:1013700070913C0777FD29C080ED9AE00E94965855
:101380008091BF0A9091C00A01969093C00A809301
:10139000BF0A1092C50A84ED9AE09F938F9383E76A
:1013A00093E19F938F938E010F5F1F4F1F930F93B6
:1013B0000E94E8D40F900F900F900F900F900F9015
:1013C0007E0185E0E80EF11C0BC08FEF9FEF90933C
:1013D000C00A8093BF0A85EA9AE00E94222616C0BE
:1013E000F7018081882349F0992787FD90950E9415
:1013F000ADD3F70181937F01F3CFC8010E94741A26
:101400008FE693E10E94E71A0E9402806E960FB663
:10141000F894DEBF0FBECDBFDF91CF911F910F912A
:10142000FF90EF9008955F926F927F928F929F92BC
:10143000AF92BF92CF92DF92EF92FF920F931F93E2
:10144000CF93DF938091D30A882309F438C1809128
:101450006D02811104C08091361482FF30C18091E9
:10146000AC098E3011F41092A40A8091A40A88234A
:1014700011F18FEF9FEF90933C0780933B07909380
:101480003E0780933D079093400780933F079093DA
:10149000420780934107909344078093430710923B
:1014A000AE0A1092AF0A1092B00A1092B10A90934D
:1014B000C00A8093BF0A80ED9AE00E94EC58909396
:1014C00033078093320790933507809334072AE0DF
:1014D00030E0B9010E947ED07093370760933607E1
:1014E000009729F090933907809338070DC0611554
:1014F0007105C1F3309339072093380761507109A2
:1015000070933707609336078091360790913707BD
:10151000892B29F4609038077090390703C07AE06E
:10152000672E712C1092310764ED7AE084E29BE023
:101530000E940B448091D40A8F32C1F410923A0772
:10154000C0E0D0E001EE1AE02AEDE22E24E0F22E17
:1015500034E1532E4AE0C42ED12C54EDA52E5AE08E
:10156000B52E69ED862E64E0962E3BC081E0809317
:101570003A07E6CF609132077091330761507109E5
:101580006C1B7D0B709335076093340780ED9AE0F8
:101590000E9496589091A40A8091E10A992309F437
:1015A00042C0811122C0BF92AF929F928F921F9230
:1015B0005F92CE01B6010E947ED0589E9001599E46
:1015C000300D11242759394F3F932F930E9470D427
:1015D0008DB79EB708960FB6F8949EBF0FBE8DBF0D
:1015E0002196C615D70531F65CC01F930F939F92C5
:1015F0008F921F925F92CE01B6010E947ED0589EBC
:101600009001599E300D11242759394F3F932F9344
:101610000E9470D48DB79EB708960FB6F8949EBFFF
:101620000FBE8DBFDDCF81111EC0BF92AF92FF9262
:10163000EF921F925F92CE01B6010E947ED0589E1B
:101640009001599E300D11242759394F3F932F9304
:101650000E9470D48DB79EB708960FB6F8949EBFBF
:101660000FBE8DBFBDCF1F930F93FF92EF921F92BE
:101670005F92CE01B6010E947ED0589E9001599E85
:10168000300D11242759394F3F932F930E9470D466
:101690008DB79EB708960FB6F8949EBF0FBE8DBF4C
:1016A0009FCF8BE49CE890936F0280936E02109220
:1016B0002B1410922C1410922D1410922E14DF91D2
:1016C000CF911F910F91FF90EF90DF90CF90BF903F
:1016D000AF909F908F907F906F905F900895CF9381
:1016E000DF93C1E0D0E0D0937B14C0937A1489E0FB
:1016F00090E090937D1480937C146DED74E087E30B
:1017000094E10E9450C8D0937B14C0937A1486E170
:1017100090E090937D1480937C146EEE74E087E3E8
:1017200094E10E9450C869EF74E087E394E10E945D
:1017300050C8D0937B14C0937A1483E290E09093C6
:101740007D1480937C146FEF74E087E394E10E9432
:1017500050C8D0937B14C0937A1480E390E09093A8
:101760007D1480937C1461E175E087E394E10E942D
:1017700050C8D0937B14C0937A148DE390E090937B
:101780007D1480937C1466E275E087E394E10E9407
:1017900050C88091361482FF10C08091AC098E3001
:1017A00019F48FE491EA02C084ED93EA90936F02FA
:1017B00080936E02DF91CF9119C8DF91CF91089588
:1017C000EF92FF920F931F93CF93DF93C1E0D0E08E
:1017D000D0937B14C0937A1489E090E090937D14A9
:1017E00080937C1462E375E087E394E10E9450C823
:1017F000D0937B14C0937A1483E190E090937D148E
:1018000080937C146EE375E087E394E10E9450C8F6
:10181000D0937B14C0937A148DE190E090937D1463
:1018200080937C1463E575E087E394E10E9450C8DF
:10183000EDEEEE2EE2E2FE2E00E210E024E030E0DB
:101840004EE150E060E370E08BE394E10E94A6BDBE
:101850008091361482FF18C08EE08093AC091092FC
:10186000CB0A8BE080936C0984E99BE990936F022B
:1018700080936E020E94F68310922B1410922C1407
:1018800010922D1410922E14DF91CF911F910F9171
:10189000FF90EF9008952F923F924F925F926F9238
:1018A0007F928F929F92AF92BF92CF92DF92EF92F0
:1018B000FF920F931F93CF93DF93CDB7DEB7AC9713
:1018C0000FB6F894DEBF0FBECDBF80916D028111BF
:1018D00004C08091361482FFEFC3209131078AE063
:1018E000289FA001112459A348A330E08091360716
:1018F000909137072817390730F448A059A02AE0FB
:10190000420E511C08C0409038075090390748A13A
:1019100059A1440E551E80912B1490912C14A09126
:101920002D14B0912E1481309048A105B10544F0DA
:1019300010922B1410922C1410922D1410922E141D
:1019400080912B1490912C14A0912D14B0912E14F1
:10195000B7FF08C010922B1410922C1410922D1463
:1019600010922E1460912B1470912C1480912D14D0
:1019700090912E1425E030E040E050E00E94C7D066
:101980008091351490E0A0E0B0E0281739074A07AD
:101990005B0714F420933514609035141F8E712C5E
:1019A000B5E0CB2ED12CE12CF12C1AE0212E312CDC
:1019B0008091310781113AC0662029F08091A40AF4
:1019C00081116DC0ABC080916D028823D1F0609110
:1019D0002B1470912C1480912D1490912E14A7012A
:1019E00096010E94C7D0232B242B252B19F426E225
:1019F00046E202C026E240E26AE673E1872D0E94D9
:101A000053828091361482FFD9CF60912B1470914C
:101A10002C1480912D1490912E14A70196010E94F0
:101A2000C7D0232B242B252B49F636C36110C6CFF4
:101A300080916D028823D1F060912B1470912C1449
:101A400080912D1490912E14A70196010E94C7D069
:101A5000232B242B252B19F420E24EE302C020E295
:101A600040E261E673E1872D0E9453828091361433
:101A700082FFA4CF60912B1470912C1480912D14AF
:101A800090912E14A70196010E94C7D0232B242BDE
:101A9000252B09F093CF0E94F683A4DB0DC38F8D15
:101AA000853008F01F8E9F8DE92FF0E0EE0FFF1FAD
:101AB000E55CF84F2081318137FD2DC080913807DA
:101AC00090913907D101A81BB90BCD01820F931F4B
:101AD000B1010E947ED0772740913107809136076F
:101AE00090913707841B910968177907A1F48091B9
:101AF0003207909133070197821B930BB1010E942B
:101B00007ED0B4E1B89FF001B99FF00D1124E759E0
:101B1000F94F2AE220833F8D3F5F3F8F4CE0749E58
:101B2000C0011124DC011396BFA3AEA3FC013C96B7
:101B3000F9A7E8A7872D90E001964CE0489F900117
:101B4000499F300D11243BA72AA788A099A011E036
:101B500051E0560D5CA7862D90E0A0E0B0E08AA38E
:101B60009BA3ACA3BDA38414950408F0D3C08091BB
:101B70003207909133070197881999099093350797
:101B8000809334071611C1C080916D02882309F437
:101B9000A1C060912B1470912C1480912D14909100
:101BA0002E14A70196010E94C7D08AA19BA1ACA1C7
:101BB000BDA1281739074A075B0709F055C0C401C2
:101BC000B1010E947ED0A4E1A89F5001A99FB00C52
:101BD0001124F501E759F94F5F0180818111138AC2
:101BE00061E08BE394E10E94FDC20CE010E020E88C
:101BF00030E04EA15FA160E070E08BE394E10E94D1
:101C000054C560E08BE394E10E94FDC210927B1406
